:100000000C9498400C943D410C943D410C943D411E
:100010000C943D410C943D410C943D410C943D4168
:100020000C943D410C943D410C943D410C943D4158
:100030000C943D410C9486430C943D410C943D41FD
:100040000C943D410C943D410C943D410C943D4138
:100050000C943D410C943D410C943D410C943D4128
:100060000C943D410C943D410C943D410C943D4118
:100070005A5501200201003808000000000000006D
:1000800000000000009F48AD487D49214D0D4DB056
:1000900048BF48CE48F54CDC48EA4800408891D239
:1000A000E4ADB5B6BEBFFFFFFFFFFF00000000FFDD
:1000B000FF0000F6F6F6F6FF00F6F6F6F6F6F6FFA7
:1000C00000F6F62727272700F6F6272727272700F9
:1000D000F6F6272727272700F6F6272727272700C2
:1000E000F6F6272727272700000000FFFFFFFFF66F
:1000F000F6F6F60000FFFFF6F6F6F6F6F600FF2736
:10010000272727F6F600FF2727272727F6F60027B9
:1001100027272727F6F6002727272727F6F6002781
:1001200027272727F6F600FFFFFFFFFFFFFFFFFF50
:10013000FFFFFFFFFFFFFFFFFFFFFFFFFFFFFFFFCF
:10014000FFFFFFFFFFFFFFFFFFFFFFFFFFFFFFFFBF
:10015000FFFFFFFFFFFFFFFFFFFFFFFFFFFFFFFFAF
:10016000FFFFFFFFFFFFFF0000000000000000F6A0
:10017000F6F6F6F6F6F6F6F6F6F6F6F6F6F6F627EE
:1001800027272727272727272727272727272727FF
:1001900027272727272727272727272727272727EF
:1001A0002727272727272700F6F62727272727008F
:1001B000F6F6272727272700F6F6272727272700E1
:1001C000F6F6272727272700F6F6272727272700D1
:1001D000F6F6272727272700F6F6272727272700C1
:1001E000F6F627272727272727272727F6F600278A
:1001F00027272727F6F6002727272727F6F60027A1
:1002000027272727F6F6002727272727F6F6002790
:1002100027272727F6F6002727272727F6F6002780
:1002200027272727F6F600272727272727272727E7
:10023000272727272727272727272727272727274E
:10024000272727272727272727272727272727273E
:1002500027272727F6F6F62727272727F6F6F62754
:1002600027272727F6F600272727272727272727A7
:10027000272727272727272727272727272727270E
:10028000272727272727272727272727272727F62F
:10029000F6F6F6F6F6F6F6F6F6F6F6F6F6F6F600F4
:1002A00000000000000000272727272727272727EF
:1002B00027272727272727272727272727272727CE
:1002C000272727272727272727272727272727F6EF
:1002D000F6F62727272727F6F6F6272727272700CA
:1002E000F6F627272727272727272727F6F6002789
:1002F00027272727F6F6F62727272727F6F6F627B4
:10030000272727272727272727272727272727277D
:10031000272727272727272727272727272727276D
:100320002727272727272700F6F62727272727F617
:10033000F6F62727272727F6F6F627272727272742
:10034000272727272727272727272727272727273D
:10035000272727272727272727272727272727272D
:100360002727272727272700F6F6272727272700CD
:10037000F6F6272727272700F6F62727272727001F
:10038000F6F62727272727FF00F6F627272727FF38
:1003900000F6F6F6F6F6F6FFFF0000F6F6F6F6FFC4
:1003A000FFFFFF000000002727272727F6F600277A
:1003B00027272727F6F6002727272727F6F60027DF
:1003C00027272727F6F60027272727F6F600FFF628
:1003D000F6F6F6F6F600FFF6F6F6F60000FFFF007A
:1003E000000000FFFFFFFF010203030303010404F9
:1003F00004040402050603030303050708080809AB
:1004000006050603030303050603030305060506A5
:10041000030303030506030303050605060303039D
:100420000305060303030506050603030303050688
:10043000030303050605060303030305060303037D
:100440000506050603030303050603030305060566
:100450000A04040402050A0404040B060C08080834
:10046000080D0C08080808080D0000000000000036
:10047000000303030300190303030303030003033F
:100480000303030303000303030000000000000054
:10049000000019030303030303000303030303031F
:1004A0000300030303030303030000000000000034
:1004B000000003000300100003030003000000031A
:1004C0000000030003000300030000000000000020
:1004D00000001000030003000300000300030003FA
:1004E00000000300030003000300000000FFFFFF03
:1004F000FF0303FF9F9F9F9F9F03FF9F0300030333
:1005000003039F030300030303FF9F000000000099
:1005100000FF9F030303030303FF9F03030303037E
:1005200003FF9F030303030303FFFFFFFF0000001C
:10053000009F9F9F9F9FFF030303030303009FFFF1
:10054000030303030300039F030000000000009F58
:10055000FF002A030303039FFF0003030303039F1A
:10056000FF0003030303039FFFFF9F000000000041
:1005700000FF9F0303002A0303FF9F0303000303FD
:1005800003FF9F030300030303009F00000000001C
:100590000000FF9F03030303030003FF9F9F9F9F30
:1005A0009F00030303FFFFFFFF0000000000009F08
:1005B000FF03030303002A9FFF0303030300039FBA
:1005C000FF0303030300039FFF0000000000009FE0
:1005D00000002A0303039FFF039F9F9F9F9FFF032A
:1005E00003FFFFFFFF0303030313B713B7B7B7B747
:1005F000B713B713B7B7B7B7B713B71313131313AB
:100600001313B713D8D8D8D8D813B713B7B7B7B709
:10061000B713B713B7B7B7B7B713B713131313138A
:100620001313B713D8D8E0D8D8B7B7B7B7B713B73D
:1006300013B7B7B7B7B713B713131313131313B70E
:1006400013D8D8D8E0D813B713B7B7B7B7B713B71D
:1006500013B7B7B7B7B713B713131313131313B7EE
:1006600013D8D8D8D8D813B71313131313131313DD
:1006700013B7B7B7B7B7B7B7B7131313131313132A
:1006800013D813B7B7D813B7B7D813B7B7D813B7AA
:10069000B7E013B7B7D813B7B7D813B7B7D813B7EE
:1006A000B7D813B7B7D813B7B7D813B7B7D813B7E6
:1006B000B7D813B7B7D813B7B7E013B7B7D813B7CE
:1006C000B7D813B7B7D813B7B7D813B7B7D813B7C6
:1006D000B71313131313131313B7B7B7B7B7B7B7CA
:1006E000B7131313131313131300000000000000BB
:1006F00000030303B7B7B7B7B70303B7B72A2A2A6C
:100700002A03B7B72A0000000000B72A0000000043
:100710006400B72A000000B7B700B72A0000B7B7D7
:10072000B700B72A0064B7B7B700000000000000A8
:1007300000B7B7B7B7B70303032A2A2A2AB7B70304
:1007400003000000002AB7B70064000000002AB7C9
:1007500000B7B70000002AB700B7B7B700002AB744
:1007600000B7B7B764002AB70000B72A0064B7B76C
:10077000B703B72A0000B7B7B703B72A000000B71E
:10078000B703B72A000000006400B7B72A000000D2
:10079000000003B7B72A2A2A2A000303B7B7B7B75E
:1007A000B70003030300000000B7B7B764002AB71F
:1007B00000B7B7B700002AB700B7B70000002AB7E4
:1007C0000064000000002AB700000000002AB7B74C
:1007D000002A2A2A2AB7B70000B7B7B7B7B7000070
:1007E0000300000000000003030000000000000000
:1007F00000030303B7B7B7B7B70303B7B72A2A2A6B
:100800002A03B7B72A0000000000B72A0000000042
:100810000000B72A000000000000B72A0000000016
:100820000000B72A000000000000000000000000E7
:1008300000B7B7B7B7B70303032A2A2A2AB7B70303
:1008400003000000002AB7B70000000000002AB72C
:100850000000000000002AB70000000000002AB7D6
:100860000000000000002AB70000B72A00000000C6
:100870000003B72A000000000003B72A00000000B0
:100880000003B72A000000000000B7B72A000000EC
:10089000000003B7B72A2A2A2A000303B7B7B7B75D
:1008A000B7000303030000000000000000002AB7A7
:1008B0000000000000002AB70000000000002AB776
:1008C0000000000000002AB700000000002AB7B7AF
:1008D000002A2A2A2AB7B70000B7B7B7B7B700006F
:1008E00003000000000000030300000000000000FF
:1008F00000030303030019030300FF00000084004A
:1009000000FFFF00C785FF00C7FFFF00FF85FF0056
:10091000FFFFFF00FF85FF00FFFFFF008585FF0051
:1009200085FFFF008585FF008500000000000000B6
:10093000000303030300190303000084000000FF09
:10094000008500FF85C700FFFF8500FF85FF00FFD2
:10095000FF8500FF85FF00FFFF8500FF858500FF05
:10096000FF8500FF858500FFFFFFFF000000FF00FF
:100970000000FFFFFFFFFFFFFFFF0000000000007F
:1009800000FFFFFFFFFFFF0000FF00000000FF006F
:1009900000FF00858500FFFFFFFF0085858500FFC4
:1009A0000000FFFFFFFFFFFFFF0000FF000000FF50
:1009B000FFFFFFFFFFFFFFFF00000000000000003F
:1009C000FF0000FFFFFFFFFFFF0000FF000000002F
:1009D000FFFFFFFF00858585FF00FF00858585857A
:1009E000FFFFFFFFFFFFFFFF0000FF00000085008B
:1009F00000FFFF008585FF0085FFFF00A7A7FF0020
:100A0000A7FFFFFFFFFFFFFFFFFFA70000000000A1
:100A1000000000A700000000EFFFFF00FFFFFFFF46
:100A2000A7FF09000900EFA7FF000085000000FFF5
:100A3000008585FF008585FFFFA7A7FF00A7A7FF0B
:100A4000FFFFFFFFFFFFFFFFFF000000000000A708
:100A5000FFEF00000000A70000A7FFFFFFFF00FF5F
:100A6000FFFFA7EF00090009FFFF000900EFA7FF44
:100A7000FFFF5B00EFEFFFFFFFFF030303EFA7FFA5
:100A8000FFFFFFFFFFFFEFA7FFFF00000000FF00D9
:100A9000A7FF00858500FFFFEFFF0085858500FF2C
:100AA0000000FFFFFFFFFFFFFFFFFFA7EF000900B0
:100AB000FFFFFFFFEFEF005BFFFFFFA7EF03030365
:100AC000FFFFA7EFFFFFFFFFFFA700FF00000000F1
:100AD000FFEFFFFF00858585FF00FF008585858589
:100AE000FFFFFFFFFFFFFFFF002A2A2A2A2A2A2AE8
:100AF0002A132A2AB72A2A2AB72A2A2AB713B71367
:100B00002A2AB72A2A2A2A2A2A2AB7132A2A2A2A42
:100B10002A2A2A2A2A2A2AB72A2A2A2A2AB713B7A5
:100B2000132A2A2A2A2A2A2A2A002A002A002A00E4
:100B30002A13002A002A002A00002A00B700B70062
:100B40002A2A002A002A002A0000B7002A002A00C8
:100B50002A2A002A002A00B700002A002A001300CF
:100B6000132A002A002A002A0013B7B713B7B7B711
:100B7000B7B7B7B7B7B7B713B7B71313B7B7B7B7F1
:100B8000B7B7B7B7B713B7B7B7B7B713B7B7B7B73D
:100B90001313B7B7B7B7B7B7B7B7B7B7B71313B775
:100BA00013B7B713B7B7B7B7B700B7001300B7009D
:100BB000B7B700B700B7001300001300B700B700C5
:100BC000B7B700B7001300B70000B700B700B70011
:100BD000131300B700B700B70000B700B700130049
:100BE00013B7001300B700B7000000000000FFFFBC
:100BF0000003030019191919190300FF1919190025
:100C00001900191919001919191919191919191986
:100C1000FFFF190019FF19001919191919191919C4
:100C2000190019191900191919FF191900000000E4
:100C300000191919191900030319001919190000CD
:100C400003191919001919190019001919001900A7
:100C50001919191919190019191919001900190068
:100C60001919191900190019001919001900191971
:100C700000001900191900191903031900001900BF
:100C80001903030303000000000000000000FF0040
:100C9000FF000303030000FFFF0003030303000042
:100CA00000000303030303030319190019191900B2
:100CB0001900001919000019001919000019000085
:100CC00000000000000000000000FFFF0000000026
:100CD0000000FF000000000003000000000003030C
:100CE000030003030303030303000000000000FFED
:100CF0000000030019001900190300FF001900008B
:100D0000000019001900190019190019001900191B
:100D1000000019001900190019190019001900190B
:100D2000000019001900190019190000000000192D
:100D3000000019001900000019030019000000004C
:100D40000000030003000000FF000000000000FF9F
:100D5000000003000300FF00FF0000030003000089
:100D60000000030003000300030019FFFFFFFFFF63
:100D7000F619FF19191919191919FF19000000009E
:100D80000019FF1900FF00000019FF1900F600000C
:100D90000019FF19000000190019FF1900001900BF
:100DA0001919FF190019001900F6FFFFF6FFFF19C6
:100DB00000191919191919FF19000000000000F68F
:100DC00019000019190000F619000019190000FF98
:100DD000190019FFF61900FF1919FFFF19FF00F696
:100DE000190019F6FF1900FF1919FF19031919192C
:100DF0001919FF19030319FF191919FFFFFFFFFF45
:100E0000FF19FF19190019031919FF1919001903FE
:100E10001919FF19001900190300FF030003190332
:100E2000000019FFFFFFF6FFFF191919191900FF3C
:100E3000191919FFF61919FF19FFFFFFFFFFFFFF2F
:100E400019190319001900191919031900190019A2
:100E500019031900190319FF19000319030003FFEF
:100E600000FFFFFFFFF6F61900000000000000BFC2
:100E7000BF03030303BFBFBFBF0303BFBFBFBFBFEA
:100E8000BF03BFBFBFBFBFBFBF00BFBFBFBFBFBFED
:100E9000BFBFBFBFBFBFBFBF16BFBFBFBF16BF165D
:100EA000BFBF16BF16BFBFBF16BFBFBF0000000049
:100EB0000016BFBFBF00030303BFBF16BFBF0303BE
:100EC00003BFBFBFBFBFBF0303BFBF16BF16BFBFB8
:100ED00000BF16BFBFBFBFBFBF16BFBF16BFBFBFDC
:100EE00016BFBF16BFBFBF03BFBFBFBF16BFBFBFC9
:100EF0001616BFBFBFBFBFBFBFBFBFBFBFBF16BFFD
:100F0000BFBF16BFBF1616BF1600BF16BF16BFBFA6
:100F1000BF0003BF16BF16BF16000303001600165E
:100F200000000303030303030316BFBFBF1603162A
:100F3000161616BF16BF160300BF1616BF160316E9
:100F40000016BFBFBF03160300BF16BF031603166C
:100F500000161603160316000016001600160000F1
:100F6000000303000000000003000000000000BFB9
:100F7000000003000300BF00BF0300BF00BF00BFAD
:100F80000000BF00BF00BF00BF0000BF00BF00BF28
:100F90000000BF00BF00BF0016BF00BF0016001654
:100FA000000016001600BF0016BF00BF00BF00BF44
:100FB0000000BF00BF00BF00BFBF00BF00BF00BF39
:100FC00000001600BF00160016000016001600BF35
:100FD000000003001600160016000003001600169D
:100FE00000000300030003000300BF16BFBFBFBF24
:100FF000BFBF16BFBFBFBFBFBF16BFBFBFBFBFBF53
:10100000BFBF16BFBFBFBFBFBF16BF16BFBFBFBFEB
:10101000BFBF16BF16BF16BF1603BF16BF16BF163B
:10102000160316161616161616BFBFBFBFBFBF0093
:1010300000BFBFBFBFBFBFBF00BFBFBFBFBFBF16E7
:1010400000BFBFBFBFBF161600BFBFBFBF16BF16D2
:1010500000BF16BF16BF1616001616161616160374
:101060000003031603030303001616BF1616161615
:1010700016BF16161616161616031616161616167A
:101080001600030303030303030300000000000032
:10109000031616161616160300161616161616162C
:1010A000001603160316030300161616161603037E
:1010B000001616161603160300160316031603036E
:1010C000000303030303030000000000000000030B
:1010D000030316161616161616BF1616161616162D
:1010E000160316161616161616030303030303003B
:1010F000000000000000000000BF161616161616AD
:101100001616031603160316030303030303030350
:1011100003000000000000000303030303030316A1
:1011200000000300030003000000030303030303A4
:101130000300000000000000001616161616160325
:10114000001603160316030300030303030303033C
:101150000000000000000000001616031603030341
:1011600003000300030003000303BFBF16BF160004
:1011700000BFBFBFBF16BF1600BFBFBFBFBF16BFF8
:1011800000BFBFBFBFBFBF1600BFBFBFBFBF16BF3F
:1011900000BFBFBFBFBFBF1600BFBFBFBFBF16BF2F
:1011A00000BFBFBFBF16BF1600BFBFBFBF16BF1671
:1011B00000BFBFBFBFBF161600BFBFBFBF16BF1661
:1011C00000BFBFBFBFBF161600BFBFBFBF16BF1651
:1011D00000BFBFBF16BF16160003BFBF161616030B
:1011E00000000303030303030000BFBFBF16BF00DB
:1011F00000BFBFBFBFBF161600BFBFBFBF16BF1621
:1012000000BFBFBFBFBF161600BFBFBFBF16BF1610
:1012100000BFBFBF16BF16160000BFBF16161600D0
:10122000000000000000000000001616161616034D
:101230000300161616160316030000031603160302
:10124000030000030303030300000000000000008C
:1012500003000000161616161600000016161616C5
:101260001600000000161616160000030003030304
:10127000030000000000000000000000000016163F
:101280000300000000001603030000000003000339
:10129000030000000000000000000000000000004B
:1012A0000300000000000000001616000303030303
:1012B000031600BFBFBFBFBFBF00BFBFBFBFBFBF21
:1012C000BFBFBFBF0000000000BFBF001616001662
:1012D00016BF00161616001616BF001616160016B4
:1012E00016BF0003030300030303030303030016F5
:1012F00016BFBFBFBFBFBF0016BFBFBFBFBFBFBF0F
:10130000000000000000BFBFBF161600161600BF89
:10131000BF16160016161600BF1616001616160073
:10132000BF0303000303030016BF0000000000001A
:1013300000BF00BFBFBF001616BF00BF16030016D8
:1013400016BF00BF1603001616BF00BF030300033D
:1013500003BF00000000000000160016161600165D
:101360001616000303030003030000000000000042
:101370001616160016161600161616001616160065
:1013800016161600161616001603030003030300B4
:1013900016000000000000001616160016161600B3
:1013A00003030300030303000316161616161603A1
:1013B00003161600000000000016000000000000E8
:1013C000000000000000000000000000000000001D
:1013D0000000030000000300000300000000000004
:1013E000000003000300030003001616BF161616C4
:1013F00016000000000000161600000000000000AB
:1014000016000000000000000000000000000000C6
:1014100000030300000000000003030000000000C0
:10142000001616000303000000000000000000008A
:101430000000030003000300030300030000000397
:101440000000030003000300030000000000000090
:101450000000030003000300030000030003000377
:10146000000003000300030003161600030300003E
:1014700000BFBF001616000300BFBF001616000312
:1014800000BFBF00BFBF001600BFBF00BFBF001638
:1014900000BFBF00BFBF00BF000000000000000091
:1014A0000000030003000300000000000000000033
:1014B00000000303FFFFFFFFFF0003FFFFFFFFFF2D
:1014C000FF00FFFFFF0000000000FFFF0000858518
:1014D0008500FFFF0085FFFF8500FFFF00FFFFFF86
:1014E000FF00FFFF00FFFFFFFF0000000000000003
:1014F00000FFFFFFFFFF000303FFFFFFFFFFFF00F1
:101500000300000000FFFFFF008585858500FFFFC9
:101510000085FFFF8585FFFF00FFFFFFFF85FFFFC1
:1015200000FFFFFFFF85FFFF0000FFFF0085FFFFBB
:10153000FF03FFFF008585FFFF03FFFF0085858513
:10154000FF03FFFFFF008585850085FFFFFFFFFF8D
:10155000FF000085FFFFFFFFFF00030085858585F5
:10156000850003030000000000FFFFFF8585FFFFEB
:1015700000FFFF858585FFFF00FF85858585FFFFCF
:101580000085858585FFFFFF00FFFFFFFFFFFF85CB
:1015900000FFFFFFFFFF8500008585858585000032
:1015A000030000000000000303D8E8D8D8D8D8D83A
:1015B000D8D8E8D8D8D8D8D8D8D8E8D8D8D8D8D88B
:1015C000D8E8D8E8E8D8D8D8D8D8D8D8D8E8D8D85B
:1015D000D8D8D8D8D8D8E8D8E8D8D8D8D8E8D8E84B
:1015E000E8E8D8E8D8D8D8D8D8D8D8D8EBD8D8D838
:1015F000D8D8D8E8D8FCD8D8D8D8D8FCD8D8EBFCDC
:10160000D8D8E8D8D8D8D8D8EBE8EBD8D8D8D8E804
:10161000D8D8D8FCD8E8EBD8D8D8D8D8FCD8D8D8DF
:10162000D8D8D8D8FCD8D8D8D8D8E8D8FCD8D8FCBE
:10163000D8D8D8FCD8FCD8D8D8D8E8FCD8D8D8D8AE
:10164000D8E8D8E8D8D8D8D8FCFCFCD8D8E8D8FC5A
:10165000D8D8D8FCD8D8E8D8E8D8D8D8D8FCD8E892
:10166000E8E8D8E8FCD8D8D8D800D800E800D800F6
:10167000D8D800D800FC00D80000D800D800FC0062
:10168000D8FC00E800D800E80000D800E800FC0022
:10169000FCD800FC00D800D80000E800D800D80032
:1016A000D8D800FC00D800D80003FFA70300A70388
:1016B000A70300A700A7FFA7FFA7A700A7A7A7A7A3
:1016C000A700A7A7A7A7A7A7A700A7A7A7A7A7A7F8
:1016D000A7A7A7A7A7A7A7A70000A7A7A7A7A7008F
:1016E000FF00A7A7A7A7A700FFA703A70300A7FFBF
:1016F00003FFA7FFA700A70003A7A7A7A7A700A707
:10170000A7A7A7A7A7A7A7A700A7A7A7A7A7A703B4
:101710000300A7A7A7A7A7A7A7FF00A7A7A7A7A7F3
:1017200003FF00A7A7A7A7A70003039FA7A700FF82
:10173000A70303A7A7A700A7A7030303A7A700A7BB
:10174000A700FFFFA7A7A7A7A70000FF000000A70B
:10175000A700009FFFFF0000000003009F9F9F0065
:10176000030000000000000000A7FF00A7A79F03E0
:1017700003A7A700A7A7A70303A7A700A7A703037B
:1017800003A7A7A7A7A7FFFF00A7A7000000FF00C8
:1017900003000000FFFF9F000300009F9F9F0003C6
:1017A00000000000000000000000FF0000009F009B
:1017B0009F009F9F0000FF00FF00009F00A7A7A7BA
:1017C000A7A7A700A7A7A7A7A700A7A7A7A7A7A7F7
:1017D000A700A7A7A7A7A7A7A7A7A7A7A7A7A7A740
:1017E000A700A7A7A7A7A7A7A79F009F000000FF84
:1017F00000FF00FF00009F9F00A7A7A7A7009F0072
:1018000000A7A7A7A7A700A7A7A7A7A7A7A7A7A7B6
:1018100000A7A7A7A7A7A70303A7A7A7A7A7A7A747
:10182000A7A7A7A7A7A7A7A7030000A70000A7A788
:10183000FF030300A7A7A7A7A703A700A7A7A7A71A
:10184000A70300A7A7A7A7A7A70000A7A700A7A768
:10185000A700A7A7A7A70000A70000A700A7A7A702
:10186000A7000000A70000A7A7FFA7A70000A700E8
:1018700000A7A7A7A7A7000303A7A7A7A7A700A735
:1018800003A7A7A7A7A7A70003A7A7A700A7A70025
:1018900000A70000A7A7A7A703A7A7A7A700A700BF
:1018A00003A7A70000A700000300A700A7A7A700A1
:1018B00000030000A7A7A7FFFF030300A7A7FFFFE0
:1018C000FF03000000A7FFFFFF00000000A7FFFFCD
:1018D000FF0000A7A700A7FFFF00A7A7FFA7000022
:1018E000000000FF00FF0000000000A7A7A700A75E
:1018F00000FFFFA7A7A7000003FFFFFFA7A70003A4
:1019000003FFFFFFA700000003FFFFFFA700000089
:1019100000FFFFA700A7A70000000000A7FFA7A7E0
:1019200000000000FF00FF00000303A70300A7A7BB
:10193000FF030300A7A7A7A7A703A700A7FFFFFF11
:10194000A70000A7A7FF0000A70000A7FFFF000057
:10195000A700A7A7A7FFFFA7A70000A700000000F8
:1019600000000000A700000000FFA7A70300A703D6
:1019700003A7A7A7A7A7000303A7FFFFFFA700A729
:1019800003A70000FFA7A70000A70000FFFFA70014
:1019900003A7A7FFFFA7A7A7030000000000A70059
:1019A0000300000000A7000000000000000000008D
:1019B00000030303A7A7A7A7A703A7A7FFFFA7A73E
:1019C000A7A7A7FFA7A7A7A7A7A7A7A7A7A7A7A74F
:1019D000A7A7A7A7A700A7A7A7A7A70000A7A7A78C
:1019E000A7A7A7A7A7A7A700A700FFA70000000019
:1019F00000A7A7000003030303A7A7A7A7030303E8
:101A000003A7A7000000030303A7A7A7A7A7000039
:101A100000A7A7A70000030303A7A7A7A7A7A7FFDF
:101A200000A7A7A7A70000FFA70000000000A7A726
:101A3000A700A7A7A7A7A7A7A70300FFFFFFFFA7C8
:101A4000A7030000FFFFFFFFA700FFA700A7FFFFFE
:101A5000A7FFFFA7A7000000000000000000FFA7ED
:101A6000A700030300FF00FFA7A7A7A7A70000A7E1
:101A7000A7A7A7A7A7A700A7A7A7A7A7A7A7A7A79D
:101A8000A7A7A7A7A7A7A7A70000A7A7A7A7000082
:101A900000A700000000030303A7A700030303033C
:101AA0000300000303030303030303A7A7A7A7A7D8
:101AB000A703A7A7FFFFA7A7A7A70000FFFFFFA7F0
:101AC000A7A70000FFFFFFA7A7A7A7A7FFFFA7A73C
:101AD000A7A7A7A7A7A7A700A7000000000000A727
:101AE000A7000000000000A7A70000000000A7FF5B
:101AF00000030303030000A7A703030303A7A7A78B
:101B0000A7030303000000A7A7000000A7A7A7A73B
:101B1000A70003030000A7A7A700FFA7A7A7A7A7E1
:101B2000A7A7FF0000A7A7A7A700000000000000CC
:101B300000A7A7A7A7A7030303A7A7A7FFFFA7A718
:101B400003A7A7A7A7A7FFA7A7A7A7A7A7A7A7A771
:101B5000A7A7A7A700A7A7A7A7A7A7A7A70000A70A
:101B6000A7A700A7A7A7A7A7A7A7A70000A7A7A7FA
:101B7000A7A7A700A7A7A7A7A7A7A7A7A7A7A7A79C
:101B8000A700A7A7A7A7A7A7A7000000A7A7A7A781
:101B90000000030300000000A7000303030300A7E5
:101BA000A70003030303030000A7A7A7000000008A
:101BB00000A7A7A7A7A7A7A700A7A7FFFFFFFF004A
:101BC00003A7FFFFFFFF000003A7FFFFA700A7FF7A
:101BD0000000000000A7A7FFFFA7A7FF000000006C
:101BE00000A7FF00FF00030303A7A7A7A7A7A7035A
:101BF00003A7A7A7FFFFA7A703A7A7FFFFFF000053
:101C0000A7A7A7FFFFFF0000A7A7A7A7FFFFA7A7FA
:101C1000A7A700A7A7A7A7A7A7A7A700000000003E
:101C200000A7A70000000000000000005B00005BB0
:101C300000035B00005B5B005B00005B005B00007F
:101C40005B5B005B0000005B00005B005B5B005BBC
:101C50005B5B000000005B005B005B005B5B5B00AC
:101C60005B005B5B5B5B5B5B5B5B00000000000041
:101C700000005B005B00000303005B5B00005B0394
:101C8000035B00005B5B000000005B00005B005B2F
:101C90005B005B005B005B00005B005B5B5B00006C
:101CA0005B5B5B5B5B5B5B5B00005B005B000000A6
:101CB0005B03005B5B5B5B5B5B030300005B5B5B8D
:101CC00000030303005B5B5B5B000000FF00005B45
:101CD0005B0000FFFFFF000000000300FF005B5BF4
:101CE0005B000303005B5B5B5B000000005B005B71
:101CF00000005B5B5B5B5B0003005B5B5B00000306
:101D0000035B5B5B5B000303035B5B0000000000A5
:101D100000000000000000000300000000000003BD
:101D2000035B5B5B5B00030303000000FF0000FF3D
:101D30000003FF0000FF5B00000000FF005B0000ED
:101D40005BFF005B000000FF00005B00FF5B005BCF
:101D500000FF000000005B005B005B005B5B5B0062
:101D600000005B5B000000000000FF0000FF0000BF
:101D70000000005BFF0000FF035B00005B00FF0052
:101D80000000FF0000005B00FF005B005BFF005BEA
:101D9000005B005B00000000FF00005B5B5B005B22
:101DA0000000000000005B5B00005B0000FFFF0024
:101DB0000003005B5B00000000030300005B5B5B53
:101DC00000030303005B5B5B000000005B005B0043
:101DD000000000FF5B5B005B5B000300FF00000096
:101DE00000000303005B5B5B5B0000FFFF00005B28
:101DF00000000000005B5B0003005B5B5B00000316
:101E000003005B5B5B0003030300005B005B0000FF
:101E1000005B5B005B5BFF000300000000FF000352
:101E2000035B5B5B5B0003030300FFFF00FFFF003E
:101E300000030300FF00FFFF00030000000000009C
:101E40000000FF20FFFF2020000000200000FF20F6
:101E5000200000200000FF202000FF20FFFF2020A6
:101E600020000020202000202000000000000000B2
:101E70000003030303001903030303030300030325
:101E8000030003030300030303000000000000003D
:101E900000200003030019000320000303001900C1
:101EA0000320000303001919000000000000202097
:101EB0002003002020202020200300FFFFFF2020FF
:101EC00020030300FFFFFF2020000000FFFFFF2092
:101ED00020001900FFFFFF202000030300FFFFFF89
:101EE000FF000303030000000000000000002020AA
:101EF0000000030303002020000003030020202033
:101F0000002000002020201900202020201019008F
:101F100000201020101900000310191019000003F0
:101F200003000000000303030300000000FF0000A3
:101F3000FF03030300190000190303000000000061
:101F400000030000FFFF20FFFF0000FF0000200053
:101F5000000000FF0000200000000020FFFF20FF25
:101F6000FF000020002020200000000000000000F2
:101F7000000003030300190303000003030003032D
:101F8000032000000300030303FF20000000000003
:101F900000FF200003002000032020000300200099
:101FA000032020000300202000000000200000008B
:101FB00020030300202020202003030020FFFFFF38
:101FC0002003030020FFFFFFFF00000020FFFFFFB2
:101FD000FF0019030019FFFFFF000303030019FFAF
:101FE000FF00030303030000002000000000202086
:101FF00000200003002020200020000020202019C5
:10200000002020202010190003202020101900009B
:10201000001020101900000303FF10190000030333
:10202000030000000303030303000000000000009E
:102030000003030303001903030303030300030363
:102040000003030303000300000000000000000081
:1020500020001900200003002000030020000300DE
:1020600020000020200003002000FF0000FF0000EF
:102070000000190000190003030000000000000028
:102080000320FFFF20FFFF0000FF0000200000FFF3
:1020900000FF0000200000FF0020FFFF20FFFF20C6
:1020A0000020002020200020000000202000000050
:1020B000000300202020000300030019202020003E
:1020C0000003030019102020200000000019102038
:1020D0002000190300001910200003030300001959
:1020E0001000030303030300002020000000200071
:1020F0000020202020202000032020FFFFFF2000C0
:102100000320FFFFFFFF20000320FFFFFFFF200051
:102110000010FFFFFF19000303FFFFFF1900030377
:1021200003000000000303030300000000000000A0
:102130000003030303001903030303030300030362
:10214000030303030300030300000000000000007A
:102150000000002000030300200000200003030013
:102160002000202000030300200000FFFF00FFFFED
:102170000000FFFF00FF000303000000000000005C
:1021800003002020FFFF20FF002020FF0000200090
:10219000002020FF0000200000202020FFFF20FF63
:1021A000002020002020200000002020000000004F
:1021B000000020200000190300002020200003035D
:1021C00000001920202000002000001910202020ED
:1021D0002000000019102010200003000019101921
:1021E0001000030303000000002020200000000076
:1021F000002020202020200003202020FFFFFF00BF
:10220000032020FFFFFF0003032020FFFFFF00004B
:10221000002020FFFFFF000303FFFFFFFF00030379
:10222000030000000003030303000000005BFFFF46
:10223000FF03005BFFFFFFFFFF005BFFFFFFFFFFF0
:10224000FF00FFFF5B005BFFFF5BFF5B0000000028
:102250005B5BFF0000000000005BFF00000000006F
:10226000FF5BFF00000000FF00FFFFFF5B000000BE
:1022700000FFFFFFFFFF5B0003FFFFFFFFFFFF5BB0
:1022800000FFFF5B005BFFFF005B000000005BFFE7
:102290005B000000000000FF5BFF0000000000FF8B
:1022A0005B00FF00000000FF5B005BFF00005BFFC6
:1022B0000000005BFFFFFFFFFF0300005B00FF006B
:1022C000FF030000FF00000000000000FFFF5BFFB5
:1022D0005B0000000000FFFFFF00000000000000A6
:1022E00000000000000000000000FF5B0000FF5B3A
:1022F00000FFFFFFFFFF5B0000FF00FF005B00002F
:102300000300000000FF0000035BFF5BFFFF000015
:1023100000FFFFFF000000000000000000000000C0
:1023200000000000000000000300000000FFFFFFAD
:10233000FF0000FFFF850303850085FF8585FFFF04
:102340008500FFFF03FFFFFFFF0085FF8585FFFF7F
:10235000850000FFFF8503038500000000FFFFFFED
:10236000FF000000000000000000008500000000E9
:1023700000FFFF00FF0085000085FF8500FF00854E
:102380000003FFFF00FF00850085FF8500FF00853B
:1023900000FFFF00FF008500000000850000000036
:1023A000000000000000000000FFFFFFFFFFFFFF34
:1023B000FFFFFFFFFFFFFFFFFF5B5B5B5B5B5B5BA9
:1023C0005B0909090909090909090909090909092B
:1023D00009000000000000000000000000000000F4
:1023E00000000000000000000000000000000000ED
:1023F00000000000000000000000000000000000DD
:1024000000000000000000000000000000000000CC
:1024100000FFFFFFFFFFFFFFFFFFFFFFFFFFFFFFCB
:10242000FF5B5B5B5B5B5B5B5BFFFF5B090900006A
:1024300000FFFF5B0909000000FFFF5B09090000C6
:1024400000FFFF5B0909000000FFFF5B09090000B6
:1024500000FFFF5B0909000000FFFF5B09090000A6
:1024600000FFFF5B09090000000000000000FFFF03
:102470005B0000000000FFFF5B0000000000FFFFAA
:102480005B0000000000FFFF5B0000000000FFFF9A
:102490005B0000000000FFFF5B0000000000FFFF8A
:1024A0005B0000000000FFFF5BFFFF000909000068
:1024B00000FF00F60000000000FF00F6F6F6000046
:1024C00000FF00F6F6F6F60000FF00F6F6F6000054
:1024D00000FF00F60000000000FFFF0009090000F7
:1024E00000FFFF5B09090000000000FFFFFFFFFF86
:1024F000FF00FFFFFFFFFFFFFFFFFFFFFFFF5B5B33
:102500005BFFFFFF5B5B090909FFFF5B5B090909D3
:1025100009FFFF5B0909090000FFFF5B09090000D3
:1025200000FFFF5B0909000000FFFFFFFFFF5B00EA
:1025300000FFFFFFFFFF5B5B005B5B5BFFFFFF5B81
:102540005B0909095B5BFFFF5B090909095BFFFF89
:102550005B0000000009FFFF5B0000000000FFFFC0
:102560005B0000000000FFFF5BFFFF5B090900004C
:1025700000FFFF5B0909000000FFFF5B0909000085
:1025800000FFFF5B5B09000000FFFFFF5B5B0900D2
:1025900000FFFFFFFFFFFFFFFF005BFFFFFFFFFFED
:1025A000FF00005B5B5B5B5B5B0000000000FFFF0C
:1025B0005B0000000000FFFF5B0000000000FFFF69
:1025C0005B00000000FFFFFF5B000000FFFFFFFF5C
:1025D0005BFFFFFFFFFFFF5B5BFFFFFFFFFF5B5B3F
:1025E000005B5B5B5B5B5B000000000000000000C9
:1025F000000000FFFFFFFFFFFF00FF0000FFFFFFE5
:10260000FF00FF0000FFFFFFFF00FFFFFFFFFFFFD6
:10261000FF00FFFFFFFFFFFFFF00FFFFFFFFFFFFC8
:10262000FF00FFFFFFFFFFFFFF00000000000000B2
:1026300000FFFFFFFFFFFF0000FFFFFFFF0000FFA5
:1026400000FFFFFFFF0000FF00FFFFFFFFFFFFFF96
:1026500000FFFFFFFFFFFFFF00FFFFFFFFFFFFFF88
:1026600000FFFFFFFFFFFFFF0000FFFFFFFFFFFF77
:10267000FF00FFFFFFFFFFFFFF00FFFFFFFFFFFF68
:10268000FF00FFFFFFFFFFFFFF00FF0000FFFFFF56
:10269000FF00FF0000FFFFFFFF0000FFFFFFFFFF45
:1026A000FF0000000000000000FFFFFFFFFFFFFF32
:1026B00000FFFFFFFFFFFFFF00FFFFFFFFFFFFFF28
:1026C00000FFFFFFFFFFFFFF00FFFFFFFF0000FF16
:1026D00000FFFFFFFF0000FF00FFFFFFFFFFFF0005
:1026E00000000000000000000000000000000000EA
:1026F0000000FFFFFFFFFF0000FFFF000000FFFFE3
:1027000000FFFF0000FFFFFF00FFFF00FF00FFFFD3
:1027100000FFFFFF0000FFFF00FFFFFF0000FFFFC3
:102720000000FFFFFFFFFF000000000000000000AE
:10273000000000FFFF0000000000FFFFFF0000009E
:102740000000FFFFFF000000000000FFFF0000008E
:10275000000000FFFFFF0000000000FFFFFF00007F
:1027600000FFFFFFFFFFFFFF000000000000000070
:102770000000FFFFFFFFFF0000FFFFFF0000FFFF63
:10278000000000000000FFFF0000000000FFFF004D
:102790000000FFFFFF00000000FFFFFF000000003F
:1027A00000FFFFFFFFFFFFFF000000000000000030
:1027B0000000FFFFFFFFFF0000FFFF000000FFFF22
:1027C000000000000000FFFF00000000FFFFFF000E
:1027D000000000000000FFFF00FFFF000000FFFFFF
:1027E0000000FFFFFFFFFF000000000000000000EE
:1027F00000000000FFFFFFFF000000FFFF00FFFFE1
:102800000000FFFF0000FFFF00FFFF000000FFFFD0
:1028100000FFFFFFFFFFFFFFFF0000000000FFFFC2
:10282000000000000000FFFF0000000000000000AA
:1028300000FFFFFFFFFFFFFF00FFFF0000000000A1
:1028400000FFFFFFFFFFFF00000000000000FFFF90
:10285000000000000000FFFF00FFFFFF0000FFFF7F
:1028600000FFFFFFFFFFFF0000000000000000006E
:102870000000FFFFFFFFFF0000FFFF000000FFFF61
:1028800000FFFF000000000000FFFFFFFFFFFF0050
:1028900000FFFFFF0000FFFF00FFFFFF0000FFFF42
:1028A0000000FFFFFFFFFF0000000000000000002D
:1028B00000FFFFFFFFFFFFFF00FFFF000000FFFF23
:1028C0000000000000FFFF00000000FFFF0000000C
:1028D000000000FFFF000000000000FFFFFF0000FD
:1028E000000000FFFFFF00000000000000000000EB
:1028F0000000FFFFFFFFFF0000FFFF000000FFFFE1
:1029000000FFFF000000FFFF0000FFFFFFFFFF00D0
:1029100000FFFFFF0000FFFF00FFFFFF0000FFFFC1
:102920000000FFFFFFFFFF000000000000000000AC
:102930000000FFFFFFFFFF0000FFFF000000FFFFA0
:1029400000FFFF000000FFFF0000FFFFFFFFFFFF91
:10295000000000000000FFFF00FFFFFF0000FFFF7E
:102960000000FFFFFFFFFF0000000000000000006C
:102970000000000000000000000000000000000057
:102980000000000000000000000000000000000047
:102990000000000000000000000000000000000037
:1029A0000000000000000000000000000000000027
:1029B000000000FFFFFFFF000000FFFF000000FF1E
:1029C0000000FFFF000000FF0000FFFF00FFFFFF0F
:1029D0000000FFFF000000FF0000FFFF000000FFFD
:1029E0000000FFFF000000FF0000000000000000EA
:1029F0000000FFFFFFFFFF000000FFFF000000FFDF
:102A00000000FFFF000000FF0000FFFF00FFFF00CD
:102A10000000FFFF000000FF0000FFFF000000FFBC
:102A20000000FFFFFFFFFF000000000000000000AB
:102A3000000000FFFFFFFF000000FFFFFF0000FF9E
:102A40000000FFFF000000000000FFFF000000008A
:102A50000000FFFF000000000000FFFFFF0000FF7C
:102A6000000000FFFFFFFF0000000000000000006A
:102A70000000FFFFFFFFFF000000FFFF0000FFFF5F
:102A80000000FFFF000000FF0000FFFF000000FF4C
:102A90000000FFFF000000FF0000FFFF0000FFFF3D
:102AA0000000FFFFFFFFFF0000000000000000002B
:102AB0000000FFFFFFFFFFFF0000FFFF000000001E
:102AC0000000FFFF000000000000FFFFFFFFFF000D
:102AD0000000FFFF000000000000FFFF00000000FA
:102AE0000000FFFFFFFFFFFF0000000000000000EC
:102AF0000000FFFFFFFFFFFF0000FFFF00000000DE
:102B00000000FFFF000000000000FFFFFFFFFF00CC
:102B10000000FFFF000000000000FFFF00000000B9
:102B20000000FFFF000000000000000000000000A7
:102B3000000000FFFFFFFF000000FFFF000000FF9C
:102B40000000FFFF000000000000FFFF00FFFFFF8C
:102B50000000FFFF000000FF0000FFFF000000FF7B
:102B6000000000FFFFFFFFFF00000000000000006A
:102B70000000FFFF000000FF0000FFFF000000FF5B
:102B80000000FFFF000000FF0000FFFF00FFFFFF4D
:102B90000000FFFF000000FF0000FFFF000000FF3B
:102BA0000000FFFF000000FF000000000000000028
:102BB000000000FFFFFFFF0000000000FFFF00001B
:102BC00000000000FFFF000000000000FFFF000009
:102BD00000000000FFFF000000000000FFFF0000F9
:102BE000000000FFFFFFFF000000000000000000E9
:102BF00000000000FFFFFFFF0000000000FFFF00DB
:102C00000000000000FFFF000000000000FFFF00C8
:102C10000000000000FFFF000000FF00FFFFFF00BA
:102C2000000000FFFFFF00000000000000000000A7
:102C30000000FFFF000000FF0000FFFF0000FF009A
:102C40000000FFFF00FF00000000FFFFFF0000008A
:102C50000000FFFF00FF00000000FFFF0000FF007A
:102C60000000FFFF000000FF000000000000000067
:102C70000000FFFF000000000000FFFF0000000058
:102C80000000FFFF000000000000FFFF0000000048
:102C90000000FFFF000000000000FFFF0000000038
:102CA0000000FFFFFFFFFFFF00000000000000002A
:102CB0000000FFFFFF00FF000000FFFF00FF00FF1C
:102CC0000000FFFF00FF00FF0000FFFF00FF00FF0C
:102CD0000000FFFF00FF00FF0000FFFF00FF00FFFC
:102CE0000000FFFF00FF00FF0000000000000000E8
:102CF0000000FFFFFFFFFF000000FFFF0000FFFFDD
:102D00000000FFFF000000FF0000FFFF000000FFC9
:102D10000000FFFF000000FF0000FFFF000000FFB9
:102D20000000FFFF000000FF0000000000000000A6
:102D3000000000FFFFFFFF000000FFFFFF00FFFF9C
:102D40000000FFFF000000FF0000FFFF000000FF89
:102D50000000FFFF000000FF0000FFFFFF00FFFF7B
:102D6000000000FFFFFFFF00000000000000000067
:102D70000000FFFFFFFFFF000000FFFF000000FF5B
:102D80000000FFFF000000FF0000FFFFFFFFFF004B
:102D90000000FFFF000000000000FFFF0000000037
:102DA0000000FFFF00000000000000000000000025
:102DB000000000FFFFFFFF000000FFFF000000FF1A
:102DC0000000FFFF000000FF0000FFFF000000FF09
:102DD0000000FFFFFFFF00FF0000FFFF0000FFFFFC
:102DE000000000FFFFFFFF000000000000000000E7
:102DF0000000FFFFFFFFFF000000FFFF000000FFDB
:102E00000000FFFF000000FF0000FFFFFFFFFF00CA
:102E10000000FFFF0000FFFF0000FFFF0000FFFFBA
:102E20000000FFFF0000FFFF0000000000000000A6
:102E3000000000FFFFFFFF000000FFFF000000FF99
:102E40000000FFFF00000000000000FFFFFFFF0088
:102E5000000000000000FFFF0000FFFF0000FFFF78
:102E6000000000FFFFFFFF00000000000000000066
:102E70000000FFFFFFFFFFFF00000000FFFF00005A
:102E800000000000FFFF000000000000FFFF000046
:102E900000000000FFFF000000000000FFFF000036
:102EA00000000000FFFF0000000000000000000024
:102EB0000000FFFF000000FF0000FFFF000000FF18
:102EC0000000FFFF000000FF0000FFFF000000FF08
:102ED0000000FFFF000000FF0000FFFFFF00FFFFFA
:102EE000000000FFFFFFFF000000000000000000E6
:102EF0000000FFFF000000FF0000FFFF000000FFD8
:102F00000000FFFF000000FF0000FFFF000000FFC7
:102F1000000000FFFF00FF00000000FFFF00FF00B7
:102F200000000000FFFFFF000000000000000000A4
:102F30000000FFFF00FF00FF0000FFFF00FF00FF99
:102F40000000FFFF00FF00FF0000FFFF00FF00FF89
:102F50000000FFFF00FF00FF000000FF00FF00FF78
:102F6000000000FFFF00FF00000000000000000064
:102F70000000FFFF0000FFFF0000FFFF0000FFFF59
:102F8000000000FFFFFFFF0000000000FFFF000047
:102F9000000000FFFFFFFF000000FFFF0000FFFF39
:102FA0000000FFFF0000FFFF000000000000000025
:102FB0000000FFFF000000FF0000FFFF000000FF17
:102FC0000000FFFF000000FF000000FFFFFFFF0008
:102FD00000000000FFFF000000000000FFFF0000F5
:102FE00000000000FFFF00000000000000000000E3
:102FF0000000FFFFFFFFFFFF000000000000FFFFD9
:103000000000000000FFFF0000000000FFFF0000C4
:10301000000000FFFF0000000000FFFF00000000B4
:103020000000FFFFFFFFFFFF00FEFEFE000000DAD2
:10303000DAFEFE00DAFFFFFFDAFE00DAFFFFDADA7F
:10304000DA00DADADADADADADA00DADADADADADA94
:10305000DADADADADADADADADADADADADADADADAD0
:10306000DAFF00DADADADADADADA000000FEFEFE97
:10307000FEFFDADADA00FEFEFEDADADADADA00FE8B
:10308000FEDADADADADADA00FEDADADADADADA000C
:10309000FEDADADADADADADAFEDADADADADADADA48
:1030A000FEDADADADADA00FFFEFEFEFE000000DA0F
:1030B000DAFEFE00DAFFFFFFDAFE00DAFFFFDADAFF
:1030C000DA00DADADADADADADA00DADADADADADA14
:1030D000DADADADADADADADADAFF00DADADADADA05
:1030E000DAFFFF00DADADADADADA000000FEFEFEF2
:1030F000FEFFDADADA00FEFEFEDADADADADA00FE0B
:10310000FEDADADADADADA00FEDADADADADADA008B
:1031100000DADADADADADADA00DADADADADADADAC3
:1031200000DADADADADA00FF00FEFEFE000000DA8A
:10313000DAFEFE00DAFFFFFFDAFE00DAFFFFDADA7E
:10314000DAFE00DADADADADADA00DADADADADADA6F
:10315000DADADADADADADADADAFFFF00DADADADA5F
:10316000DAFFFFFF00DADADADADA000000FEFEFE4C
:10317000FEFFDADADA00FEFEFEDADADADADA00FE8A
:10318000FEDADADADADA00FEFEDADADADADADA00E7
:1031900000DADADADADADA0000DADADADADADA00F7
:1031A00000DA000000DA00FF00FEFEFE000000DA98
:1031B000DAFEFE00DAFFFFFFDAFE00DAFFFFDADAFE
:1031C000DA00DADADADADADADA00DADADADADADA13
:1031D000DADADADADADADADADADADADADADADADA4F
:1031E000DAFFDADADADADADADADA000000FEFEFE3C
:1031F000FEFFDADADA00FEFEFEDADADADADA00FE0A
:10320000FEDADADADADADA00FEDADADADADADA008A
:1032100000DADADADADADA0000DADADADADA00FF51
:1032200000DADADADA00FFFF00FEFEFE000000DA64
:10323000DAFEFE00DAFFFFFFDAFE00DAFFFFDADA7D
:10324000DA00DADADADADADADA00DADADADADADA92
:10325000DADADADADADADADADADADADADADADADACE
:10326000DAFFDADA000000DADADA000000FEFEFE49
:10327000FEFFDADADA00FEFEFEDADADADADA00FE89
:10328000FEDADADADADADA00FEDADADADADADA000A
:1032900000DADADADADADADA00DADADADA00FFFFD2
:1032A00000DADADA00FFFFFF00FF00DADADADADA52
:1032B000DAFF00DADADADADADAFFFF00DADADADAB3
:1032C000DA00FFFF00DADADADAFE00000000DADA0C
:1032D000DAFEFE00FFFF00DADAFEFE00000000006A
:1032E000DAFEFEFEFEFEFEFEFEDADADADADA00FFD3
:1032F000FEDADADADADA00FFFEDA00DADA00FFFF05
:10330000FE00DADA00FFFF00FE00DA00000000FE37
:10331000FEDA00FFFF00FEFEFE0000000000FEFEE1
:10332000FEFEFEFEFEFEFEFEFEFFFF00DADADADA49
:10333000DAFFFF00DADADADAFFFFFF00DADADADAE8
:10334000DA00FF0000DADADADAFE0000000000003E
:1033500000FEFE000000FEFEFEFEFEFEFEFEFEFE85
:10336000FEFEFEFEFEFEFEFEFEDA0000DADA00FFE2
:1033700000DADADA00DA00FF00DADADA0000FF0059
:10338000FEDADADADA0000FEFEDA00000000FEFE05
:10339000FE0000FFFF00FEFEFE00FFFFFF00FEFE3E
:1033A000FE00000000FEFEFEFE00FFFF00DADADA9B
:1033B000DAFFFFFF00DADADADAFFFFFF00DADADA43
:1033C000DA00FF0000DADADADAFE0000000000DAE4
:1033D000DAFEFEFEFEFEFE0000FEFEFEFEFEFEFE2D
:1033E000FEFEFEFEFEFEFEFEFEFFDADADA0000FF63
:1033F00000DADADADA00000000DADADADA00DA0023
:10340000FEDADADA000000FEFE0000000000FEFE38
:10341000FE0000FFFF00FEFEFE00FFFFFF00FEFEBD
:10342000FE00000000FEFEFEFEFFDADADA0000DA3F
:10343000DAFFDADA00DAFFDADA00FFDA00DADADA0B
:10344000DAFE0000DADADADADAFEFE00000000DA8C
:1034500000FEFE00FFFF0000FEFEFE00FFFFFF007B
:10346000FEFEFEFE00000000FEDADADADA00FFFF00
:1034700000DADA000000FFFF00DA00DADA00FFFF0E
:103480000000DADA0000FF00FE000000000000FE8D
:10349000FEFEFE000000FEFEFEFEFEFEFEFEFEFE46
:1034A000FEFEFEFEFEFEFEFEFE00DA00FFFFDADAA2
:1034B000DA00DA00DADADADADA00DA00DADADADAD4
:1034C000DAFEFEDA00DADADADAFEFE0000000000E8
:1034D00000FEFE00FFFF0000FEFEFE00FFFFFF00FB
:1034E000FEFEFEFE00000000FEDADADA00FFFF005A
:1034F00000DADA0000FFFFFF0000DADA00FFFFFF6A
:1035000000DA00000000FF00FE000000000000FEE6
:10351000FEFEFEFEFEFEFEFEFEFEFEFEFEFEFEFECB
:10352000FEFEFEFEFEFEFEFEFEFEFEFE000000DAD9
:10353000DAFEFE00DAFFFFFFDAFE00DAFFFFDADA7A
:10354000DAFE00DADADADADADA00DADAFFFFFFDAFC
:10355000DA00DAFFFFFFFFFFDA00DAFFFFFF00000B
:10356000DA0000FFFFFF0000DADA000000FEFEFED6
:10357000FEFFDADADA00FEFEFEDADADADADA00FE86
:10358000FEDADADADADA00FEFEDAFFFFFFDADA0074
:10359000FEFFFFFFFFFFDA00FE0000FFFFFFDA0083
:1035A000FE0000FFFFFF0000FEFEFEFEFE0000DA50
:1035B000DAFEFE0000FFFFFFDAFE00DAFFDADADAF9
:1035C000DAFE00DADADADADADA00DADAFFFFDADAA1
:1035D000DA00DAFFFFFFFFDAFFFFDAFFFF0000DAB1
:1035E00000FFDAFFFF0000DA00DA0000FEFEFEFE58
:1035F000FEFFDADA0000FEFEFEDADADADADA00FEE0
:10360000FEDADADADADA00FEFEFFFFFFDADADA00F3
:10361000FEFFFFFFFFDADA00FE00FFFFFFDA00FF28
:103620000000FFFFFFDA00FF00FEFEFE000000DAF0
:10363000DAFEFE00DAFFFFFFDAFE00DAFFDADADA9E
:10364000DAFE00DADADADADADA00DADAFFDADADA45
:10365000FF00DAFFFFFFDAFFFFFFDAFF0000DAFF0B
:1036600000FFDAFF0000DAFF00DA0000FEFEFEFED7
:10367000FEFFDADA0000FEFEFEDADADADA0000FE39
:10368000FEDADADADADA00FEFEFFFFDADADAFF0073
:1036900000FFFFFFDADA00FF0000FFFFDADA00FFC9
:1036A0000000FFFFDADA00FF00FEFEFEFE00000071
:1036B000DAFEFEFE00FFFFFFDAFEFE00FFFFDADAB1
:1036C000DAFE00DADADADADADA00DADADAFFFFFF7B
:1036D000DA00DADAFFFFFFFFFFFF00DAFFFFFF008B
:1036E00000FF00DAFFFFFF0000DA0000FEFEFEFE32
:1036F000FEFFDADA0000FEFEFEDADADADADA00FEDF
:10370000FEDADADADADA00FEFEDADAFFFFDADA0017
:10371000FEDAFFFFFFFFDA00FEDA0000FFFFDAFF4C
:10372000FEDA0000FFFFDAFFFEFEFEFEFE000000F4
:10373000DAFEFEFE00FFFFFFDAFEFE00FFFFFFDA0B
:10374000DAFE00DADADADADADA00FFDADADAFFFFFA
:10375000FFFF00DADAFFFFFFFFFF00DADAFFFF000A
:1037600000FF00DADAFFFF0000DA0000FEFEFEFED6
:10377000FEFFDADA0000FEFEFEDADADADADA00FE5E
:10378000FEDADADADADA00FEFEDADADAFFDADA00BC
:10379000FEFFDAFFFFFFDA00FEFFDA0000FFDAFFCC
:1037A000FEFFDA0000FFDAFFFEFF00FFFFFFFFFF72
:1037B000DAFF0000FFFFFFDADA00FF00DADADADA18
:1037C000DA00FFFF0000DADADAFE00000000000095
:1037D00000FEFE00FFFFFF00FEFEFE0000000000F6
:1037E000FEFEFEFEFEFEFEFEFEFFFFFFFFFF00FFF1
:1037F00000DAFFFFFFDA00FF00DADADADA00FF00B2
:10380000FEDADA0000FFFF00FE000000000000FE0C
:10381000FE00FFFFFF00FEFEFE0000000000FEFEB7
:10382000FEFEFEFEFEFEFEFEFEFFFF00FFFFFFDAD5
:10383000FFFFFFFF00FFDADADAFFFFFFDADADADA9A
:10384000DA00FF0000DADADADAFE0000FFFFFF003C
:1038500000FEFEFE000000FEFEFEFEFEFEFEFEFE80
:10386000FEFEFEFEFEFEFEFEFEFFFFFFFFDA00FF95
:1038700000FFFFFFDADA00FF00DADADADA00FF0031
:10388000FEDADADADA00FEFEFE0000000000FEFEDC
:10389000FE00FFFFFF00FEFEFE00FFFFFF00FEFE3A
:1038A000FE00000000FEFEFEFEFFFF00FFFFDAFF4D
:1038B000FFFFFFFF00DADADAFF00FFFFDADADADA19
:1038C000DAFEFEFE00DADADA00FEFEFE000000009C
:1038D00000FEFEFEFEFEFEFEFEFEFEFEFEFEFEFE06
:1038E000FEFEFEFEFEFEFEFEFEFFFFFFDA00000013
:1038F00000FFFF00000000FE000000FFFF00FEFED2
:10390000FE00FFFFFF00FEFEFE00FFFFFF00FEFEC9
:10391000FE00FFFF0000FEFEFE00000000FEFEFEB7
:10392000FEFEFEFEFEFEFEFEFEFF00DAFFFFFFFFD4
:10393000FFFF00DADAFFFFFFDA00FF00DADADADA97
:10394000DAFEFE00DADADADADAFEFE000000000063
:1039500000FEFE00FFFFFF00FEFEFE00FFFFFF0077
:10396000FEFEFEFE000000FEFEDAFFFFFF00FFFF8E
:1039700000DADAFF00FFFFFF00DADADADAFFFFFF32
:1039800000DADADA0000FF00FE00FFFFFF000000AF
:10399000FEFE000000FEFEFEFEFEFEFEFEFEFEFE41
:1039A000FEFEFEFEFEFEFEFEFE0000DADAFFFFFF78
:1039B000FFFE00DA000000FFFFFEFE000000000036
:1039C000DAFEFE00FFFFFF0000FEFE00FFFFFF002B
:1039D00000FEFE00FFFFFF00FEFEFEFE000000FEF8
:1039E000FEFEFEFEFEFEFEFEFEFFDAFFFF00FFFF14
:1039F000FEDADADA00FFFFFFFEDADADADAFFFF00DA
:103A0000FEDADADA000000FEFE0000000000FEFE32
:103A1000FEFEFEFEFEFEFEFEFEFEFEFEFEFEFEFEC6
:103A2000FEFEFEFEFEFEFEFEFEFEFEFE000000D8D6
:103A3000D8FEFE00FFFFD8FFD8FE00FFD8D8D8D8A8
:103A4000D800D8D8D8D8D8D8D800D8FFFFFFD8D831
:103A5000D8D8FFFFFFFFFFD8D8D80000FFFFFFD85E
:103A6000D8D80000FFFFFFD8D8D8000000FEFEFE27
:103A7000FED8D8D80000FEFEFED8D8D8D8D800FE90
:103A8000FED8D8D8D8D8D800FED8D8D8D8D8D8001A
:103A900000D8D8D8D8D8D8D800D8D8D8FFFFFF00B9
:103AA00000D8D8D8D8FFFFFF00FEFEFE000000D8E7
:103AB000D8FEFE00FFD8FFD8D8FE00FFD8D8D8D84F
:103AC000D800D8D8D8D8D8D8D800D8FFFFD8D8D8D8
:103AD000D8D8FFFFFFFFD8D8D8D800FFFFFFD8D82D
:103AE000D8D800FFFFFFD8D8D8D80000FEFEFEFED1
:103AF000FED8D8D80000FEFEFED8D8D8D8D800FE10
:103B0000FED8D8D8D8D8D800FED8D8D8D8D8D80099
:103B100000D8D8D8D8D8D8D800D8D8D8FFFF00D85F
:103B200000D8D8D8FFFFFF0000FEFEFE000000DA3C
:103B3000DAFEFE00FFDADAFFDAFE00FFDADADADABE
:103B4000DA00DADADADADADADADAFFDADADADADA8A
:103B5000DAFFFFFFDADADADADA00FFFFDADADADAE6
:103B6000DA00FFFFDADADADAFFDA0000FEFEFEFE44
:103B7000FEDADADA0000FEFEFEDADADADADA00FE7F
:103B8000FEDADADADADADA00FEDADADADADADA0001
:103B900000DADADADA00DADA00FFFF00FFFF00DA33
:103BA00000FFFFFFFFFF00DADAFEFEFE000000DA92
:103BB000DAFEFE00FFFFFFDADAFE00FFDADADADA19
:103BC000DA00DADADADADADADADADADAFFFFFFDAC0
:103BD000DAFFDAFFFFFFFFFFDAFFDA0000FFFFFF87
:103BE000DAFFDA0000FFFFFFDADA000000FEFEFE77
:103BF000FEFFDADADA00FEFEFEDADADADADA00FE00
:103C0000FEDADADADADA00FEFEDADADADADADA005C
:103C1000FEDADADADADA0000FEDADADADAFFFF0000
:103C200000DADADADA00FFFF00FEFEFE000000D85C
:103C3000D8FEFE00FFFFFFD8D8FE00FFFFD8D8D87F
:103C4000D800D8D8D8D8D8D8D8D8D8D8D8FFFFFF57
:103C5000D8FFFFD8FFFFFFFFFF00FFD80000FFFFE6
:103C6000FF00FFD80000FFFFFFD8000000FEFEFEAF
:103C7000FEFFFFD8D800FEFEFED8D8D8D8D800FE68
:103C8000FED8D8D8D8D80000FED8D8D8D8D8D800F0
:103C900000D8D8D8D8FFFF0000D8D8D8D8FFFFFF69
:103CA00000D8D8D80000FFFF00D8FFFFFFFFFFD8E3
:103CB000D800D8FFFFFFD8D8D8FED8D8D8D8D8D8C1
:103CC000D8FE0000D8D8D8D8D8FEFE0000000000EA
:103CD000FFFEFEFEFEFE00FFFFFEFEFEFEFE0000FB
:103CE00000FEFEFEFEFEFEFEFED8D8FFFFFFFFFF39
:103CF00000D8FFFFFFFFFFFFFED8D8FFFFFFFF0048
:103D000000000000D80000D8D8FFFFFF000000002E
:103D100000FFFFFF00FEFEFEFE00000000FEFEFEB4
:103D2000FEFEFEFEFEFEFEFEFED8FFFFFFFFD8D821
:103D3000D800D8FFFFD8D8D8D8FED8D8D8D8D8D867
:103D4000D8FE0000D8D8D8D8D8FE00FF0000000068
:103D500000FE00FFFFFF00FE00FEFE00000000FE70
:103D600000FEFEFEFEFEFEFEFED8FFFFFFFFFF0090
:103D700000FFFFFFFFFFFF00FED8FFFFFFFF000077
:103D800000000000000000D8D800FFFFFFFF000087
:103D9000D8FFFFFFFFFF000000000000000000FE52
:103DA00000FEFEFEFEFEFEFEFEFFFFFFDADADADABE
:103DB000FFDAFFDADADADADA0000DADADADADADACD
:103DC000DAFE0000DADADADADA00FFFF00000000DB
:103DD000000000FFFFFF00FEFEFEFE000000FEFEF2
:103DE000FEFEFEFEFEFEFEFEFEFFFFFFFFFF00DA10
:103DF00000FFFFFFFF00DA000000000000DADA0039
:103E0000DADADADA0000DADA0000000000FF000097
:103E1000000000FFFFFF00FEFE0000000000FEFEAD
:103E2000FEFEFEFEFEFEFEFEFEFFDAFFFFFFFFFFD0
:103E3000DA00DADAFFFFFFDADA00DADADADADADA27
:103E4000DAFE000000DADADADAFE00FFFFFFFF0038
:103E500000FE00FFFFFFFFFF00FEFE00000000006D
:103E6000FEFEFEFEFEFEFEFEFEDADADADAFFFFFFFF
:103E700000DADAFFFFFFFFFF00DADAFFFFFFFF00E3
:103E800000DADADA000000DAFEDA00000000DADA3E
:103E90000000FFFFFFFF00FEFE0000000000FEFE2E
:103EA000FEFEFEFEFEFEFEFEFEFFFFD8FFFFFFFF52
:103EB000FF00D8D8D8FFFFFFD800000000D8D8D81E
:103EC000D800FFFFFF00D8D8D800FFFFFF0000D8C0
:103ED000D8FE00FFFFFF000000FEFE000000FEFE17
:103EE00000FEFEFEFEFEFEFEFED8D8D8FFFFFFFF5E
:103EF00000D8D8D8FFFFFF0000D8D8D800000000B5
:103F0000D8D8D8D8D8D8D8D8FED80000000000001B
:103F1000FE00FFFFFFFFFF00FE000000000000FEAC
:103F2000FEFEFEFEFEFEFEFEFEFEFEFEFE000000AB
:103F300000FEFE0000DADADADAFE00DADAFFFFDA93
:103F4000DA0000DAFF0000FFDAFFDAFFFF0000FF0F
:103F5000DAFFDAFFFFFFFFFFDA00DAFFFFFFFFFF04
:103F6000DA00DADAFFFFFFDADA000000FEFEFEFE1A
:103F7000FEDADADA0000FEFEFEDAFFFFFFDA00FE0C
:103F8000FEFFFFFFFFFF0000FEFFFFFFFFFF00FF40
:103F900000FF0000FFFF00FF00FF0000FFFF00FF29
:103FA00000DAFFFFFFDADA000000DADADADADADA6A
:103FB000DA00DADA0000000000FE00DA00FFFF009D
:103FC000FF00FF00DA0000000000FFFF00DADADA8D
:103FD000DA00FFFF0000000000FE0000FEFEFEFE13
:103FE000FEFEFEFEFEFEFEFEFEDADADADADADAFEC9
:103FF000FE00000000DADAFEFEFF00FF00DA00003B
:10400000FE000000DA00FFFF00DADADA00DAFFFF74
:1040100000000000FFFFFF00FEFEFEFE000000FEAD
:10402000FEFEFEFEFEFEFEFEFEFEFEFEFE000000AA
:1040300000FEFE0000DADADADAFE00DADAFFFFDA92
:10404000DA00DADAFFFFFFFFDAFF00FFFF0000FF10
:10405000DAFF00FFFF0000FFDA00DAFFFFFFFFFFDB
:10406000DA00DADAFFFFFFDADA000000FEFEFEFE19
:10407000FEDADADA000000FEFEDAFFFFFF00DA0007
:10408000FEFFFFFFFFDA00FFFFFFFFFFFFFFDAFF8A
:10409000FFFF0000FFFFDAFFFFFF0000FFFFDAFF76
:1040A000FFDAFFFFFFDADA00FF00DADADADADADA6B
:1040B000DAFE00DADADADA0000000000DADA00000C
:1040C0000000FF0000DA00FFFF00FFFF000000001B
:1040D000FF0000FF00FE000000FE000000FEFE00EA
:1040E00000FEFEFEFEFEFEFEFEDADADADADA00FF9F
:1040F000FF00DADADADA00FFFF0000DADADA0000CD
:1041000000FF00DA0000FFFF0000000000FFFFFFDB
:1041100000000000FFFFFF00FE00FE00000000FEA8
:10412000FEFEFEFEFEFEFEFEFEFEFEFEFE000000A9
:1041300000FEFE0000DADADADAFE00DADADADADADB
:10414000DA00DADAFFFFFFFFDAFF00FFFFFFFFFF11
:10415000DAFF00FFFF0000FFDA00DADAFF0000DA22
:10416000DA00DADADADA000000000000FEFEFEFE15
:10417000FEDADADA000000FEFEDADADADA00DA0075
:10418000FEDAFFFFFFDA00FFFFFF0000FFFFDAFFAC
:10419000FFFF0000FFFFDAFFFFFFFFFFFFFFDAFF77
:1041A000FFDAFFFFFFDADA00FF00DADADA00FFFFFA
:1041B000FF0000DADA00000000000000DA00000072
:1041C0000000FF0000DA00000000FFFF0000DADA64
:1041D000DAFE00FF0000000000FEFE0000FEFEFE12
:1041E000FEFEFEFEFEFEFEFEFE00DADADADA00FF7A
:1041F000FF00DADADADA00FF0000DADADADA0000F1
:1042000000DADADA0000FFFF00DADA0000FFFFFF71
:1042100000000000FFFFFF00FEFEFEFE000000FEAB
:10422000FEFEFEFEFEFEFEFEFEFEFEFEFE000000A8
:1042300000FEFE0000DADADADAFE00DAFFFFFFDA6B
:10424000DA00DAFFFFDADADADA00DADADADADADA38
:10425000DADADADADADADADADADADAFFFFFFDADA4F
:10426000DADAFFFFFFFFFFDAFF000000FEFEFEFECE
:10427000FEDADADA00000000FEFFFFDADA00DA0028
:10428000FEDADADADADA0000FEDADADADA00FFFF8A
:1042900000DADADADAFFFFFF00FFFFFFDAFFFFFFE5
:1042A000FFFFFFFFFF00FFFFFFDAFFFF0000FFDA65
:1042B000FF00FFFFFFFF00DA000000FF0000FFDA51
:1042C000FF000000FFFFDADADA00FFFF0000DADAB1
:1042D000DA00FFFFFF000000000000000000FEFE0B
:1042E000FEFEFEFEFEFEFEFEFE0000FFFFDA00FF09
:1042F000FFFFFFFFFF00FFFF000000FFFF000000C7
:10430000FEFFFFFFDA00FFFF00DADA0000FFFFFF29
:1043100000000000FFFFFF00FEFEFE00000000FEA8
:10432000FEFEFEFEFEFEFEFEFEFEFEFEFE0000DACD
:10433000DAFEFE00DADAFFFFDAFEDADADADADADA01
:10434000DA00DAFFFFFFDADAFFDAFFFFFFFFDAFF5A
:10435000FFDAFFFF0000DAFF00DAFFFF0000DAFFFC
:1043600000DAFFFFFFFFDADAFFDA00FEFEFEFEFEF4
:10437000FEFFDADA00FFFF00FEDADADA00FFFFDA2A
:1043800000FFFFDA00DAFFFF00FFFFFF00DAFFFFA8
:104390000000FFFFDA00FFFF0000FFFFDA00FFFF71
:1043A00000FFFFFFDADAFFFF00DADAFF00000000AB
:1043B00000FEDADA00FFFF0000FE00DA0000000075
:1043C0000000FFDA0000000000FE0000DA0000003C
:1043D000DAFEFE000000000000FE00FFFFFFFF000D
:1043E000FEFEFE00000000FEFEFFFFDADADAFF004C
:1043F00000DADADADADA0000FEDADADADADA00003B
:10440000FEDADADA000000FEFEDA0000000000FE4C
:10441000FE0000FFFFFF00FEFE0000FFFFFFFF00A9
:10442000FEFE000000000000FEDA00FEFEFEFEFEC2
:10443000FEFFDADA00FEFEFEFEDADADA00FFFF0047
:10444000FEFFFFDADAFFFFFF0000FFFFDA0000FFE8
:10445000FFFF00FFDADADA00FFFF00FFDADADAFF47
:10446000FFFFFFFFDADAFFFFFFFEFEFE000000DACB
:10447000DAFEFE00DAFFFFFFDAFE00DAFFFFDADA2B
:10448000DAFE00DADADADADADA00DADA909090DAFA
:10449000DA00DA9090909090DA00DA909090909014
:1044A000DA00009090909090DADA000000FEFEFEB4
:1044B000FEFFDADADA00FEFEFEDADADADADA00FE37
:1044C000FEDADADADADA00FEFEDA909090DADA0072
:1044D000FE9090909090DA00FE9090909090DA008C
:1044E000FE90909090900000FEFEFEFE000000D82E
:1044F000D8FEFE00FFFFD8FFD8FE00FFD8D8D8D8DE
:10450000D800D8D8D8D8D8D8D800D8909090D8D8B3
:10451000D8D89090909090D8D8D89090909090D8EB
:10452000D8D89090909090D8D8FF0048909090481C
:10453000DAFF0000484848DADA00FF00DADADADAAF
:10454000DA00FFFF0000DADADAFE00000000000007
:1045500000FEFE00FFFFFF00FEFEFE000000000068
:10456000FEFEFEFEFEFEFEFEFE489090904800FF1E
:1045700000DA484848DA00FF00DADADADA00FF0049
:10458000FEDADA0000FFFF00FE000000000000FE7F
:10459000FE00FFFFFF00FEFEFE0000000000FEFE2A
:1045A000FEFEFEFEFEFEFEFEFED84890909048D82D
:1045B000D800D8484848D8D8D8FED8D8D8D8D8D8DD
:1045C000D8FE0000D8D8D8D8D8FEFE0000000000E1
:1045D000FFFEFEFEFEFE00FFFFFEFEFEFEFE0000F2
:1045E00000FEFEFEFEFEFEFEFEFEFE9FFFFF9FFEA5
:1045F000FEFEFFFFFFFFFFFFFEFEFF9F00009FFF8D
:10460000FEFF9F9FFFFF9F9FFFFF00FFFFFFFF0039
:10461000FFFF00FFFFFFFF00FFFF9F9FFFFF9F9F28
:10462000FFFEFF9F00009FFFFEFEFFFFFFFFFFFF5B
:10463000FE9FFE9FFFFF9FFE9FFEFFFEFEFEFEFF12
:10464000FEFEFEFFFFFFFFFEFEFE9FFEFEFEFE9F44
:10465000FEFEFE9F9F9F9FFEFEFEFEFEFEFEFEFEF6
:10466000FEFEFEFE9F9FFEFEFEFEFF9F00009FFFE0
:10467000FEFF9F9FFFFF9F9FFFFF00FFFFFFFF00C9
:10468000FFFF00FFFFFFFF00FFFF9F9FFFFF9F9FB8
:10469000FFFEFF9F00009FFFFEFEFFFFFFFFFFFFEB
:1046A000FEFEFE9FFFFF9FFEFEFEFEFE9F9FFEFEA4
:1046B000FEFEFEFEFEFEFEFEFEFEFE9F9F9F9FFE96
:1046C000FEFE9FFEFEFEFE9FFEFEFEFFFFFFFFFEC4
:1046D000FEFEFFFEFEFEFEFFFE9FFE9FFFFF9FFE13
:1046E0009FFEFFFFFFFFFFFFFEFEFEFEFEFEFEFE43
:1046F000FEFEFEFEFEFFFFFFFFFEFEFFFF9F00002F
:104700009FFE9FFF9F9FFFFF9FFE9FFF9F9FFFFFBB
:104710009FFEFEFFFF9F00009FFEFEFEFEFFFFFFCD
:10472000FFFEFEFEFEFEFEFEFEFEFEFEFEFEFEFEA8
:10473000FEFEFE9FFEFEFEFEFEFFFFFEFFFE9FFE54
:10474000FE9FFF9FFEFFFE9FFE9FFF9FFEFFFE9FBF
:10475000FEFFFFFEFFFE9FFEFEFEFE9FFEFEFEFE34
:10476000FEFEFEFEFEFEFEFEFEFEFEFEFEFEFEFE69
:10477000FEFEFEFEFE00FEFEFEFEFEFEFEFFFE0054
:10478000FEFEFEFEFEFFFE00FEFEFEFEFEFFFEFF44
:10479000FEFEFE00FEFFFEFFFEFEFE00FEFFFEFF31
:1047A000FEFEFEFFFEFFFEFFFEFEFEFFFEFFFEFF23
:1047B000FEFEFEFFFE00FEFFFEFEFEFFFE00FEFF11
:1047C000FEFEFEFFFEFEFE00FEFEFEFFFEFEFEFE05
:1047D000FEFEFEFFFEFEFEFEFEFEFE00FEFEFEFEF6
:1047E000FEFEFEFEFEFEFEFEFEFEFEFEFEFEFEFEE9
:1047F000FEFEFEFEFEFEFEFEFEFE00FFFFFFFFFFD2
:10480000FFFEFEFEFEFEFEFEFEFEFEFEFEFE0000C3
:10481000FFFEFEFEFEFEFEFEFEFEFEFEFE00FFFFB3
:10482000FFFEFEFEFEFEFEFEFEFEFEFEFEFEFEFEA7
:10483000FEFEFEFEFEFEFEFEFEFF0000FEFEFEFE93
:10484000FEFEFEFEFEFEFEFEFEFFFFFFFFFFFF0080
:10485000FEFEFEFEFEFEFEFEFEFFFFFFFF0000FE70
:10486000FEFEFEFEFEFEFEFEFEFEFEA7A7A7A7FEC4
:10487000FEFEA7A7FFA7A7A7FEA7A7FFA7A7FFA7BB
:10488000A7A7A7A7FFFFA7A7A7A7A7A7A7FFA7A7B0
:10489000A7A7A7FFA7A7FFA7FEA7A7A7A7A7A7A7A1
:1048A000FEFEA7A7A7A7A7A7A7FEFEA7A7A7FEFE8E
:1048B000A7FEA7A7A7A7A7A7A7A7A7FFA7A7FFA781
:1048C000A7A7A7A7FFFFA7A7A7A7FFA7FFA7A7A718
:1048D000A7A7A7FFA7A7FFA7A7FEA7A7A7A7A7A761
:1048E000A7FEFEA7A7A7A7A7FE0019FFFFFFFFFFD0
:1048F000F619FF19191919191919FF1900000000E3
:104900000019FF1900FF00000019FF1900F6000050
:104910000019FF19000000190019FF190000190003
:104920001919FF190019001900F6FFFFF6FFFF190A
:1049300000191919191919FF19000000000000F6D3
:1049400019000019190000F619000019190000FFDC
:10495000190019FFF61900FF1919FFFF19FF00F6DA
:10496000190019F6FF1900FF1919FF19FE19191975
:104970001919FF19FEFE19FF191919FFFFFFFFFF93
:10498000FF19FF19190019FE1919FF19190019FE4D
:104990001919FF1900190019FE00FFFE00FE19FE8B
:1049A000000019FFFFFFF6FFFF191919191900FF81
:1049B000191919FFF61919FF19FFFFFFFFFFFFFF74
:1049C0001919FE19001900191919FE1900190019F1
:1049D00019FE190019FE19FF1900FE19FE00FEFF4D
:1049E00000FFFFFFFFF6F61900FEFEFEFEFEFEFED4
:1049F000FEFEFEFEFEFEFEE7E7FEFEFEFEFEE7FF1B
:104A0000FFFEFEFEE7FFFFFFFFFEFEE7FFFFFFFFEB
:104A1000FFFEFEE7FFFFFFFFFFFEE7FFFFFFFFFFD9
:104A2000FFFEE7FFFFFFFFFFFFFEE7FFFFFFFFFFC8
:104A3000FFFEE7FFFFFFFFFFFFFEE7FFFFFFFFFFB8
:104A4000FFFEE7E7FFFFFFFFFFFEFEE7FFFFFFFFC1
:104A5000FFFEFEE7E7FFFFFFFFFEFEFEE7E7E7E7FB
:104A6000FFFEFEFEFEFEE7E7E7FEFEFEFEFEFEFEAA
:104A7000FEFEFEFEFEFEFEE7E7FEFEFEFEFEE7FF9A
:104A8000FFFEFEFEE7FFFFFFFEFEFEE7FFFFFFFF6C
:104A900000FEFEE7FFFF0000FFFEE7FFFF00FFFF55
:104AA00000FEE7FFFFFFFF00FFFEFEFEFEFEFEFE34
:104AB000FEFEE7FEFEFEFEFEFEFE00E7FEFEFEFE42
:104AC000FE00FFFFFFE7FEFEFE0000FFFFFFE7FE28
:104AD000FE00FF00FFFFE7FEFEFFFFFF00FFFFE716
:104AE000FEFF00FFFFFFFFE7FEFEFE9F9F9F9FFE72
:104AF000FEFE9FEFF7F7EF9FFE9FEFFFFFFFFFEF39
:104B00009F9FF7FFFFFFFFF79F9FF7FFFFFFFFF755
:104B10009F9FEFFFFFFFFFEF9FFE9FEFF7F7EF9FD6
:104B2000FEFEFE9F9F9F9FFEFEFEFE00009F9F00D9
:104B3000FEFE00FFFF9F00FEFE00FF9F9F0000FEA5
:104B4000FE009F9F9F9F0000FE009F9F9FFFFF9F73
:104B50009F009F9F9FFFFFFF9FFE009F00000000A0
:104B60009FFE009F00FFFF009FFEFE00000000FE72
:104B7000FEFE00FFFF9F9FFEFE009F9F9F9F00FE87
:104B8000FE009F9F9FFFFF9F9F009F9F9FFFFFFF34
:104B90009FFE009F000000009FFE009F00FFFF009F
:104BA0009FFE009F9F0000009FFE009F9F0000004F
:104BB0009FFE009F9F9F9F9F9FFE009F00FF9F9FC4
:104BC0009FFE009F000000FF00FE00009F00009F6E
:104BD00000FE0000009F9F9F9FFE009F00000000BE
:104BE00000FEFE009F9F00FF00FE009F9F9F9F9F73
:104BF0009FFE009F00FF9F9F9FFE009F000000FF01
:104C000000FE009F0000000000FE00009F00009FCB
:104C100000000000009F9F9F9F009F000000000079
:104C200000FE009F9F00FF0000FEFEFEFEFE5B5B9D
:104C30005BFEFEFE5B5BFFFFFFFEFE5BFFFFFFFF19
:104C4000FFFE5BFFFFFFFFFFFF5BFFFF5B005BFF04
:104C5000FF5BFF5B000000005B5BFF0002020000E7
:104C6000005BFF0000020000FFFEFEFEFEFE5B5B3D
:104C70005BFEFEFE5B5BFFFFFFFEFE5BFFFFFFFFD9
:104C8000FFFE5BFFFFFFFFFFFF5BFFFF5B005BFFC4
:104C9000FF5BFF5B005B00005B5BFF0004075B00EA
:104CA000005BFF005B070400FFFEFEFEFE5B5B5B3C
:104CB0005BFEFE5BFFFFFFFFFFFE5BFF5B005BFF3A
:104CC000FFFEFFFF005B00005B5BFF005B07040073
:104CD000005BFF005B070700FF5BFF00005B00FF5E
:104CE000005BFFFF005B00FF005BFF00000000FFB8
:104CF00000FE5BFF00005BFF00FEFE5BFFFFFFFFAF
:104D0000FFFEFEFE5B00FF00FFFEFEFEFF00000058
:104D100000FEFEFEFFFF5BFF5BFEFEFEFEFEFFFFF2
:104D2000FFFEFEFEFEFEFEFEFE5BFF00005B00FFE0
:104D300000FE5BFF00005BFF00FEFE5BFFFFFFFF6E
:104D4000FFFEFEFE5B00FF00FFFEFEFE5B000000BC
:104D500000FEFEFEFF0000FF00FEFEFEFEFF5BFF0A
:104D60005BFEFEFEFEFEFFFFFFFEFFFFFFFFFFFFFD
:104D7000FFFEFEFFFF5BFF00FFFEFEFE5B0000008C
:104D800000FEFEFE5B00000000FEFEFEFF000000D5
:104D900000FEFEFEFF0000FF00FEFEFEFEFF5BFFCA
:104DA0005BFEFEFEFEFEFFFFFFFEFEFE00005B5B05
:104DB0005BFEFE005B5B000000FE005B0000FFFF8F
:104DC000FF005B00FF5B5B5B5B005B005B5B5B00B2
:104DD000005B005B5B00005B5B5B005B005B5B5B45
:104DE0005B5B005B005B5B5B5BFEFEFE00005B5B96
:104DF0005BFEFE005B5B000000FE005B00005BFFF3
:104E0000FF005B00FF5B5B5B5B005B005B5B5B0071
:104E100000005B5B5B5B005B5B5B005B5B005B5BA9
:104E20005B5B005B00005B5B5B5B5B5B0000FEFE53
:104E3000FE000000005B00FEFEFFFFFF0000000020
:104E4000FE5B5B5B5BFF005B00000000005B5B00E8
:104E5000005B5B5B5B005B005B5B5B5B5B000000C4
:104E60005B5B5B5B5B5B00005BFEFEFE00005B5B15
:104E70005BFEFE005B5B000000FE005B0000FFFFCE
:104E8000FF005B00FF5B5B5B5B005B005B5B5B5B96
:104E90005B005B5B5BFFFF5B5B5B005BFFFF00FF3F
:104EA0005B5B005BFFFF00FF5BFEFEFE00005B5BE9
:104EB0005BFEFE005B5B5B0000FE005B5B0000FFD7
:104EC000FF005B5B00FF5B5B5B005B005B5B5B5B56
:104ED0005B005B005B5B5B5B5B5B005B5BFFFF5BEB
:104EE0005B5B005BFFFF00FF5B5B5B5B0000FEFE4C
:104EF000FE000000005B00FEFEFFFF5BFF00000005
:104F0000FE5B5B5B5BFF005B005B5B5B5B5B5B00BB
:104F1000005B5B5B5B5B5B005B5B5BFFFF5B5B00AA
:104F20005B5BFF00FFFF5B005BFEFEFE0000FF5BC4
:104F30005BFEFE00FF5B5B5B5BFE00FF5B5B5B5B46
:104F400000005B5B5B5B5B5B00005BFFFF5B5B5BD5
:104F5000005BFF00FFFF5B005B5BFF00FFFF5B0090
:104F60005B5BFFFFFFFF5B5B00005B5B00FEFEFE29
:104F7000FE005B5B5B00FEFEFE5B5B5B005B00FEBE
:104F8000FE5B5B00005B00FEFE5B5B005B5B5B004F
:104F9000FE5B005B5B5B5B00FE5B005B5B5B00FEE4
:104FA000FE005B5B5B005B00FEFEFEFE00005B5BE9
:104FB0005BFEFE00FF5B5B5B00FE00FF5B5B5B007C
:104FC0005B005B5B5B5B5B005B00FFFF5B5B5B0055
:104FD0005BFF00FFFF5B005B5BFF00FFFF5B005BB5
:104FE0005BFFFFFFFF5B5B5B00005B0000FEFEFE04
:104FF000FE5B5B5B5B00FEFEFE5B5B00005B00FE3E
:10500000FE5B005B5B5B00FEFE5B005B5B5B5B0073
:10501000FE005B5B5B5B5B00FE005B5B5B0000FEBE
:10502000FE5B5B5B005B5B00FEFEFEFE0000FF5B69
:105030005BFEFE00FF5B5B5B5BFE00FF5B5B5B5B45
:1050400000005B5B5B5B5B5B00005B5BFFFF5B5BD4
:1050500000FF5BFF00FFFF005BFF5BFF00FFFF0047
:105060005BFF5BFFFFFFFF5B00005B0000FEFEFEDF
:10507000FE005B5B5B00FEFEFE5B5B5B005B00FEBD
:10508000FE5B5B5B005B00FEFE5B5B5B005B5B00F3
:10509000FE5B5B005B5B5B00FE5B5B005B5B0000E1
:1050A000FE00005B5B005B00FEFEFEFEFEFE0000FD
:1050B00000FEFEFE00005B5B5BFEFE005B00FFFF90
:1050C000FFFE005B5BFF005B5B005B5B5B5B005BB1
:1050D0005B005B5B5B5B5B005B5B0000005B5B0042
:1050E000005B5B5B5B00005BFF000000FEFEFEFE02
:1050F000FE5B5B5B0000FEFEFEFFFF005B5B00FEF5
:10510000FE5B5B00FF5B5B00FE5B005B5B5B5B5B16
:10511000005B005B5B5B5B5B005B5B5B5B5B0000A6
:105120005BFF5B0000005B5B5BFEFEFEFEFE0000C3
:1051300000FEFEFE00005B5B00FEFE005B5BFFFF0F
:1051400000FE005B5BFF5B5B00005B00005B5B5B8A
:1051500000005BFF5B005B5B5B005B5B5B5B005BC2
:10516000005B5B5B5B5B5B00FF000000FEFEFEFE26
:10517000FE5B5B5B0000FEFEFEFFFFFF5B5B00FE75
:10518000FE5B5B5BFF005B00FE5B5B5B5B005B5B96
:1051900000005B5B005BFF5B00005B005B5B5B5BDD
:1051A0005BFF5B005B5B5B5B005B005B005B0000CD
:1051B000005B5B005B005B5B5B005B5B005B5B5B06
:1051C0005BFE005B005B5B0000FEFE005B005B5B68
:1051D0005BFE005B5B5B00005BFE005B5B5B5B00A0
:1051E00000FEFE00000000FEFE5B005B005B5B5B00
:1051F000005B005B005B00005B005B0000005B5B32
:105200005B005B5B000000005BFE00005B5B5B5BC8
:1052100000FE005B5B5B5B5B5BFEFE005B5B5B5B06
:1052200000FEFEFE0000000000000000005B000029
:10523000005B5B5B005B005B005B5B5B5B0000003B
:10524000FE5B00005B005B00FE005B5B005B00FE42
:10525000FE0000000000FEFEFE00FEFEFEFEFEFE62
:10526000FEFEFEFEFEFEFEFEFE5B5B5BFFFFFFFF43
:105270005B005B0000FFFF005BFE005B5B00005B10
:105280005BFE005B005B5B5B5BFEFE000000005BA7
:105290005BFE005B5B5B000000FE005B5B5B5B003A
:1052A00000FE000000000000FE5B5B5BFFFF00FFF4
:1052B0005B005B00FFFFFFFF5B005B5B00FFFF002D
:1052C0005BFE005B5B00005B5BFE005B00000000C0
:1052D0005BFEFE005B5B5B5B00FE005B5B5B5B5B46
:1052E0005BFEFE0000000000005BFF00FFFF5B00B4
:1052F000005BFFFFFFFF005B005B00FFFF005B5BED
:10530000005B5B00005B5B5B005B5B5B00005B006A
:10531000FE0000005B5B5B00FE00FEFE000000FE86
:10532000FEFEFEFEFEFEFEFEFE5BFFFFFFFF5B5B82
:10533000005B00FFFF005B5B5B005B00005B5B00F2
:1053400000FE00005B5B00005BFEFEFE0000005BF9
:105350005BFEFEFEFEFE00005BFEFEFEFE005B5BF3
:105360005BFEFEFEFE00000000005B5B5B005B007E
:10537000FE005B5B005B005B000000005B5B005BB2
:10538000005B5B5B005B005B5B5B5B5B5B0000008F
:10539000005B5B5B0000FEFEFE5B5B5B5B00FEFE9A
:1053A000FE00000000FEFEFEFEFFFFFFFF5B5B5BFA
:1053B0000000FFFF005B5B5B005B00005B5B0000CD
:1053C00000FE5B5B5B0000005BFEFEFE5B0000001E
:1053D0005BFEFEFEFE00FF0000FEFEFE00FF000082
:1053E00000FEFEFE00000000005B5B5B005B5B00FC
:1053F000FE000000005B005B005B5B5B005B005B32
:105400005B5B5B5B5B00005B005B5B5B5B5B0000B3
:10541000FE5B5B5B5B0000FEFE005B5B5B5B00FEBC
:10542000FE000000000000FEFEFF5BFFFFFFFF5BD1
:1054300000005B00FFFF005B5B005B5B00005B5BF1
:1054400000FE005B5B5B5B0000FEFE005B5B5B00E5
:105450005BFEFEFE0000005B5BFEFEFE005B5B5B36
:105460005BFEFEFEFE0000000000005B5B005B00D8
:10547000FE005B5B005B5B00FE0000005B5B005BB3
:10548000005B5B5B005B005B005B5B5B5B005B5B33
:10549000005B5B5B00000000FE5B0000000000FEA4
:1054A000FE00FE000000FEFEFE5B5B5B5B5B5BFFE5
:1054B0005B5B5B5B5B5B005B5B005B5B5B00005BA8
:1054C0005B005B00005B5B005B00005B005B5B0004
:1054D0005BFE005B5B005B005BFEFE005B5B000055
:1054E0005BFEFEFE00000000005BFF5B5B5B5B5B46
:1054F0005B5B5B00005B5B5B5B5B5B005B00005BC3
:105500000000005B5B5B5B00005B5B005B5B005B68
:10551000005B5B005B005B00FE00005B005B00FE6D
:10552000FE0000000000FEFEFE5B5B5B00005BFF18
:105530005B0000005B5B005B5B005B5B5B5B5B00DD
:105540005B005B5B5B5B005B00FE005B005B005B2A
:105550005BFE005B5B005B5B5BFEFE005B005B5B1E
:1055600000FEFEFE00000000005BFF5B000000008C
:10557000005B5B005B5B5B5B5B5B5B005B5B5B5B8C
:105580000000005B005B005B00005B5B005B5B5B43
:1055900000005B5B5B005B00FE5B005B005B00FE92
:1055A000FE0000000000FEFEFE00010A0B000203E8
:1055B0000C0D0004050E0F0002030C0D0000010A83
:1055C0000B0006071011000809121300060710113E
:1055D0000014151E1F001617202100181922230081
:1055E000161720210014151E1F001A1B2425001C4D
:1055F0001D2627001A1B24250028293233002A2BB8
:105600003435002C2D3637002A2B3435002829322A
:1056100033002E2F38390030313A3B002E2F3839E5
:105620000029283332022B2A3534022D2C3736023A
:105630002B2A35340229283332022F2E39380231F1
:10564000303B3A022F30393A023C3D3E3F00404168
:10565000424300444546470048494A4B004C4D4EA2
:105660004F00505152530050545253005152545510
:1056700000532956330029533356025D5D5E5E00A8
:105680005D5D5E5D025F605F6000605F605F026342
:10569000646566006C6C6F6F016D6D6E6E016D6D93
:1056A0006E6E016767686801696A6868076B6C6994
:1056B0006A00707073730171717474017272757520
:1056C00001717174740175757D7D0176767E7E0140
:1056D00077777F7F017878808001797A8182007B7B
:1056E0007C8384007A798281027C7B848302767653
:1056F000868601777887880076768686017877882F
:10570000870279798989017A7B8A8B0079798989FD
:10571000017B7A8B8A027C7D8C8D007E7F8E8F0050
:105720007C7D8C8D0080819091007D7C8D8C027FB2
:105730007E8F8E027D7C8D8C02818091900282838F
:10574000929300848594950082839293008485943B
:1057500095000000000000010001010101010100AD
:105760000100010100000001010100010000000032
:105770000001494A4B4C4F505152555657585A5BAD
:105780005C5D4D4E4B4C53545152595657585A5ECE
:105790005C5D0002020000DD00FF0002020000F676
:1057A00000FF0002010106000100E000FF0001010E
:1057B0000007900000E208050000FF000202010857
:1057C00050010853010854010850010851010850C4
:1057D00001085101084F01084E01084901084B0119
:1057E000084801084601084201084401084101082F
:1057F0004001083B01083D01083A00050000FF0098
:1058000002020000FC00083C0108440108490108AC
:105810004601084001084801084D01084A010849AD
:1058200001084201084A01084F01084C01084301E0
:10583000084C01085101084901084E0108490000BF
:10584000FA01084501084D01085201084F010846B8
:1058500001084E0108530108500108480108500191
:10586000085501085201084A010852010857010869
:105870005401084B01085301085801085501084C10
:1058800001084901085401085901085601085A0144
:10589000050000FF00020201084501084901084611
:1058A00001084A01084701084B01084801084C015A
:1058B000084901084D01050000FF000202010851DE
:1058C0000108550108520108560108530108570103
:1058D000085401085801085501085901050000FF46
:1058E00000020201083801083701083401083301B9
:1058F000082B01082701082301082201081F0108BD
:105900001E01081901050000FF000200000000034D
:10591000083203083603083703083903083E030832
:105920004203084302084502084A02084E02084A98
:1059300002084E02084A02084E02084A02084E02B5
:10594000050000FF0002020008320308310108329E
:1059500003083703083E04083D01083E04084304D9
:10596000083E04084305084705084901084A060897
:105970004E02084F07084A18050000FF0002020007
:10598000081901081A01081902081801082E01084F
:105990002F01082E02082D010823010824020823E4
:1059A00001050000FF00020100081C030827010890
:1059B0001E01082401082C010830010822010835C5
:1059C00001082F01082101082701082C01081F01E7
:1059D000082501081D01082A01083002081D0108D8
:1059E0002A01083002081D01082A010830020500BA
:1059F00000FF00020200081B03081F01082601081F
:105A00002701082501082801082B01082E01083468
:105A100001083501082E010831010832010838015A
:105A2000082801081F01082E01083501082801086F
:105A30001F01082E01083501082801081F01082E42
:105A400002050000FF00020201084001083F0408AF
:105A50004901084A01084B08083C01083B05084574
:105A600001084601084701084801084901084A01A0
:105A7000084B03083801083703082D01082E0108D8
:105A80002F01083001083103082C06050000FF0033
:105A900000009257000000000000009A570000002C
:105AA00000000000A25700000000010000AD5700F8
:105AB000000000000000BB5700000000000000FFD5
:105AC0005700000000000000945800000000000093
:105AD00000E058000000000000000959000000002C
:105AE000000000BA58000000000000004459000007
:105AF00000000000007C5900000000000000A559D3
:105B000000000000000000F259000000000000004A
:105B1000455A0000000000FF06015300C00000B01D
:105B2000075500C0000090436400C10000B1075554
:105B300000C10000913B6400C20200B2077900C2BC
:105B40000200922B6400C30300B307450093034691
:105B500010903E6400913B6400922B6400930346D6
:105B60000890426400913C640092326400930346C2
:105B70000890406408426400930346089043640020
:105B8000913B64009237640093034610903E64009A
:105B9000913B64009237640093034608904264008E
:105BA000913E64009232640093034608904064087A
:105BB000426400913C640093034608904364009162
:105BC0003B6400922B640093034610903E64009166
:105BD0003B6400922B640093034608904364009159
:105BE0003E64009232640093034610904764009133
:105BF0004364009232640093034607C10101C0016F
:105C000000904A6400914764009237640093034611
:105C100008922B64082B640093034608904C6400A0
:105C200091476400923764009303461092366400F3
:105C300093034607C10001C00000904D64009145E8
:105C400064009235640093034610904864009145C7
:105C500064009235640093034608904C64009146BA
:105C600064009230640093034608904A64084C64D0
:105C70000093034608904D6400914564009235649A
:105C80000093034610904864009145640092356487
:105C90000093034608904C640091486400923C6471
:105CA0000093034608904A64084C640091466400DF
:105CB00093034608904D640091456400924164004E
:105CC00093034610904D6400914564009235640042
:105CD00093034608904C640091436400923C640036
:105CE00093034608904A6408486400914064009217
:105CF00030640093034607C10101C00100904A646B
:105D00000091436400923E64009303461092326413
:105D10000093034607C1000191426400923264007F
:105D20009303460EC00002903E6400913C640092D2
:105D30002664009303460890436400913B640092FC
:105D40002B640093034610903E6400913B640092E4
:105D50002B64009303460890426400913C640092D7
:105D60003264009303460890406408426400930341
:105D7000460890436400913B6400923764009303AB
:105D80004610903E6400913B640092376400930398
:105D9000460890426400913E64009232640093038E
:105DA000460890406408426400913C6400930346B6
:105DB0000890436400913B6400922B640093034677
:105DC00010903E6400913B6400922B640093034664
:105DD0000890436400913E6400923264009303464D
:105DE000109047640091436400923264009303462C
:105DF00007C10101C00100904A640091476400920C
:105E000037640093034608922B64082B64009303C5
:105E10004608904C640091476400923764009303F5
:105E200046109236640093034607C10001C000008B
:105E3000904D6400914564009235640093034610D0
:105E400090486400914564009235640093034608CD
:105E5000904C6400914664009230640093034608BD
:105E6000904A64084C640093034608904D64009186
:105E70004564009235640093034610904864009195
:105E80004564009235640093034608904C64009189
:105E9000486400923C640093034608904A64084CAE
:105EA00064009146640093034608904D6400914558
:105EB00064009241640093034610904D6400914544
:105EC00064009235640093034608904E6400914A42
:105ED0006400923E640093034608904A64084E644E
:105EE00000914864009232640093034608C00100A8
:105EF000904F64009147640092376400930346001A
:105F0000C101180000C0000090436400913B640090
:105F1000922B640093034608904764084A64084C37
:105F2000640091436400923C640093034610904BDC
:105F300064009142640093034608904C64009143CE
:105F400064009230640093034610904B64009142C9
:105F5000640093034608C10100C00100904C640036
:105F600091436400923C64009303461092306400B5
:105F700093034608904E6400914564009232640099
:105F8000930346109230640093034608C10000C09A
:105F90000000904A640091436400922F64009303D0
:105FA0004600C000109049640091426400922E6443
:105FB0000093034608C00100904A640091436400C6
:105FC000922F640093034610913B64009232640068
:105FD00093034608C00000913E640092376400932A
:105FE00003461103460890436400913E6400922BDF
:105FF0006400930346089045640847640093034691
:10600000089048640091406400923C640093034609
:1060100010904764009230640093034608904864EF
:1060200000914364009230640093034610904764EB
:106030000093034607C10100C0010190486400912C
:10604000426400923E6400930346109232640093CF
:10605000034607C10000C00001904A6400914264F9
:1060600000923E64009303461090486400930346F8
:106070000890476400913E640092376400930346A1
:106080001090466400922B64009303460890476486
:1060900000913E6400922D64009303461090486482
:1060A0000091426400922E640093034608C00100F0
:1060B000904A640091436400922F64009303461059
:1060C000913E64009232640093034608913B640061
:1060D000923764009303460AC0000690436400931D
:1060E000034608904B64009143640092306400932F
:1060F000034610904A640093034608904B64009155
:10610000466400923C640093034610904F640093F1
:10611000034607C10101C00100904D640091456430
:10612000009235640093034610922964009303465D
:1061300008904B64009145640092296400930346E3
:1061400010034607C10001C00000904A640091415D
:106150006400922E640093034610904964009140BD
:106160006400922D640093034608C00100904A64C5
:106170000091416400922E640093034610913E64A6
:1061800000930346089143640092336400930346EE
:1061900000C00010922B64009303460890486400EE
:1061A00092336400930346109046640093034608BC
:1061B0009045640091436400923964009303461053
:1061C000904464009303460890456400913D640048
:1061D000922D640093034610904964009303460790
:1061E000C10101C00100904C6400913D64009239EE
:1061F000640093034610922D640093034608904E6A
:106200006400914364009239640093034610922D18
:10621000640093034608C10000904A640091426400
:1062200000923264009303461091426400923264FB
:10623000009303460891436400923464009303463C
:1062400008034608914464009235640093034608AD
:10625000914564009236640093034600C00010919B
:106260003E640092326400930346089142640092B7
:106270003E640093034608034608903E6400913C48
:10628000640093034608FF06014500FF2F0000C38A
:106290000300C20200C10100C00000B0077F00B1CE
:1062A000077F00904E7F00B00B7F00914F7F00B1C1
:1062B0000B7F00FF06015301904F7F00B00B7F0161
:1062C00091507F00B10B7F0190507F00B00B7F0198
:1062D00091517F00B10B7F0190517F00B00B7F0087
:1062E00091527F00B10B7F0190527F00B00B7F0273
:1062F0000B0000B10B0003914D7F00B10B7F0190AB
:106300004C7F00B00B7F00B10B0001B00B0000917F
:106310004D7F00B10B7F01904C7F00B00B7F00B12F
:106320000B0001B00B0000914B7F00B10B7F009080
:106330004A7F00B00B7F00B10B0001B00B00009151
:106340004B7F00B10B7F01904A7F00B00B7F00B103
:106350000B0001B00B000091497F00B10B7F019051
:10636000487F00B00B7F00B10B0001B00B00009123
:10637000497F00B10B7F0090487F00B00B7F00B1D8
:106380000B0001B00B000091477F00B10B7F019023
:10639000467F00B00B7F00B10B0001B00B000091F5
:1063A000477F00B10B7F0190467F00B00B7F00B1AB
:1063B0000B0001B00B000091457F00B10B7F0090F6
:1063C000437F00B00B7F00B10B0001B00B000091C8
:1063D000457F00B10B7F0190437F00B00B7F00B180
:1063E0000B0001B00B000091417F00B10B7F0190C9
:1063F0003F7F00B00B7F00B10B0001B00B0000919C
:10640000417F00B10B7F00903F7F00B00B7F00B158
:106410000B0001B00B0000913D7F00B10B7F01909C
:106420003B7F00B00B7F00B10B0001B00B0000916F
:106430003D7F00B10B7F01903B7F00B00B7F00B12F
:106440000B0001B00B000091397F00B10B7F009071
:10645000377F00B00B7F00B10B0001B00B00009143
:10646000397F00B10B7F0190377F00B00B7F00B107
:106470000B0001B00B000091357F00B10B7F019044
:10648000337F00B00B7F00B10B0001B00B00009117
:10649000357F00B10B7F0090337F00B00B7F00B1E0
:1064A0000B0001B00B000390377F00B00B7F019011
:1064B000397F00B00B7F01903A7F00B00B7F0190D5
:1064C0003C7F00B00B7F01903F7F00B00B7F0190BD
:1064D000427F00B00B7F0190457F00B00B7F0090A2
:1064E0004A7F00B00B7F0190517F00B00B7F01907D
:1064F0005C7F00B00B7F010B000290510114510131
:10650000009148010C480183A97DFF06014500FF69
:106510002F000000C20200C10100C00000B0077FD0
:1065200000B1077F00B2077F00903E7F00B00B7F75
:106530000490407F00B00B7F0490427F00B00B7F3F
:106540000490437F00B00B7F00913B7F00B10B7F35
:106550000092375A10903E7F00B00B7F00913B7F36
:1065600000B10B7F00922B5A0790437F00B00B7F46
:1065700000913B7F00B10B7F00922B5A102B5A07E2
:106580002B5A10903B7F00B00B7F0091377F00B1FA
:106590000B7F08903E7F00B00B7F00913B7F00B1E6
:1065A0000B7F0790437F00B00B7F00913E7F00B1CF
:1065B0000B7F00922B5A0890477F00B00B7F009111
:1065C000437F00B10B7F00922B5A08904A7F00B0A6
:1065D0000B7F0091477F00B10B7F0092375A0F90DD
:1065E000437F00B00B7F00913E7F00B10B7F009294
:1065F0002B5A08904A7F00B00B7F0091477F00B173
:106600000B7F00922B5A102B5A072B5A10903E7F6B
:1066100000B00B7F00913B7F00B10B7F0890437F60
:1066200000B00B7F00913E7F00B10B7F0790477F4A
:1066300000B00B7F0091437F00B10B7F00922B5A7B
:1066400008904A7F00B00B7F0091477F00B10B7F1D
:1066500000922B5A08904D7F00B00B7F00914A7F2B
:1066600000B10B7F0092375A0F2B5A08904C7F00D5
:10667000B00B7F0091487F00B10B7F00922B5A171F
:10668000904A7F00B00B7F0091477F00B10B7F00E5
:10669000922B5A10375A0790487F00B00B7F009119
:1066A000407F00B10B7F0092305A08904A7F00B0C3
:1066B0000B7F0091427F00B10B7F00923C5A089003
:1066C0004C7F00B00B7F0091437F00B10B7F0092A5
:1066D000305A08904A7F00B00B7F0091427F00B192
:1066E0000B7F0092325A0F265A08265A08265A075C
:1066F000265A08265A19904A01009142010792260B
:106700000183E81CFF0601538406FF06014500FFD4
:106710002F004E4557004C4F4144004C4556454CC8
:10672000004C4F434B4544004241434B00524554BB
:10673000525900464F52464549540051554954005C
:106740004C5600505700555A45424F580057454245
:106750004552002828282828280028281E1E281EE0
:106760001E2841000028281E1E001E1E2828280062
:106770002828281E00001E1E2828002828281EFF62
:1067800000000028280028281E4200000000000009
:106790006700280000001E1E00000000000000002E
:1067A0001E1E1E1E0000001E1E00001E1E1E1E00BD
:1067B00000001E1E1E00281E1E28120000001E1EA5
:1067C0000028282828282800000000000C000000CD
:1067D00000FFFFFF0000004A0028282800000000FA
:1067E00042000000282828004100000000000000AE
:1067F0001E1E0000004545454506454545450645E4
:10680000454545450645454545064512001E1E00C1
:1068100000000000004500001E1E0000001E1E00BB
:1068200045000000000028281E1E00454C00000006
:10683000002828410000450000000000002400005E
:10684000004541000000FF00454545454512000058
:106850000000FFFFFF00000000000000000000003B
:1068600000001E1E1E1E004545450000451E1E1E42
:106870001E4145454500004545454545454545457D
:10688000000045121E0067001E00000000080028DE
:106890000028001E0000000045002842284100009A
:1068A00000000045002800281E45454500764500AB
:1068B0001E0000FF45454500004506454545454548
:1068C000454541000000000000004100001E0A0094
:1068D000000000FFFFFF0000007700000000000044
:1068E0000000282828282828240000000000240070
:1068F00000000000002800000000000000282828F8
:1069000028004145454545002841002400064545ED
:10691000451200284177240042454545450028415D
:1069200000240000000000000028282828000000A3
:10693000240000000000002800002828282828281B
:10694000240000000000007700FF00000000000AA3
:1069500000000000FFFFFF28282828000000240076
:106960000028284100240000002841282828280069
:10697000280000002828282800000000000000004F
:10698000282828000000000000000000000000008F
:1069900000B4001200B4000000000000000000007D
:1069A000000000002824280000000000000000284B
:1069B00000282800000028282428000000240000C7
:1069C00000284100282841282800FF002828002806
:1069D0000A00000000FFFFFF2800000041124100F4
:1069E000000028000000000000000000000000007F
:1069F0001E00000000001E00004100000000B30067
:106A00000000004141002800000000002800410073
:106A100000240000000000240000001E1E000000F2
:106A200000001E1E00001E1E00000000001E1E00B2
:106A30000000280000000000280000000028242892
:106A40002828242800001E00000000FF000000008D
:106A50001E1000000000FFFFFF28282828282828F3
:106A600028002828282800411E121E410028281E20
:106A70000000000000000000001E000000000000F8
:106A8000000000000000005F00004100005F000007
:106A9000000000240000002400000000001E00246C
:106AA0000024001E00004100000000000000000063
:106AB000411E0041000000000041001E2828000087
:106AC000000000000028280000002800FF002828FF
:106AD00028281000000000FFFFFF454545454545BB
:106AE000454545064500000000000000000000008C
:106AF000004128000000000028410000280000009C
:106B00000000000028000028410000B100004128DA
:106B1000000028280000000000282800004128006C
:106B20001E001E0028410000000000282828000048
:106B3000000000001E00241224001E0000000000BF
:106B400000000000000000000000000000FF000046
:106B50000000001200000000FFFFFF00B400000072
:106B600000000000001E002800002800412800004E
:106B700000001E00282828282800000000410000EE
:106B800028422828410041001E00002828281E1EF7
:106B9000001E000000001228411E00000000001E20
:106BA00000000067281E001EFF000000000000001B
:106BB000000041000000000000000000002800006C
:106BC0000000000000000000000000001E411E2820
:106BD00041281E000A0002000007FFFF2828281E87
:106BE000B31E28280000007700421E771E410000D7
:106BF000000028000000000000001E00001200003D
:106C000000000000000000FF2800000067000000F6
:106C100000000077000000000000000000001A1AC9
:106C20001A1A1A282828280A281A1A1A1A1A28009A
:106C30000024001E0000001A1A28000024001E0074
:106C4000B3001A1A2841002400414100001A1A28F2
:106C50000000241E1E100001000003FFFF7741000A
:106C600000004545450000120000002400450000DA
:106C7000000000000000454545000000001E4100E6
:106C800000450000000000005F7700004541004122
:106C90000000001E00001E45001E00000000000055
:106CA0000000454100410000001E00002445000096
:106CB000000000005F000000454542280067001EFC
:106CC00028002400450000000000002800000045C6
:106CD00000FF00000041100003000005FFFF00005E
:106CE000410008410024000000004545454545009D
:106CF00000002800414545451E4500000028B3001E
:106D00004545450045000000001E7745004100450F
:106D100000001E00001E45006700450000006700DF
:106D200012454545454500001E001E000000284252
:106D30002800000000280000000000007700002468
:106D40002800000000000000000000000000FF001C
:106D5000000000000000281000000000FFFFFF12EC
:106D600000007600000000000000001E0000001E71
:106D700028282824000000412800280000410000A5
:106D800076002828001E4128282800000000000066
:106D9000002828000000001E281E001E28410000B8
:106DA000000028004128282828282800002800283A
:106DB0002841281E00410000284128000028001E0C
:106DC0001E0000240028000028411E1E00000000B4
:106DD00000000000000000FF0A00000000FFFFFFAD
:106DE0000000410000004128280000002800282859
:106DF0002800280024000028002800280024FF285C
:106E0000000028002800280028002800002800286A
:106E10000028002800280000280028772877002470
:106E20000000002800284124002800280000280035
:106E300028002800280028000028242800280028EE
:106E4000122800000041000028002828000000004F
:106E50002400000041000000001200000000FFFFBD
:106E6000FF1C1C1C00410041001C1C1C1C1C1C1E87
:106E70001E4A1E1E1C1C1C002800000000000000F2
:106E8000280000000000004100000000001E00007B
:106E90001E0049001E00001E410024004B124C0041
:106EA0004100411E00001E0000001E00001E0000E8
:106EB000001E0000001E0000001E00004100000037
:106EC0004100001E1E2800000000000000001E00FF
:106ED0000028490000004928FF001000000000FFC2
:106EE000FFFF00000000B100280000000000411E6C
:106EF0000000002800004100000041242400280078
:106F0000411E0000000000000000002400002828AE
:106F10002800000000002400B20000000000120061
:106F200000000000B2002400000000002828280013
:106F300000240000000000000000001E41002800A6
:106F4000242441000000410000280000001E4100F0
:106F5000000000FF2800B100000000100000000049
:106F6000FFFFFF00000000000000000000000067BD
:106F7000494949474848486700004946454547450B
:106F80004546480000451A1A1A471A1A1A45001CA5
:106F9000451A1A4147411A1A451C1C451A1A1A4724
:106FA0001A1A1A451C1C4545454547454545451C8B
:106FB0001C4145454547454545411C00001E1E1ED8
:106FC000411E1E1E000000001E1E1E671E1E1E000B
:106FD0000012000000004200000000FF0A00000054
:106FE00000FFFFFF412800280028002800284A0051
:106FF00028002800280000002800002800000028A1
:107000000028002400002800280028002800240070
:10701000002877280028000000240000280028000D
:107020002400280A280000240028002800284A28D4
:107030000000280000002800280024000028002864
:1070400000280028000000000000280000002800A0
:10705000280000280028FF00492812285F080000A7
:107060000000FFFFFF0000B1000000000000000072
:107070004100001E00001E0000000077000000001C
:1070800000000000004145454545454545451E0A6F
:107090001E45001E1E1E1E454500001E4500000028
:1070A0000077454545064545000000004A1E454518
:1070B0000645450000000000240000001E450000B9
:1070C000002800000000000045001E2812280000D3
:1070D0001E1E0045424C000000FF001E1E410A001B
:1070E00003000003FFFF42001E45244524451E0007
:1070F0004200001E455F45B1451E000000001E0015
:10710000004100001E000024241E1E0606061E1E4E
:1071100024240000284C0000004B28000000002818
:107120004C0000004B2800000000284C0000004BE1
:1071300028000000672828000000282867000000B9
:107140006700000000006700000000000000000071
:107150000000000012000000000000000000FF0816
:1071600000000000FFFFFF00454545454545450639
:1071700045000024454545451E0800240000240024
:107180004545454545002400002441244545452406
:1071900000244A0024002400004124002400FF248D
:1071A0000024412400244124120024002400004132
:1071B000240024000024412445454524002449009E
:1071C00024004545454545002400002445454545E6
:1071D000454545240000454545454545454545004F
:1071E0001000000000FFFFFF2828000000001E0024
:1071F000410028284100000000004100000000007C
:107200001E00002800005F0012000000001E001E8B
:107210000000001EFF006700000000281E0B280071
:10722000000000006700000000410000000000288E
:10723000000028000024282428004100000000004D
:10724000004100240028242828000041004128286B
:1072500028000C24000000000000000000002800AE
:1072600000080001000004FFFF0000000000FF1EF6
:107270004A005F00672842280B2828000000000011
:1072800042280000002800000000672842001E6716
:1072900028422400410042281E2800282828001ED9
:1072A00067284100006700121E007700421E1E1E64
:1072B0000028001E001E671E4200280028001E0035
:1072C0007700421E0028001E0028241E67240000AC
:1072D00000001E002800770042280000002800005F
:1072E000001E0600000000FFFFFF120000004545E1
:1072F000454545004B00FF00004541244145000045
:107300000000000008244124454506454545064542
:107310004124424545064545450645454506454502
:107320000645454506454545064545066767450604
:1073300045454500000800426708000808080000AD
:107340004545676745064545454506454545454527
:1073500006454545457777774542244100000000C2
:1073600077416704000303000302FF4100000D00A2
:107370000C410028001228002800280028002400C2
:10738000410000280B000D000024002800412800C7
:1073900028005F000D00000028280A0000000028D7
:1073A00028280D00000C28FF00000D00000D000033
:1073B0000C2828280A280B24242828000000000D67
:1073C00024000C0B00282824282824280A0B000C51
:1073D00024000A002841280D000A0041002800006E
:1073E0000A0000280600000000FFFFFF00284141BE
:1073F00041284141412800002800000028000000E9
:107400002800002824242424242424280000000008
:1074100000004100000000001E001E0000120000DD
:107420001E001E5F0000000000000000005F00243E
:107430000041005F00410024000000000000000047
:10744000000000001E0000000041000000001E00BF
:1074500000002400240024000000001E5F2800FF1C
:1074600000285F1E000E00000000FFFFFF28FF0045
:10747000001E1E1E1E00411E2800000000002400E9
:10748000004141280000002828282800001E28006C
:107490000000284100120000002800000000000049
:1074A000000000001E1E1E24241E000000670000B5
:1074B000001E00001E000000000000000000001E72
:1074C000000000675F2424241E001E000000002826
:1074D0000000001E001E00000000004141411E008F
:1074E000005F5F0000410600000000FFFFFF00009A
:1074F0000028284100000000000028001228410058
:10750000000076000000000000282828000000008D
:107510005F004100000028282428001A1A1A0000E1
:107520000028410041001A1A1A00240000280028EF
:1075300000000000002800001E001E1A1E0000416E
:107540001E005F0000001A1AFF0000281E2800001D
:1075500000454500000000000000000045454500D2
:107560000000000000001E1000000000FFFFFF28C8
:1075700028282828282800282828772828281E0096
:10758000000000FF2800004228000067001E1E289F
:107590000045002800454500281E28004500280019
:1075A00045410000002800450000004545454524B0
:1075B0002800454545454500244500000024004578
:1075C00045455F0045000000000000454545454534
:1075D00045451E284100454545454512241E1E28A7
:1075E00000000000410000000E0003000003FFFF48
:1075F000454545454545454545454545454545453B
:107600004545454545454545410045005F001E450A
:107610004545454100450000002445454545454553
:107620004500000000454545450000000000001EE3
:107630004545454500002400454545454545452807
:10764000000000454545454545451E280067454520
:1076500012FF454545454545454545416745454535
:107660004545454545450045450600000000FFFFEE
:10767000FF00001E001E001E001E0000001E00284D
:1076800000000028001E001E002800244A240028B4
:10769000001E00280024410041240028001E002470
:1076A000412441244124000000414C00411241008A
:1076B0004B42FF1E002441244124412400000028A5
:1076C0000024410041240028001E002800244924F1
:1076D0000028001E001E002800000028001E0000D8
:1076E000001E001E001E001E00000A00000000FF19
:1076F000FFFF280000B12812280000B12800000078
:107700000000B4000000000000005F000024000042
:107710005F00000024002400240024002400000056
:1077200000002800280000000000002400005F0086
:107730000024000000284C00000000004B28B2008C
:107740000000000000000000000000000000002415
:1077500000000000000000000024002400000000E1
:10776000B228000041FF41000028000E0000000088
:10777000FFFFFF000000004C124B000000005F0004
:1077800000001E411E0000005F000000004C004B86
:1077900000000000000077001E001E007700001AA5
:1077A0000000001E001E0000001A1A1A00001E0031
:1077B0001E00001A1A1A1A41001E001E00411A1A51
:1077C0001A1A00001E001E00001A1A1A0000001EDD
:1077D000001E0000001A000077001E001E00770047
:1077E000000000000000FF00000000000400000096
:1077F00000FFFFFF1200000D00000000000000006D
:107800000000280B2828286728280B280B77410020
:107810000D4100000D000D410C0D0000280A28410B
:10782000002800280A28282800280A0B0D0B280BFE
:1078300028000C0C28000A0D0A28000041284128C5
:1078400041412800280A282828000D0B000C000CB4
:10785000410D0000002800FF2828282828280A2891
:10786000280000000000000000000000000A0001E5
:1078700001000301FF1E0000000000000000001EC8
:1078800000004128282828284100000024282877C3
:1078900028772828240000001E77410041771E0029
:1078A0000000000C1A0000001A0D00001E000C1A47
:1078B0000012001A0D001E00000C1A0000001A0D24
:1078C000000000001E77410041771E0000002428C0
:1078D00028772877282824000000412828282828ED
:1078E0004100001E00000000FF000000001E060016
:1078F0000101000304FF000028412441000000288A
:10790000415F00280000000000002800000028005F
:10791000412800002800001E28281E2828280028AA
:10792000000000411E1E1E28280028242400001EDE
:107930001E0024000028000000001E1E00000000A1
:107940002800000000244A001A1A002824240000FD
:107950000000001A1A00280000001E0000000000AD
:1079600000000000121E28280000FF000000000692
:107970000002000005FFFF41000000240024000079
:1079800000416700000024122400000067004C0042
:107990000024002400FF4B00000000282400241EC7
:1079A000000000000000001E0028000000005F0032
:1079B00000000000000000005F281E1E282800288C
:1079C000281E1E28410000002841280000004128F0
:1079D0001E1E00244124001E1E280000000000413D
:1079E00000000000005F0000000041000000005F98
:1079F0000400000000FFFFFF1E1E004112000000F7
:107A0000001E1E1E0000000000000000001E1E00E0
:107A10000000240000280000001E411E000000009D
:107A20005F280000000028000000000000000000A7
:107A3000001E0000005F00000000000028000000A1
:107A400028000000000000285F000024240000003F
:107A50001E00001E00002400001E241E1E00000048
:107A60000000001E41001E1E1E0000FF000024003A
:107A7000000600000000FFFFFF00000000002800DB
:107A80000000000000242424000C0000282800002E
:107A900000240000280000772800000000000041BA
:107AA0000C000000000000000B00000000000000BF
:107AB000280B2841005F0041280A28000000000030
:107AC00000000A000000000000000D41000000005E
:107AD000000028FF000028000012280000282800CD
:107AE000000D000028280000000000002800000011
:107AF00000000600000000FFFFFF0041000D0041F4
:107B0000000C0041000028282824242428282800CC
:107B1000002800240024002400280000000A280B6C
:107B2000280A280A00FF41000000000000000000B1
:107B30004100000000000000000000B20000000052
:107B40001E1E1E00000000000041001E121E00410B
:107B500000000000000000000000000000B21E0055
:107B60000000000000001E0028285F000041000007
:107B70005F28280600000000FFFFFF4545454545FA
:107B8000454506454545454100B3004545000012C1
:107B900045454506450645454506454545450000DC
:107BA00000454500004545454545064545450645D2
:107BB0004545450008004545450008004545064542
:107BC00045454545454506454500004500080045F5
:107BD00000004545450645064506450645454545DB
:107BE000FF00000800000045454545064545454560
:107BF000454545450E00000000FFFFFF4C0000001A
:107C00001E121E0000004B004C00001E001E000053
:107C10004B001E004C001E001E004B001E0000000A
:107C20000000000000000000002828282828002864
:107C3000282800410D410041004100410D4124240C
:107C4000242424242424242424004100410041002D
:107C50004100410024242424242424242424240016
:107C6000000000000000000000001E001E001EFFBB
:107C70001E001E001E1000000000FFFFFF1A1A2841
:107C80001C1C1C1C410D004C1A1A280B28282828E3
:107C90001A00281A1A0000000000000000001A1A3A
:107CA0000000000000000000001A1A280028002828
:107CB000412800001A1A2800280028122800FF0076
:107CC00000285F28002849280000000028282800F4
:107CD000282828000000000000000000000000002C
:107CE000412828282828282828282800000076004D
:107CF0007600760076001200000000FFFFFF4100D2
:107D000024001E1E451E4C120042002400000045A7
:107D1000000028004100240000000800002800287E
:107D2000282828281E4500002800280000001E1EC4
:107D3000451E00280028242800001E451E0028009B
:107D40000000282800004500000000000000002876
:107D50001E45FF00000028280028281E454524282D
:107D6000494C00006700422445001E1E28000028E0
:107D700028281E45454545060003000003FFFF1E59
:107D80001E1E00120000002828281E1E00000000F1
:107D90005F00001E1E1E1E005F000000001E001E71
:107DA0001E0000280024000000004B4C001E0000B4
:107DB00000005F001E1E00285F0024240028000031
:107DC0001E1E00000041000000001E1E1E0000419B
:107DD0000000000000004B00000024000000005FD5
:107DE000001E005F28000000244128001E00000043
:107DF0000000FF000000001E0A00000000FFFFFF5F
:107E00000000FF1A1A1A1A777700410000001A1AA8
:107E10001A1A0000006728240024282828000000DF
:107E20000028002400281228000000001E2400243E
:107E3000281C28777700001E000000281C2828280E
:107E4000000028410041281C1C1C1C0000281E1E8C
:107E50001E2828282828000000B10000000000008B
:107E6000000067000000000000000000000041006A
:107E7000004B001E1E1E0000000A00000000FFFF55
:107E8000FF1E1A1A1A1A1A004B001A004124000089
:107E90000000001E000000280000000000004B0051
:107EA0001E0000004C1E0B000000001E004C0000D5
:107EB00000001E1E1A1A1E121E1E1E00001E1E1E6E
:107EC0001E1E1E410000670000001E0000767600A6
:107ED000001E000000670000411E1E1E1E00000064
:107EE0001E1E1E1E410000670000001E0000767668
:107EF00000001E00FF00670000410A00000000FFB4
:107F0000FFFF414B000000120000004C4100002820
:107F10002800B200282800000000000028002800E7
:107F200000000045454545280028454545450000D9
:107F300000240028002400000000000000000000D1
:107F40000000000000000067000000670000000063
:107F50000041282841282841000000000028000096
:107F60000028000000000000280000002800000099
:107F700041005F2800FF00285F0041080002000068
:107F800007FFFF5F281A00770077001A0CB2001E67
:107F90001E1E2800281E1E1E000000001E2812287B
:107FA0001E0000004200001E1E0B1E1E00004200AC
:107FB0000000000000000000000042000000006718
:107FC0000000000028000000000000000000000089
:107FD0000000000000000000000000280024000055
:107FE000000000240000000000000000000000006D
:107FF000005F00410000FF000041005F0A00020036
:1080000000FFFFFF00000000FF28282800000000FC
:10801000454500000000000B4100004C45450606A8
:1080200045004B0000004C4545000045454B000015
:10803000004C4545000045454B0000004C454500BF
:108040000045454B0028004C4545000000454B00CD
:1080500000004C4545000000454B0028004C450001
:10806000000045454B0000004C001E0000451E4B23
:108070000000004C00000012000000005F02000041
:108080000000FFFFFF13140103030C0104040C01A3
:108090000C0203030F02050C02040402020E030289
:1080A00002030311010F020E04010103050F030275
:1080B0000203030F010F02100312010A040C010A4C
:1080C000030C010C020A040F02050C020303020256
:1080D0001204020204040F010D021203010104053F
:1080E0000B04020204040F01040412011602FF141F
:1080F000012C380437210708090A3B0C3C0E2E27B7
:10810000111213001539173F191A1B1C1D1E1F20B1
:1081100006222324253D1028292A2B022D0F2F303B
:1081200031323A343536050316330B0D263E18002E
:1081300011241FBECFEFD0E1DEBFCDBF14BE88E15A
:108140000FB6F89480936000109260000FBE11E0AB
:10815000A0E0B1E0E2E4FBEF02C005900D92A63092
:10816000B107D9F710E1A0E2B1E001C01D92A2373A
:10817000B107E1F70E946648882311F40E947C4809
:10818000F894E4E4FCE080E090E020E802C0219371
:10819000019632E08C309307D4F384E49CE0909312
:1081A000510E8093500E1092520EE5E5FEE080E0F5
:1081B00090E003C0108201963A9684309105D4F382
:1081C0009093890E8093880E91E09093750E909312
:1081D000760E9093740E1092810015BC8FEF87B9C4
:1081E00084B988E98AB95C9A8CE081B98BEF82B94D
:1081F0001092180C86E08093190C10928500109252
:10820000840083E0809389008DE88093880089E072
:108210008093810082E080936F0082E484BD17BC6C
:1082200095BD83E88093B0001092B3009093B100A5
:1082300081E185B910922D0C10921C0C10921D0C2E
:108240001092280C1092270C10922C0C10922B0CD0
:108250001092400C0E944B4880E00E942C4880FF06
:1082600003C084E00E9429480E944C4D78940E94EB
:108270004B4D0E94ED7C0C949F7D0C940000E4EA31
:10828000FBE0C0E2D1E02091F70E0027A081B18190
:10829000AC0FBD1F1C911283021708F4102F1C9302
:1082A000339603950C3190F30DE216E01A95F1F731
:1082B0000A95D9F7C0E2D1E000EDA02E662778E05C
:1082C00055D233E23A95F1F70E94A0413FE03A954A
:1082D000F1F700C0AA94A9F0000063950000000027
:1082E000683029F0C895C895C8950000E9CF662781
:1082F00000243EE1C30FD01D00000000000000007C
:10830000DFCFC895C895C895C895C89500000000EE
:108310002DD20E94344D11E000911B0C01270093D7
:108320001B0C20911C0C002309F0212720931C0C0E
:10833000E1E0E0931A0CE2E0E093360011240895A6
:10834000DE01679F00000091220C1091230C005069
:108350001740000D111D180104EA14E0000D111D55
:10836000280130E41EE12D912C316FB660FA239F75
:10837000A1010EF4A201040E151EF001F6F0059104
:1083800008B92D91059108B9239F059108B92C31A1
:108390006FB6059108B908F4A201059108B960FA11
:1083A000040E059108B9151E1A95059108B9059195
:1083B00039F1F00108B91EF700C0019108B92D91FB
:1083C0000191000008B9239F0191000008B92C31E8
:1083D0006FB660FA019108B90EF0A1010191040E87
:1083E00008B9151E00C0019108B9000000C0019134
:1083F00008B901911A9521F0F00108B906F6DDCF10
:1084000008B90027C895000008B905E00A95F1F7FA
:10841000089520E4E091220CF091230C8C51829F6E
:10842000E00DF11DA4EAB4E0629FA00DB11D00248F
:1084300005900D9205900D9205900D9205900D926C
:1084400005900D9205900D9205900D9205900D925C
:1084500005900D9205900D9205900D9205900D924C
:1084600005900D9205900D9205900D9205900D923C
:1084700005900D9205900D9205900D9205900D922C
:1084800005900D9205900D9205900D9205900D921C
:1084900005900D9205900D9205900D9205900D920C
:1084A00005900D9205900D9205900D9205900D92FC
:1084B00005900D9205900D9205900D9205900D92EC
:1084C00005900D9205900D9205900D9205900D92DC
:1084D00005900D9205900D9205900D9205900D92CC
:1084E00005900D9205900D9205900D9205900D92BC
:1084F00005900D9205900D9205900D9205900D92AC
:1085000005900D9205900D9205900D9205900D929B
:1085100005900D9205900D9205900D9205900D928B
:1085200005900D9205900D9205900D9205900D927B
:10853000112408950F931F9395E0899FECE2F4E0D6
:10854000E00DF11D048182819381E0E48E9FD001D2
:108550009E9FB00DE091F80BF091F90BEA0FFB1F15
:10856000A4EAB4E090E4699FA00DB11D112440304D
:1085700051F4A20FB11D822F122F00FF11C03796A8
:1085800010E1121B0DC088E0821B00FD04C0182FF3
:10859000E80FF11D05C018E0120FE20FF11D319731
:1085A000503031F498E0939FA00DB11D932F06C079
:1085B00098E0931B58E0599FE00DF11D11243EEF08
:1085C000E89400FD689458E0591B48E0481B3EF0D1
:1085D000259123132C9311964A95D1F707C0249126
:1085E000319723132C9311964A95C9F7E10FF11D8A
:1085F000A80FB11D5A9549F711241F910F910895A5
:10860000C443CE43DC43044328980E949A45E7E1E3
:10861000EA95F1F7289A0FD1E0E0F6E0F2D0E0FF1A
:1086200032D0E0FF2FC02F933F934F935F936F9310
:108630007F938F939F93AF93BF9378941124E0918E
:108640001E0CF0911F0CE115F10509F009950E942F
:10865000734E0E945E480E9465480E94C7441124E0
:10866000E091200CF091210CE115F10509F009953C
:10867000BF91AF919F918F917F916F915F914F913A
:108680003F912F910895EF93E091190CE13EE0F5B1
:10869000E131D0F12F923F924F925F926F927F9291
:1086A0008F929F92AF92BF92CF92DF92EF92FF9202
:1086B0000F931F932F933F934F935F936F937F93EA
:1086C0008F939F93AF93BF93CF93DF930E943F41CC
:1086D000DF91CF91BF91AF919F918F917F916F91DA
:1086E0005F914F913F912F911F910F91FF90EF90CC
:1086F000DF90CF90BF90AF909F908F907F906F90C2
:108700005F904F903F902F90EF910895FF93EF93DC
:10871000EFB7EF93E0918400EE50E13000F0E230EB
:1087200000F0E33000F0E43000F0E53000F0E63037
:1087300000F0E73000F0E83000F0E93000F005D05C
:10874000EF91EFBFEF91FF9118950F921F92E0E02C
:10875000F6E80090180C000C1124E00DF11D0590B6
:108760001490F00109951F900F90089528980E9489
:108770009A45E5E1EA95F1F7E091190CEA95E09365
:10878000190C289A00C0089528980E94C145289A7B
:108790000000E1E0F6E035D047D0089528980E9427
:1087A000C145E0EB0000EA95E9F700000000289AD7
:1087B000F6E0E2E026D0089528980E94C145289A64
:1087C0000000E3E0FDEF1DD0E091190CE53091F4DD
:1087D000E0911B0CE1300000F0912D0C19F4F091A8
:1087E0002D0CF195E3E0E0938900EDE8EF0FE093C5
:1087F00088000895E3E0E0938900EDE8E0938800C5
:1088000008950090190C0A9410905F0011FC0F2E2F
:108810000092190C0090180C11FC0E2E0092180CEE
:10882000E0E011FCE1E00895E3E0E0938900EDE889
:10883000E09388000895E7E0E0938900EBE1E0939E
:108840008800089500000000000000000000000003
:108850000000000000000000000000000000000018
:108860000000000000000000000000000000000008
:1088700000000000000000000000000000000000F8
:1088800000000000000000000000000000000000E8
:1088900000000000000000000000000000000000D8
:1088A00000000000000000000000000000000000C8
:1088B00000000000000000000000000000000000B8
:1088C00000000000000000000000000000000000A8
:1088D0000000000000000000000000000000000098
:1088E0000000000000000000000000000000000088
:1088F0000000000000000000000000000000000078
:1089000099277727833008F00895E0E0FFE8660FA5
:10891000771FE60FF71FA591B491E5E5FEE02AE089
:10892000289FE00DF11DA183B28311240895909139
:10893000740E9170880F892B8093740E0895992777
:108940007727E5E5FEE02AE0289FE00DF11D6E3F68
:1089500031F46091740E6E7F6093740E0BC06F3FA4
:1089600031F46091740E6E6F6093740E03C07CE8F6
:10897000760F75831124089599277727E5E5FEE0A2
:108980002AE0289FE00DF11D6083112408950E94C4
:108990002B4A0090520E002019F4A4E4BCE002C05F
:1089A000AAE4BDE021E002260092520E22E02093CC
:1089B000530E2F923F924F925F926F927F928F92BF
:1089C0009F92AF92BF92CF92DF92EF92FF920F935E
:1089D0001F93CF93DF935091730E6091750E70913A
:1089E000760E8091770E2090560E3090570E409064
:1089F000590E50905A0E6090580E1091550E70906E
:108A0000600E8090610E9090620EA090630EB09008
:108A1000640E20915F0EC0906A0ED0906B0EE090B5
:108A20006D0EF0906E0E00916C0E3091690E9FEFFE
:108A3000620C431CF2014491410300240008C12D43
:108A4000D02D970CA81CF501449142030024000886
:108A5000C10DD01D0C0DED1CF70144914303002402
:108A60000008C10DD01D8A956AF44091740E842FC0
:108A70008695062E0694062600FA7695679576F971
:108A800040FF66F940E860FD4FE745030024000819
:108A9000C10DD01D0024C038D0050CF0CFE70A94DA
:108AA000C038D0050CF4C0E8C058CD939A9509F0B1
:108AB000BFCF4091530E4A954093530E97E009F073
:108AC000B7CF6092580E4092590E9092620EA092CB
:108AD000630E00936C0EE0926D0E6093750E7093B2
:108AE000760E8093770EDF91CF911F910F91FF90BB
:108AF000EF90DF90CF90BF90AF909F908F907F903E
:108B00006F905F904F903F902F900895E091500E9E
:108B1000F091510E019100000093B3000EE0E0359A
:108B2000F00704E41CE008F0F801E093500EF09325
:108B3000510E08950C949C450C949E450F931F93E1
:108B40002F93E091500EF091510E01910093B300DC
:108B50000EE0E035F00710F40000000010F0E4E44F
:108B6000FCE0E093500EF093510EC895C895C8955F
:108B7000C895C895C895000000002F911F910F91CE
:108B800008950000E091190CE0FFD8CFE1E1EA95EB
:108B9000F1F7000000000895000000000000000050
:108BA00000000000000000000000000000000000C5
:108BB00000000000000000000000000000000000B5
:108BC00000000000000000000000000000000000A5
:108BD0000000000000000000000000000000000095
:108BE0000000000000000000000000000000000085
:108BF0000000000000000000000000000000000075
:108C0000808182838485868788898A8B8C8D8E8FEC
:108C1000909192939495969798999A9B9C9D9E9FDC
:108C2000A0A1A2A3A4A5A6A7A8A9AAABACADAEAFCC
:108C3000B0B1B2B3B4B5B6B7B8B9BABBBCBDBEBFBC
:108C4000C0C1C2C3C4C5C6C7C8C9CACBCCCDCECFAC
:108C5000D0D1D2D3D4D5D6D7D8D9DADBDCDDDEDF9C
:108C6000E0E1E2E3E4E5E6E7E8E9EAEBECEDEEEF8C
:108C7000F0F1F2F3F4F5F6F7F8F9FAFBFCFDFEFF7C
:108C8000000102030405060708090A0B0C0D0E0F6C
:108C9000101112131415161718191A1B1C1D1E1F5C
:108CA000202122232425262728292A2B2C2D2E2F4C
:108CB000303132333435363738393A3B3C3D3E3F3C
:108CC000404142434445464748494A4B4C4D4E4F2C
:108CD000505152535455565758595A5B5C5D5E5F1C
:108CE000606162636465666768696A6B6C6D6E6F0C
:108CF000707172737475767778797A7B7C7D7E7FFC
:108D000000020406080A0C0E10121416181A1C1E73
:108D100020222426282A2C2E30323436383A3C3E63
:108D200040424446484A4C4E50525456585A5C5E53
:108D300060626466686A6C6E70727476787A7C7E43
:108D40007F7D7B79777573716F6D6B696765636123
:108D50005F5D5B59575553514F4D4B494745434113
:108D60003F3D3B39373533312F2D2B292725232103
:108D70001F1D1B19171513110F0D0B0907050301F3
:108D8000FFFDFBF9F7F5F3F1EFEDEBE9E7E5E3E1E3
:108D9000DFDDDBD9D7D5D3D1CFCDCBC9C7C5C3C1D3
:108DA000BFBDBBB9B7B5B3B1AFADABA9A7A5A3A1C3
:108DB0009F9D9B99979593918F8D8B8987858381B3
:108DC00080828486888A8C8E90929496989A9C9EB3
:108DD000A0A2A4A6A8AAACAEB0B2B4B6B8BABCBEA3
:108DE000C0C2C4C6C8CACCCED0D2D4D6D8DADCDE93
:108DF000E0E2E4E6E8EAECEEF0F2F4F6F8FAFCFE83
:108E00007F7F7F7F7F7F7F7F7F7F7F7F7F7F7F7F72
:108E10007F7F7F7F7F7F7F7F7F7F7F7F7F7F7F7F62
:108E20007F7F7F7F7F7F7F7F7F7F7F7F7F7F7F7F52
:108E30007F7F7F7F7F7F7F7F7F7F7F7F7F7F7F7F42
:108E40007F7F7F7F7F7F7F7F7F7F7F7F7F7F7F7F32
:108E50007F7F7F7F7F7F7F7F7F7F7F7F7F7F7F7F22
:108E60007F7F7F7F7F7F7F7F7F7F7F7F7F7F7F7F12
:108E70007F7F7F7F7F7F7F7F7F7F7F7F7F7F7F7F02
:108E800080808080808080808080808080808080E2
:108E900080808080808080808080808080808080D2
:108EA00080808080808080808080808080808080C2
:108EB00080808080808080808080808080808080B2
:108EC00080808080808080808080808080808080A2
:108ED0008080808080808080808080808080808092
:108EE0008080808080808080808080808080808082
:108EF0008080808080808080808080808080808072
:108F000022002400260028002B002D003000330012
:108F1000360039003D004000440048004C0051003C
:108F200056005B00600066006C00730079008100F1
:108F3000880090009900A200AC00B600C100CC00EF
:108F4000D800E500F30001011001210132014401C4
:108F500057016C0181019801B001CA01E5010202CB
:108F60002102410264028802AE02D70203033003E9
:108F700061039403CB03050442048304C704100572
:108F80005D05AF0505066106C206290796070908B3
:108F9000830805098E09200ABA0A5D0B0A0CC10C68
:108FA000840D510E2B0F121007110A121D134014BD
:108FB0007415BA1614188319071BA31C571E2420F6
:108FC0000E22142439267F28E82A752D29300633ED
:108FD0000F364539AD3C49401B442848734CFE5080
:108FE000CF55EA5A51600C661D6C8B725A7992808B
:108FF00037885090E598FDA19FABD3B5A3C0000082
:109000008093F80B9093F90B0895ECE0F3E0A0E265
:10901000B1E06CE16D933197E9F711240895992738
:1090200077272EE1629F080E191EA0E2B1E0A00D85
:10903000B11D445E4C93112408958093220C9093AB
:10904000230C089580911A0C0895112410921A0C83
:10905000089580932D0C0895882329F48091250C80
:109060009091260C08958091290C90912A0C0895D6
:10907000F999FECF92BD81BD60BDF894FA9AF99A34
:1090800078940895F999FECF92BD81BDF894F89A2D
:1090900080B578940895129A129880E090E020E0CC
:1090A000969587951398009B9068139A2F5F2031AF
:1090B000B9F79093260C8093250C089580910001B8
:1090C000882311F00E944B48089508951F9380E073
:1090D00090E00E944248182F81E090E00E944248B0
:1090E00090E0382F20E0210F311D2A55354509F435
:1090F00091E0892F1F910895CF93DF93C0E0D0E0D6
:10910000FE01E059FF4FE491CE016E2F0E943848D6
:109110002196C531D105A1F7C0E4D0E0CE016FEFB3
:109120000E943848CE0101966FEF0E943848A09601
:1091300088E0C030D80791F7DF91CF91089590E093
:1091400026E130E0829FF001839FF00D929FF00DA9
:109150001124E457F14F628708956093740E0895C7
:1091600090E026E130E0829FF001839FF00D929F16
:10917000F00D1124E457F14F13861182089590E009
:1091800026E130E0829FF001839FF00D929FF00D69
:109190001124E457F14F81E0838B089590E026E19C
:1091A00030E0829FF001839FF00D929FF00D11241B
:1091B000E457F14F6187089590E026E130E0829F07
:1091C000F001839FF00D929FF00D1124E457F14FB1
:1091D0006483089590E026E130E0829FF001839F50
:1091E000F00D929FF00D1124E457F14F658308951F
:1091F0009093E70E8093E60E8FE68093EC0E10922C
:10920000430CECE8FEE021E08FEF98E1208310862C
:109210008683878314861182958376963EE0E43EAA
:10922000F307A1F7089510928D0E1092A30E1092DD
:10923000B90E1092CF0E01969093F00E8093EF0E20
:1092400090938B0E80938A0E9093F30E8093F20E80
:109250001092EE0E1092ED0E1092E50E1092E40EAA
:109260001092E80E81E08093430C1092EB0E109266
:10927000EA0E08958091960E87FD03C08AEF8093D1
:10928000960E8091AC0E87FD03C08AEF8093AC0EE2
:109290008091C20E87FD03C08AEF8093C20E809139
:1092A000D80E87FD03C08AEF8093D80E1092430C2E
:1092B0000895DC01ED91FC911197AF014F5F5F4F75
:1092C00011965C934E93E4912E2F30E0E7FF13C08C
:1092D0002F7730703695322F222737952795FA0150
:1092E0004F5F5F4FE4918E2F8F77280F311DE7FD81
:1092F000F1CF4D935C93C90108950E949F44089556
:10930000EF92FF920F931F93CF93DF93182F062FA7
:10931000F42EE22EC82FD0E086E190E0C89FF00145
:10932000C99FF00DD89FF00D1124E457F14F8385AC
:10933000882321F08181882309F088C0EE2091F4F0
:1093400086E190E0C89FF001C99FF00DD89FF00D15
:109350001124E457F14F138A8285882309F076C0DF
:10936000108674C0133059F481E091E09093760E2A
:109370008093750E81E08093740E0F2D08C0812FAD
:1093800060E00E949F44812F6F2D0E9480440F3720
:1093900099F486E190E0C89FF001C99FF00DD89F35
:1093A000F00D1124E457F14F8091E90E87878AEE82
:1093B0009EE0958B848B30C089E0089FC00111240A
:1093C000E091E60EF091E70EE80FF91F3396459114
:1093D00054914115510571F486E190E0C89FF00168
:1093E000C99FF00DD89FF00D1124E457F14F158A55
:1093F000148A12C0FA01249186E190E0C89FF0011E
:10940000C99FF00DD89FF00D1124E457F14F278725
:109410004F5F5F4F558B448B86E190E0C89FF00112
:10942000C99FF00DD89FF00D1124E457F14F108A19
:109430001286048711829FEF9187E086F282118A5B
:1094400081E08387138A128A14829683CDB7DEB7B0
:10945000E6E00C94907DCF92DF92FF920F931F93E2
:10946000CF93DF93E5E9FEE08181282F332727FDA5
:1094700030958081280F311D2F3F310519F014F0F0
:109480002FEF30E0C90137FF02C080E090E0808319
:1094900076964EE0ED3EF40739F78091430C882331
:1094A00009F028C144C1E091EF0EF091F00E9F0148
:1094B0002F5F3F4F3093F00E2093EF0E44914F3FBC
:1094C00069F5A9014F5F5F4F5093F00E4093EF0E87
:1094D000F90184918F3219F41092430C19C186302E
:1094E00009F0FBC0FA013196CF0101969093F00E7E
:1094F0008093EF0EE491E33529F49093F30E80937B
:10950000F20EEBC0E53409F0E8C08091F20E9091C4
:10951000F30E9093F00E8093EF0EDFC047FF02C072
:109520004093E80E542F5F70842F90E0807F9070FE
:10953000803B910531F1803C910581F180399105A5
:1095400009F043C0C9010196F90144910196909335
:10955000F00E8093EF0E0197FC012491852F90E08F
:109560008C9FF0018D9FF00D9C9FF00D1124E4570E
:10957000F14F8081882309F4B0C0220F852F6485C4
:1095800053C0C9010196F901449101969093F00EE0
:109590008093EF0E0197FC01249153C02F5F3F4F42
:1095A0003093F00E2093EF0E21503040F9012491BA
:1095B000852F90E08C9FF0018D9FF00D9C9FF00D0A
:1095C0001124E457F14F248788C08091E80E582F6A
:1095D0005F7090E0807F9070803B910541F1803C0E
:1095E000910509F46EC08039910509F076C02F5FAE
:1095F0003F4F3093F00E2093EF0E21503040F90191
:109600002491852F90E08C9FD0018D9FB00D9C9F61
:10961000B00D1124A457B14F8C91882309F45DC07B
:10962000220F852F1C966C910E94804956C02F5F97
:109630003F4F3093F00E2093EF0E21503040F90150
:109640002491473071F4852F90E08C9FF0018D9F1D
:10965000F00D9C9FF00D1124E457F14F220F27834A
:109660003CC04B3071F4852F90E08C9FF0018D9FB2
:10967000F00D9C9FF00D1124E457F14F220F26832B
:109680002CC04C3571F4852F90E08C9FF0018D9F9C
:10969000F00D9C9FF00D1124E457F14F220F24830D
:1096A0001CC04436D1F4852F90E08C9FF0018D9F33
:1096B000F00D9C9FF00D1124E457F14F220F2583EC
:1096C0000CC0852F90E08C9FF0018D9FF00D9C9F2A
:1096D000F00D1124E457F14F44878FEE9EE00E9475
:1096E00059499093EE0E8093ED0E1092E50E109274
:1096F000E40E02C0C6E1D0E06091E40E7091E50E88
:109700008091ED0E9091EE0E6817790709F4CBCE9B
:109710006F5F7F4F7093E50E6093E40E8091EA0EC9
:109720009091EB0E01969093EB0E8093EA0E05E577
:109730001EE0CDE8DEE0FF24BFEFCB2ED12C8A89DE
:10974000882309F05EC08B899C89892B09F456C057
:109750009F858E85981708F04CC050C08B852B894B
:109760003C898F37E9F4D9018D91BC8BAB8B8F3F4E
:1097700001F1F90161811196BC8BAB8BE82FF0E010
:10978000EE0FFF1FEB57FF4F0190F081E02D8F2D63
:109790000995EB89FC8981918E87FC8BEB8B28C026
:1097A000A9014F5F5F4F5C8B4B8BF90184918F3F19
:1097B00021F418821C8A1B8A21C04F5F5F4F5C8B8B
:1097C0004B8B41505040FA01649190E0880F991FF3
:1097D0008B579F4FFC01259134918F2DF9010995ED
:1097E000EB89FC893196FC8BEB8B3197E491EE870A
:1097F0001F869F858E85981709F4B0CF8F858F5F60
:109800008F878A85882319F420E030E06BC088892F
:109810008F3F11F08F5F888B9F81992309F45CC083
:109820002885222309F458C08E81882309F454C066
:109830004091EC0E442309F44FC0899FC0011124CC
:1098400080509F4F892F992730E0B901869F900162
:10985000879F300D969F300D112420503F4F232FAE
:1098600033278D8190E0FC012E9FC0012F9F900D2A
:109870003E9F900D112480509F4F892F9927242FB0
:1098800030E0AC01429FC001439F900D529F900D6C
:10989000112480509F4F292F33278B818823F1F08B
:1098A000EA81F0E0E050F447E491E058E89FC0011D
:1098B000112480509F4F892F9927B601681B790B7F
:1098C000629FC001639F900D729F900D1124805084
:1098D0009F4F292F332702C020E030E08A819C81EE
:1098E000890F8A83F8012083F394065F1F4F6696E1
:1098F000F4E0FF1609F023CFDF91CF911F910F9174
:10990000FF90DF90CF9008951F93CF93DF93582F50
:1099100089E0589FC00111242091E60E3091E70E96
:10992000280F391FC9010396FC01A591B491F901D3
:1099300084918150823010F413E01DC08091A30EF9
:109940008823B1F08091AF0E851711F4442381F480
:109950008091B90E882371F08091C50E851711F49E
:10996000442341F49091B30E8091C90E891710F4ED
:1099700011E001C012E0212F30E0FD01449186E1A9
:1099800090E0289FE001299FD00D389FD00D112431
:10999000C457D14F4F871196BD8BAC8B188A80E589
:1099A0008A8368878FEF89871A861B8A198A21E044
:1099B0002B871A8A5D8729831C828E83133049F492
:1099C00081E091E09093760E8093750E2093740E53
:1099D00008C0812F60E50E948044812F6A890E941F
:1099E0009F44DF91CF911F910895FF920F931F9392
:1099F000082FF62E0E94804410E086E190E0089F38
:109A0000F001099FF00D189FF00D1124E457F14F5C
:109A1000F2821F910F91FF900895962F482F50E0EA
:109A200026E130E0429FF001439FF00D529FF00D80
:109A30001124E457F14F6281691B62830E948044C4
:109A40000895482F50E026E130E0429FF001439F07
:109A5000F00D529FF00D1124E457F14F9281690FE0
:109A600062830E94804408953091F70E20E010C078
:109A7000822F90E0FC01EE0FFF1FE80FF91FEC555D
:109A8000F44FA081B181A05EBE4F82818C932F5F85
:109A9000231770F3089508950895982F882319F4D3
:109AA0008FEF87B9089581E08093FA0E8093F50EC9
:109AB0009093F40E1092F90E8093F80E662321F025
:109AC0008091F80E8823E1F70895982F882311F4E8
:109AD00017B808958CE08093FA0E8FEF8093F50EFF
:109AE0009093F40E1092F90E81E08093F80E6623A5
:109AF00021F08091F80E8823E1F708958091F60E09
:109B0000882341F0E091FA0EF0E0E656FF4FE49131
:109B1000E7B908958091F80E8823F9F08091F90E45
:109B20008823C1F48091F40E8093F90E8091FA0E8F
:109B3000E82FF0E0E656FF4FE491E7B99091F50E7B
:109B4000980F9093FA0E992311F09D3031F41092F2
:109B5000F80E089581508093F90E08951F93CF93C6
:109B6000DF93EC0110E007C00E9422488823E1F354
:109B70000E9425481F5F812F90E08C179D07A4F35A
:109B8000DF91CF911F910895A8E0B0E0EAECFDE4E9
:109B90000C94687D1092F70E7CE2872E74E0972E6D
:109BA000CC24DD24CD82DE82F4018081803F09F463
:109BB00074C09181F82FF695F695F695F983282FC4
:109BC000277019F082E08B8302C0E1E0EB83F92F6C
:109BD000F695F695F695FC83892F877019F092E03B
:109BE0009A8302C0E1E0EA83B82EAA241501220E6E
:109BF000311C00E010E046C08981FF818F0FA20177
:109C0000480F511D60E2E62E61E0F62EE40EF51ECF
:109C1000F70160816C31F0F02091F70E2C3120F5C6
:109C2000822F90E0FC01EE0FFF1FE80FF91FEC55AB
:109C3000F44F518340836283862F622F0E94094232
:109C40006091F70EF70160836F5F6093F70E6150CC
:109C50006C3150F44F815885460D571D8D819E8182
:109C600070E091010E949A428F81988501969887B1
:109C70008F839B81891708F4BFCF0F5F1F4FEA8145
:109C80000E1758F48C81800FFEE18F9F2001112464
:109C9000702E662418861F82AFCF0894C11CD11C79
:109CA00085E090E0880E991E98E1C916D10409F06C
:109CB00079CF3091F70E20E010C0822F90E0FC01A8
:109CC000EE0FFF1FE80FF91FEC55F44FA081B18193
:109CD000A05EBE4F82818C932F5F231770F328966E
:109CE000E2E10C94847D0E947E4D0E94C44D089553
:109CF000ECE2F4E080EF8083359694E0E43AF907F3
:109D0000D1F71092220F0895AF92CF92DF92EF9287
:109D1000FF920F931F93CF93DF93F22ED02EC22F7B
:109D2000D0E0B6E0CC0FDD1FBA95E1F79EE1699F68
:109D300080011124E42FF52FBF018F5F005E1E4FBD
:109D400003C06F5F7F4F8F5F582F5150FB0194917D
:109D5000992379F19032A9F39F779052E92FFF2749
:109D6000E7FDF095A6E0EE0FFF1FAA95E1F7E75992
:109D7000FE4D9E012F5F3F4FDE01AC55BB4F40E0D3
:109D800094919D1511F4EC9205C09C1511F4AC92C0
:109D900001C09C93E9014F5F31962F5F3F4F1196B1
:109DA000403471F7F801E50FF11DF082F3948E3124
:109DB00040F28F2DDF91CF911F910F91FF90EF9087
:109DC000DF90CF90AF900895AF92CF92EF920F9324
:109DD000CC24AA240E94844E0F91EF90CF90AF9094
:109DE0000895982F8756803110F481E00895892FC7
:109DF0008F558830D0F38A5E8631B8F380E097576C
:109E00009430A0F781E00895982F442309F451C0BD
:109E10004A3109F44EC04C3109F44BC0453409F0C5
:109E20004AC047C0483030F490FD02C046E041C00F
:109E300047E03FC060FD02C048E03BC049E039C098
:109E40004A3041F4992319F4662351F532C0662350
:109E500059F528C04B3051F4992321F4662331F190
:109E60004CE027C0662321F14DE023C04C3049F47B
:109E7000992321F46623E9F44AE01BC06623A1F488
:109E800017C04D3041F4992319F4662349F40EC0EC
:109E9000662379F407C0940F462F440F490F09C079
:109EA00040E107C04BE005C041E103C04EE001C006
:109EB0004FE0842F0895842F8650843008F4B2CF69
:109EC0008450883008F4BCCFE6CF1F93182F0E942F
:109ED000F14E882321F4812F815B823018F481E0D8
:109EE0001F910895133BD9F31637C9F3143BB9F307
:109EF000812F8452843098F38D51843080F380E038
:109F00001F3F71F7ECCF482F909168108091C20FDE
:109F1000981739F49091030F8091140F891708F462
:109F200066C05091140F20E030E0842F90E0DC01F7
:109F300011970196F901ED5BFF4EE0814E1739F064
:109F4000F0E0AE17BF0719F08E179F0749F4F9012B
:109F5000E55BF04FE081E61718F45E1708F447C0A0
:109F60002F5F3F4F2430310529F720E030E0842F68
:109F700090E0DC0111970196F901E45DF04FE0817A
:109F80004E1739F0F0E0AE17BF0719F08E179F0794
:109F900041F4F901EF59FF4EE081E61710F45E1726
:109FA00030F12F5F3F4F2430310531F7262F2250FB
:109FB0008EE1689FF0011124E40FF11DEC51FF4F79
:109FC00012C09081892F8C51843218F091569430B0
:109FD00070F49181892F8C51843218F0915694300D
:109FE00030F42250FC97521760F381E0089580E02E
:109FF0000895482F909168108091C20F981739F4F6
:10A000009091030F8091140F981708F466C0509137
:10A01000140F20E030E0842F90E0DC0111970196CE
:10A02000F901ED5BFF4EE0814E1739F0F0E0AE171D
:10A03000BF0719F08E179F0749F4F901E55BF04F50
:10A04000E0816E1718F4E51708F447C02F5F3F4F03
:10A050002430310529F720E030E0842F90E0DC0146
:10A0600011970196F901E45DF04FE0814E1739F048
:10A07000F0E0AE17BF0719F08E179F0741F4F90102
:10A08000EF59FF4EE0816E1710F4E51730F12F5FA6
:10A090003F4F2430310531F7262F2E5F8EE1689F28
:10A0A000F0011124E40FF11DE45AFE4F12C090811B
:10A0B000892F8C51843218F09156943070F491812C
:10A0C000892F8C51843218F09156943030F42E5FE1
:10A0D000FC96251760F381E0089580E008951F93B2
:10A0E000CF93DF93782F909168109F3F21F080915C
:10A0F000C20F891770F01091C20FABE4BFE0E3E428
:10A10000F0E1862F90E0EC012197AC014F5F5F4FAB
:10A1100007C09091030F8091140F981761F75CC0EE
:10A120002C91621751F0808190E0C817D90729F06F
:10A13000822F90E04817590731F48081871718F46F
:10A14000181708F449C0119631968FE0AF34B8075C
:10A1500039F720E030E0862F90E0AC0141505040CC
:10A160000196F901EF59FF4EE0816E1739F0F0E0EA
:10A170004E175F0719F08E179F0741F4F901E45D50
:10A18000F04FE081E71710F41E1730F12F5F3F4FBB
:10A190002430310531F7272F22508EE1689FF001DE
:10A1A0001124E70FF11DE25EFE4F12C09081892F4E
:10A1B0008C51843218F09156943070F4968D892F1A
:10A1C0008C51843218F09156943030F422503297EA
:10A1D000121760F381E001C080E0DF91CF911F9101
:10A1E00008951F93CF93DF93782F1091C20F809122
:10A1F0006810811738F49091030F8091140F98170D
:10A2000009F467C0ABE4BFE0E3E4F0E1862F90E03F
:10A21000EC012197AC014F5F5F4F2C91621751F019
:10A22000808190E0C817D90729F0822F90E0481765
:10A23000590731F48081781718F4811708F449C060
:10A24000119631968FE0AF34B80739F720E030E04F
:10A25000862F90E0AC01415050400196F901EF5932
:10A26000FF4EE0816E1739F0F0E04E175F0719F0EE
:10A270008E179F0741F4F901E45DF04FE0817E17EE
:10A2800010F4E11730F12F5F3F4F2430310531F7E3
:10A29000272F2E5F8EE1689FF0011124E70FF11D3B
:10A2A000EE5DFE4F12C09081892F8C51843218F0E0
:10A2B0009156943070F4968D892F8C51843218F019
:10A2C0009156943030F42E5F3296211760F381E07E
:10A2D00001C080E0DF91CF911F910895CF93DF936C
:10A2E000782FABE4BFE020E030E0C82FD0E0462F6D
:10A2F00050E0F901ED5BFF4E9081993C30F5F9019A
:10A30000E85DF04F808186FD20C0971761F48C9145
:10A31000861711F48CED20C090E001968417950704
:10A32000A1F48EED19C0892F90E001968C179D073E
:10A3300061F48C91861711F48DED0EC090E00196BA
:10A340008417950711F48FED07C02F5F3F4F1196CB
:10A350002430310571F680E0DF91CF91089583506C
:10A360006350669570E086952BE030E0629FF001C7
:10A37000639FF00D729FF00D1124E80FF11DE8535B
:10A38000F04FE0818091310F982F90FF06C0EB30A5
:10A3900021F48091140F80FD18C091FF06C0EA30AF
:10A3A00021F48091140F80FD10C092FF06C0ED30A3
:10A3B00021F48091C20F80FD08C093FF08C0EC30EB
:10A3C00031F48091C20F8170089581E0089580E09A
:10A3D0000895EF92FF920F931F93F82EE62E462FCB
:10A3E00050E0682F70E0CA01880F991FFA0115E04C
:10A3F000EE0FFF1F1A95E1F7E81BF90BE60FF71FA9
:10A40000E05EFE4F0081A1E6B0E120E030E0F9011E
:10A41000E754F04F8081882361F1F901E45DF04F4A
:10A42000E081FE1631F08E2F90E0019668177907D3
:10A4300061F48C91E81609F44EC090E0019648173B
:10A44000590709F448C0FE1631F08E2F90E00196AE
:10A450006817790741F48C91E816E9F190E00196CC
:10A4600048175907C1F12F5F3F4F1196253031052D
:10A4700071F6102F1C51802F8652883090F48F2D4A
:10A480006E2D0E94AF5117C0163020F0802F8653DA
:10A49000823098F410E0812F1F910F91FF90EF9080
:10A4A0000895802F80548430B0F38F2D6E2D0E943C
:10A4B0006E51882349F3182FEECF802F8D558430AD
:10A4C00048F3815D883030F3845F843018F308539B
:10A4D00010E0023000F311E0DECF0F931F93082F3E
:10A4E000162F20E030E0862F90E0BC0161507040D4
:10A4F000DC011196802F90E0AC0141505040019654
:10A50000F901ED5BFF4EE081EF3FB1F0E01739F06C
:10A51000F0E0E417F50719F0E817F90769F4F90115
:10A52000E55BF04FE081E11771F0F0E0E617F70727
:10A5300051F0EA17FB0739F02F5F3F4F2430310508
:10A54000F9F680E001C081E01F910F9108950F930B
:10A550001F93CF93DF93082F162F20E030E0862F34
:10A5600090E0EC012197BC016F5F7F4F802F90E05E
:10A57000DC011197AC014F5F5F4FF901E754F04FD9
:10A580008081882311F1F901ED5AF04FE081E4FD5B
:10A590001CC0E7FD1AC0F901E45DF04FE081E0174F
:10A5A00039F0F0E0EA17FB0719F0E417F50769F452
:10A5B000F901EF59FF4EE081E11771F0F0E0EC177F
:10A5C000FD0751F0E617F70739F02F5F3F4F2530B1
:10A5D000310599F680E001C081E0DF91CF911F91B4
:10A5E0000F910895FF920F931F93CF93DF93182F2E
:10A5F000062FF42EA62FB0E0C82FD0E0CD01880F93
:10A60000991FFD0135E0EE0FFF1F3A95E1F7E81BBA
:10A61000F90BEC0FFD1FE05EFE4F80818C51823103
:10A6200008F048C0622F70E04F2D50E0CB01880F3A
:10A63000991FFB0135E0EE0FFF1F3A95E1F7E81B8C
:10A64000F90BE40FF51FE05EFE4F80818C518231E3
:10A6500088F5809168108F3F11F13091AA0F131780
:10A6600031F0832F90E00196C817D90751F48091FB
:10A6700069100817F9F090E00196A817B90779F466
:10A6800019C0F31619F04817590749F48091691059
:10A69000281781F090E001966817790759F0812F0B
:10A6A000602F0E94A752882329F4812F602F0E94D7
:10A6B0006D5201C081E0CDB7DEB7E5E00C94917D2D
:10A6C000A0E0B0E0E6E6F3E50C946D7D082F10E025
:10A6D000F801E450F14F8081882309F08CC0BB243D
:10A6E000E801CD5AD04FFCE2CF2EFFE0DF2EC00EA6
:10A6F000D11EE1E6EE2EE0E1FE2EE00EF11E72E04C
:10A70000772E8824839464E0962E58E0A52E8881C5
:10A7100080FF06C0F6014081F7012081215007C06B
:10A7200081FF09C0F6014081F70120812E5F842F4F
:10A73000622F4F5F0EC082FF04C0F601408141507E
:10A7400003C0F60140814E5FF7012081842F622F04
:10A750002F5F0E94F252882309F44DC0988196FF22
:10A7600004C080E49827988378C090FF0FC0A88227
:10A77000F60140814E5FF7012081842F622F2F5F09
:10A780000E94F252882389F198822FC091FF0FC056
:10A790009882F60140814150F7012081842F622F79
:10A7A0002F5F0E94F252882301F1A8821EC092FFFF
:10A7B0000FC08882F6014081F70120812150842F4B
:10A7C000622F4F5F0E94F252882379F078820DC089
:10A7D0007882F6014081F70120812E5F842F622F5D
:10A7E0004F5F0E94F25281118882B394F4E0BF1649
:10A7F00009F08DCF2DC0F801E450F14F80818F5FBB
:10A8000080838830F8F01082F801ED5AF04F808193
:10A8100081FF04C0F801EF59FF4E0BC082FF04C056
:10A82000F801E45DF04F0BC083FF06C0F801E45D62
:10A83000F04F80818F5F05C0F801EF59FF4E808196
:10A840008150808381E0CDB7DEB7EDE00C94897D47
:10A850000D5A104F82E0F801808380E0F4CFCF934F
:10A86000DF93C82FD0E0FE01E450F14F10820E9428
:10A870006053882349F4FE01ED5AF04F908196FF12
:10A8800003C080E498279083FE01E956F04F808151
:10A890008F5F8083873050F01082FE01E057F04FC9
:10A8A00080818F5F8083843008F01082DF91CF91A8
:10A8B00008952091C20F281781F0422F50E0282FD1
:10A8C00030E0C90101974817590739F02F5F3F4F12
:10A8D0004217530711F080E008958091140F8617F6
:10A8E00081F0282F30E070E0CB010197281739075D
:10A8F00041F080E06F5F7F4F2617370719F481E042
:10A90000089581E00895209168102F3F21F12817C4
:10A9100071F0422F50E0282F30E0C901019748170D
:10A92000590729F02F5F3F4F42175307A1F4809139
:10A93000030F861791F0282F30E070E0CB010197CC
:10A940002817390751F080E06F5F7F4F26173707D0
:10A9500029F481E0089580E0089581E00895A0E061
:10A96000B0E0E5EBF4E50C94707DF82EE62EA02F18
:10A97000062F10E0A82EBB24C801880F991FF801EC
:10A98000B5E0EE0FFF1FBA95E1F7E81BF90BEA0DF2
:10A99000FB1DE05EFE4F3081532F5C51622F70E053
:10A9A000C42EDD24CB01880F991FFB01B5E0EE0F0B
:10A9B000FF1FBA95E1F7E81BF90BEC0DFD1DE05EFA
:10A9C000FE4FE081EC51573028F0832F86538230C0
:10A9D00008F056C0E23008F05CC065C0FD01E754E5
:10A9E000F04F8081882351F1FD01ED5AF04F8081B5
:10A9F00087FD24C0FD01E45DF04FE081FE1631F0DB
:10AA00008E2F90E00196A816B90641F48881E816C9
:10AA100079F190E001960817190751F14E1731F0BE
:10AA20008E2F90E00196C816D90641F48881281728
:10AA3000F9F090E0019668177907D1F01196219608
:10AA4000A530B10559F616C0852F8A509E2F9A5011
:10AA5000883070F5983060F48F2D6E2D0E94AF51C4
:10AA60000AC05554543020F480E0E554E43018F026
:10AA700081E001C080E0CDB7DEB7EAE00C948C7DC8
:10AA8000832F8252843008F4A5CF38533230E0F659
:10AA9000A1CF8E2F8A51823030F08C5E843018F036
:10AAA0008651823088F6C1E6D0E1A0E0B0E096CFD2
:10AAB000983000F3AA23A9F6DBCF982F8E5283316A
:10AAC00018F0805F863010F481E00895892F885255
:10AAD0008630D0F389518430B8F380E094529430BA
:10AAE000A0F781E00895382FE9EBFFE02FEF90E029
:10AAF0002F3F21F48081882309F4292F9F5F31960D
:10AB00009530B1F72F3F09F460C0A22FB0E0FD01EE
:10AB1000E45DF04F3083FD01EF59FF4E6083FD018E
:10AB2000E450F14F1082842F8757843008F043C0DF
:10AB3000FD01E754F04F83ED8083FD01E057F04FB6
:10AB400081E08083FD01E956F04F208330C0FD0194
:10AB5000E754F04F82ED8083FD01E057F04F81E034
:10AB60008083FD01E956F04F2083FD01ED5AF04F3F
:10AB7000413B11F488E401C081E480830895FD0124
:10AB8000E754F04F80ED09C0FD01E754F04F84ED2C
:10AB900004C0FD01E754F04F81ED8083FD01E057D3
:10ABA000F04F1082FD01E956F04F81E08083AD5AED
:10ABB000B04F8C930895842F815B823040F2433BE9
:10ABC000F1F2463709F3443B21F30895CF93DF9325
:10ABD000982F4EE1649F90011124C82FD0E0F90115
:10ABE000E05EFE4FEC0FFD1F80818C518630F8F443
:10ABF0009F5FA92FB0E0FD01E05EFE4FE20FF31F63
:10AC000080818C51863098F46F5F649FB00111246D
:10AC1000605E7E4FC60FD71F88818C51863038F416
:10AC200090E0A60FB71F8C918C51863008F091E010
:10AC3000892FDF91CF9108951F93CF93DF93C0E0C9
:10AC4000D0E01C2FFE01E55BFF4E90819F3F99F005
:10AC5000FE01E559FF4E8081882349F4FE01EF5E35
:10AC6000F04F892F60810E94E655882329F02196B4
:10AC7000C330D10531F71FEF812FDF91CF911F91A5
:10AC80000895A0E0B0E0E7E4F6E50C946F7DA82E0F
:10AC9000B62E85E0489FA0011124FA01E355FA4A37
:10ACA000E491F090220FCE2FD0E0CC0FDD1FCC0F1F
:10ACB000DD1FCE5AD84ABA0167557A4AEE24992444
:10ACC000939435C0FA01D490F901C490F7E1FF15CF
:10ACD000E8F08F2D90E0DC01AA0FBB1FAA0FBB1F6D
:10ACE000A80FB91FA45DBB4F0C931196BC9211978E
:10ACF0001296DC92129713961C921397CC2019F09F
:10AD000014969C9202C014961C92F394085F1F5FE5
:10AD10004F5F5F4F2F5F3F4F1230A1F6E3942296B3
:10AD20006E5F7F4F82E0E81639F0E8E0BE0E0A2D34
:10AD3000AB019E0110E0C6CFF092220FCDB7DEB777
:10AD4000EBE00C948B7D0F931F939091210F9F3F0D
:10AD500009F43FC18091060F80FF4EC0292F30E0DB
:10AD600003E0220F331F0A95E1F72C5F3F4FA22F1C
:10AD70008091AB0F682F70E0509142104091220FEC
:10AD80004831E8F4842F90E0FC01EE0FFF1FEE0F36
:10AD9000FF1FE80FF91FE45DFB4F2083CB01B3E0F9
:10ADA000880F991FBA95E1F70496851B818387E583
:10ADB00090E09383828314824F5F4093220F20910F
:10ADC000220F283108F005C1822F90E0FC01EE0F20
:10ADD000FF1FEE0FFF1FE80FF91FE45DFB4FA0837D
:10ADE0008CE0851B93E0660F771F9A95E1F7860F3D
:10ADF000818388E590E09EC081FF4DC0292F30E01F
:10AE000003E0220F331F0A95E1F72C5F3F4FA22F7B
:10AE10008091AB0F682F70E0509142104091220F4B
:10AE20004831E8F4842F90E0FC01EE0FFF1FEE0F95
:10AE3000FF1FE80FF91FE45DFB4F2083CB01B3E058
:10AE4000880F991FBA95E1F70496850F81838AE5EB
:10AE500090E09383828314824F5F4093220F20916E
:10AE6000220F283108F0B5C0822F90E0FC01EE0FD0
:10AE7000FF1FEE0FFF1FE80FF91FE45DFB4FA083DC
:10AE8000545F83E0660F771F8A95E1F7560F518371
:10AE900089E590E04FC0492F50E09091AB0F709141
:10AEA00042106091220F82FF49C0292F30E003E059
:10AEB000220F331F0A95E1F72C5F3F4FA22F683115
:10AEC000E8F4862F90E0FC01EE0FFF1FEE0FFF1F4E
:10AED000E80FF91FE45DFB4FCA01B3E0880F991F2B
:10AEE000BA95E1F70496871B808321838BE590E078
:10AEF0009383828314826F5F6093220F2091220FCD
:10AF0000283108F066C0822F90E0FC01EE0FFF1F91
:10AF1000EE0FFF1FE80FF91FE45DFB4F8CE0871B6E
:10AF200093E0440F551F9A95E1F7840F8083A18326
:10AF30008CE590E093838283148248C0292F30E00F
:10AF400083E0220F331F8A95E1F72C5F3F4FA22F3A
:10AF50006831F0F4862F90E0FC01EE0FFF1FEE0F3A
:10AF6000FF1FE80FF91FE45DFB4FCA0113E0880FD4
:10AF7000991F1A95E1F70496870F808321838CE54A
:10AF800090E09383828381E084836F5F6093220FDC
:10AF90002091220F2831E8F4822F90E0FC01EE0F7F
:10AFA000FF1FEE0FFF1FE80FF91FE45DFB4F745FFB
:10AFB00063E0440F551F6A95E1F7740F7083A18316
:10AFC0008BE590E09383828381E084832F5F2093DD
:10AFD000220F8091310FE82FF0E0DF01A470B070F4
:10AFE00082FF06C01091950F119500E040E113C05B
:10AFF00083FF05C01091950F00E048E10CC06091FF
:10B00000950F81FF04C0062F10E048E004C0062F12
:10B01000019510E040E08091950F882311F410E035
:10B0200000E080917F0E813041F480914E10480FF6
:10B030008091C20F6091140F71C080918A0F882394
:10B0400009F06EC02091040F8091070F821740F520
:10B05000E4FD26C0E0FD24C030E090E004968217B5
:10B06000930744F41092040F80919C0F880F880F6F
:10B070008093070F8091C20F880F880F880F810F70
:10B080006091140F660F660F660F600FE1FF02C03C
:10B0900047E244C0AB2B11F048E240C049E23EC059
:10B0A0008091C20F880F880F880F6091140F660F70
:10B0B000660F660F600F90914E10490F810F0E942E
:10B0C0004156209168102F3F59F18091850E609173
:10B0D000030F882359F4220F220F220F660F660FE9
:10B0E000660F600F812F820F4EE218C0E09167104B
:10B0F000F0E0EE0FFF1FE85AF04F80819181843B12
:10B10000910514F042E301C043E3220F220F220F06
:10B11000660F660F660F600F812F820F0E944156E7
:10B120001F910F910895ECE2F4E080EF8083359653
:10B1300094E0E43AF907D1F71092220F0E94A35647
:10B140002091220F30EF0DC0822F90E0FC01EE0F16
:10B15000FF1FEE0FFF1FE80FF91FE45DFB4F308369
:10B160002F5F283188F308951092800E10927F0E81
:10B17000ECE2F4E080EF8083359694E0E43AF9075E
:10B18000D1F71092220F89E694E00E941D4889E2CF
:10B1900090E30E940048089581E08093800E8093A0
:10B1A0007F0E83E061E00E94654D0895FF920F934A
:10B1B0001F93082FF62E142F842F6AE00E94357DEE
:10B1C000492F50E046575F4F802F8F5F6F2D0E94B1
:10B1D0000F48812F6AE00E94357D882329F4802F53
:10B1E0006F2D44E950E006C0482F50E046575F4FAE
:10B1F000802F6F2D0E940F481F910F91FF9008958F
:10B20000482F80E068E10E94D6580895A0E0B0E0A1
:10B21000ECE0F9E50C946E7DB82ED62E142F922E0C
:10B2200042E850E00E940F48A12EAB0C8A2D6D2DF4
:10B2300043E850E00E940F48C92CCD0C8B2D6C2D9B
:10B2400044E850E00E940F488A2D6C2D45E850E0FC
:10B250000E940F488B2C8394082DEB2CFF24E10EC9
:10B26000F11C0DC0802F6D2D4DE750E00E940F485E
:10B27000802F6C2D4EE750E00E940F480F5F802F0B
:10B2800090E08E159F0574F30D2D0F5F102FCD2DBF
:10B29000D0E0C90DD11D0DC08B2D612F4FE750E0BF
:10B2A0000E940F488A2D612F40E850E00E940F480D
:10B2B0001F5F812F90E08C179D0774F30DC0812FC5
:10B2C000602F44E950E00E940F481F5F812F90E0FB
:10B2D0008E159F05A4F30F5F802F90E08C179D07BC
:10B2E00014F4182DF3CFCDB7DEB7ECE00C948A7DC3
:10B2F000A0E0B0E0EEE7F9E50C946D7D782E862EA7
:10B30000942EA22EB02EF02EEE24E394C42EDD2433
:10B31000CC27DD27C01BD10B16C0872D682D4E2DE5
:10B3200021E00E94065917FF04C0CE010E94AE4DD5
:10B3300009C0FF2031F481E090E00E94AE4DFB2C6B
:10B3400001C0FA94E3948E2D90E0C816D9062CF72C
:10B35000FB2CEE24E394CA2CDD24CC27DD27C01B74
:10B36000D10B16C0872D682D492D2E2D0E94065910
:10B3700017FF04C0CE010E94AE4D09C0FF2031F47A
:10B3800081E090E00E94AE4DFB2C01C0FA94E39462
:10B390008E2D90E0C816D9062CF7CDB7DEB7EDE0BC
:10B3A0000C94897DFF920F931F93F82E00E00CC040
:10B3B000802F612F4F2D50E00E940F481F5F1C31DE
:10B3C000B9F70F5F0E3111F010E0F2CF1F910F911E
:10B3D000FF900895DF92EF92FF920F931F93E82E54
:10B3E000162FD42E082F0F5FF62EF39486E0481701
:10B3F000B1F48E2D46E050E00E940F48802F612F5F
:10B4000047E050E00E940F488E2D6F2D46E050E03F
:10B410000E940F48802F6F2D47E050E015C08E2D01
:10B4200048E050E00E940F48802F612F48E050E034
:10B430000E940F488E2D6F2D49E050E00E940F486A
:10B44000802F6F2D49E050E00E940F48812F90E03F
:10B4500003979595879590E02E2D30E0235030404E
:10B46000359527954BE050E0849FF001859FF00DC6
:10B47000949FF00D1124E20FF11DE853F04FD0829C
:10B480001F910F91FF90EF90DF900895DF92EF9260
:10B49000FF920F931F93182F062FD42E8AE0481780
:10B4A000C1F4812F4AE050E00E940F48E12EE3945E
:10B4B0008E2D602F4BE050E00E940F48F02EF39449
:10B4C000812F6F2D40E150E00E940F488E2D6F2D8F
:10B4D00035C08BE04817C1F4812F4EE050E00E9448
:10B4E0000F48E12EE3948E2D602F4FE050E00E9434
:10B4F0000F48F02EF394812F6F2D4CE050E00E9406
:10B500000F488E2D6F2D30C0F12EF394E62EE3946C
:10B510008CE04817B1F4812F4AE050E00E940F48B8
:10B520008F2D602F4FE050E00E940F48812F6E2D2D
:10B530004CE050E00E940F488F2D6E2D41E150E00D
:10B5400015C0812F4EE050E00E940F488F2D602FD4
:10B550004BE050E00E940F48812F6E2D40E150E0FB
:10B560000E940F488F2D6E2D4DE050E00E940F4835
:10B57000135003500695202F30E016958BE090E095
:10B58000289FF001299FF00D389FF00D1124E10F45
:10B59000F11DE853F04FD0821F910F91FF90EF9073
:10B5A000DF90089543E00E94465A0895A0E0B0E07D
:10B5B000ECEDFAE50C94727DE82EF42EFF0CFF0CF6
:10B5C000062FC62EDD24C82FD0E014C0EF2DF0E0EA
:10B5D000EE58F84AF394E491812F602F4E2F50E0FB
:10B5E0000E940F481F5F812F90E08C1B9D0B0297DC
:10B5F0006CF30F5F802F90E08C199D09029714F473
:10B600001E2DF1CFCDB7DEB7E8E00C948E7DA0E023
:10B61000B0E0EDE0FBE50C946D7DD82E062FEDEF4C
:10B62000EE2EE80E162F1350912F96958BE0989FD3
:10B63000E00111248E2D8695882E9924FE01E85371
:10B64000F04FE80DF91D4081EE2081F4442311F400
:10B6500041E013C04C3111F44DE10FC04A3111F4F7
:10B660004BE10BC0612F617080E004C0612F6170FD
:10B670008E2D81700E94044F482F8D2D602F50E039
:10B680000E940F487D2C73947EEFF72EFD0C8F2DBA
:10B690008695A82EBB24F501E853F04FEC0FFD1F53
:10B6A0004081FF2079F4442311F441E012C04C3171
:10B6B00011F44DE10EC04A3111F44BE10AC0117092
:10B6C00080E003C011708F2D8170612F0E94044FA4
:10B6D000482F872D602F50E00E940F48C02EC39442
:10B6E000102F1250912F96958BE0989FE001112416
:10B6F000FE01E853F04FE80DF91D4081EE2081F482
:10B70000442311F441E013C04C3111F44DE10FC05A
:10B710004A3111F44BE10BC0612F617080E004C02D
:10B72000612F61708E2D81700E94044F482F8D2DE6
:10B730006C2D50E00E940F48FE01E853F04FEA0DD7
:10B74000FB1D4081FF2079F4442311F441E012C035
:10B750004C3111F44DE10EC04A3111F44BE10AC0F5
:10B76000117080E003C011708F2D8170612F0E94D5
:10B77000044F482F872D6C2D50E00E940F48CDB705
:10B78000DEB7EDE00C94897DCF92DF92EF92FF92CD
:10B790000F931F93E82EF62ED82ED394C62EC39463
:10B7A0004423A9F440E050E00E940F488D2D6F2DF6
:10B7B00040E050E00E940F488E2D6C2D40E050E09C
:10B7C0000E940F488D2D6C2D40E050E018C0042FD2
:10B7D0000F5F50E00E940F48102F1F5F8D2D6F2DBF
:10B7E000402F50E00E940F488E2D6C2D412F50E0CD
:10B7F0000E940F481F5F8D2D6C2D412F50E00E943D
:10B800000F481F910F91FF90EF90DF90CF90089518
:10B81000482F2DE530E063E010C080818E528830E3
:10B8200088F4440F440F4E5E892F0E94C45B089534
:10B83000245C3F4F6E5F693151F0F901E05EFE4FCD
:10B8400093E0EBCF9E5F3296993139F7F1CF0895AF
:10B85000FF920F931F93CF93DF93082FF62E142F91
:10B86000A8E3BFE0E0E08C91882329F0EF5F119618
:10B87000EC30C9F7E0E0CE2FD0E0FE01E258F04F07
:10B880000083FE01EB5EF04FF082FE01EB5AFF4EAB
:10B890000083FE01E256F04FF082802F6F2D412F82
:10B8A0000E94C45B812F8F55883088F5C85CD04FCB
:10B8B0008DEC03C0C85CD04F8CEC88832EC0412F28
:10B8C0004954463138F5FE01E85CF04F8EEC808338
:10B8D000442321F4C355D04F81E005C0413029F401
:10B8E000C355D04F82E0888309C0FE01E355F04F75
:10B8F000423011F484E001C088E08083802F6F2DF6
:10B900000E94D65A0AC0C85CD04F83EDD6CF1736F6
:10B91000B1F6D0CF17571430B0F3CDB7DEB7E5E0AE
:10B920000C94917D1F93CF93DF9390E0FC01E75837
:10B93000F04FE081EC01CC0FDD1FCE018D5E182FA2
:10B94000EE2321F48BE1612F46E821C0E330D1F4EE
:10B950008BE1612F46E050E00E940F488CE1612F9F
:10B9600047E050E00E940F48CE018C5E182F8BE11B
:10B97000612F46E050E00E940F488CE1612F47E0C4
:10B9800050E021C0E23031F48BE1612F48E20E94A7
:10B99000C45B1BC08BE1612F4AE050E00E940F485E
:10B9A0008CE1612F4BE050E00E940F48CE018C5E8D
:10B9B000182F8BE1612F40E150E00E940F488CE18D
:10B9C000612F41E150E00E940F48DF91CF911F911C
:10B9D0000895CF92DF92EF92FF920F931F93E82E7C
:10B9E000E091830E81E8E89FF0011124E453F849C7
:10B9F000D49084E18D1590F4EE20E9F18D2D65E170
:10BA00000E94357D292F2D5F8D2D0E94357D682F59
:10BA10006D5F822F4DE30E94C45B2DC013E0C12EE9
:10BA2000CD0CFF248701000F111F000F111F075CB1
:10BA30001F4F8C2D61E0A8010E940F4894E0D90EA1
:10BA40000F5F1F4F8D2D61E0A8010E940F480F5F0F
:10BA50001F4F8C2D62E0A8010E940F488FE090E0FC
:10BA6000E80EF91EEE0CFF1CEE0CFF1C8D2D62E0A3
:10BA7000A7010E940F481F910F91FF90EF90DF9058
:10BA8000CF900895A0E0B0E0E8E4FDE50C94717D6E
:10BA90008091840E81FD87C082608093840EC0E017
:10BAA000D0E0FC2EBC2EB3948E01017010709EE28B
:10BAB000C92ED12CC00ED11E8B2D60E0A6010E9494
:10BAC0000F4883E0E82EEC0E005D1F4F8E2D61E0E5
:10BAD000A8010E940F480E5F1F4F8C2F8E5F62E0FF
:10BAE000A8010E940F480E5F1F4F81E06C2FA80134
:10BAF0000E940F4888E18C1750F082E06B2DA8015E
:10BB00000E940F488E2D69E1A6010E940F482196E0
:10BB1000CB31D10531F6C1E0D0E005E3C02ED12C08
:10BB20000C2FCA3150F4CE0181709070A601481BD1
:10BB3000590B89E16C2F0E940F480150CE01817092
:10BB40009070A601481B590B8AE1602F0E940F4894
:10BB50002196CC31D10521F783E061E047E350E045
:10BB60000E940F4883E062E048E350E00E940F48E3
:10BB700082E060E046E350E00E940F4889E160E027
:10BB800046E350E00E940F4882E069E146E350E05E
:10BB90000E940F4889E169E146E350E00E940F48A6
:10BBA00080E00E94E95CCDB7DEB7E9E00C948D7DC2
:10BBB000FF920F931F93F82E162F042F442339F072
:10BBC0004A3129F04C3119F0453409F061C0EEE1F9
:10BBD0001E9FF0011124EF0DF11D802F845EE05EA9
:10BBE000FE4F80838183868F878F83E0F81609F06C
:10BBF00062C0802F8554843008F04DC083E0612FEF
:10BC000048E450E00E940F481F5F83E0612F48E442
:10BC100050E03BC083E0612F41E050E00E940F48BC
:10BC20001F5F83E0612F41E050E02FC083E0612F70
:10BC30004DE150E00E940F481F5F83E0612F4DE10E
:10BC400050E023C083E0612F4CE250E00E940F4897
:10BC50001F5F83E0612F4DE250E017C083E0612F4A
:10BC60004BE150E00E940F481F5F83E0612F4BE1E2
:10BC700050E00BC083E0612F42E250E00E940F4889
:10BC80001F5F83E0612F43E250E00E940F4813C022
:10BC90000E94C45BAACF023008F4BCCF802F8C5125
:10BCA000823020F28C50863068F2825F8230B0F2AF
:10BCB0000E510630F8F21F910F91FF900895A0E009
:10BCC000B0E0E5E6FEE50C946E7D182FECE2F4E0C2
:10BCD00080EF8083359694E0E43AF907D1F781E06C
:10BCE00061E00E94654D84E90E94D25981E090E0B4
:10BCF0000E94AE4D1092310F10924E101092960F7E
:10BD00001092950F123318F41093830E02C0109204
:10BD1000830E10924A0F8FEF80934F0F8093FB0E8C
:10BD20001092100F109266101092080F1092490F87
:10BD30001092840E8093C30F8093C40F8093C50F1D
:10BD40008093C60F80E090E02FEFFC01E754F04FA6
:10BD50001082FC01E45DF04F20830196853091054F
:10BD6000A1F780E090E02FEFFC01E355F04F108247
:10BD7000FC01E85CF04F1082FC01E258F04F208398
:10BD800001968C30910581F780E090E02FEFFC0167
:10BD9000ED5BFF4E2083FC01E85DF04F10820196C1
:10BDA00084309105A1F720934B1010926B102093D3
:10BDB0004C1010926C1020934D1010926D10E8EC06
:10BDC000FFE0119280E1E134F807D9F7BB24882421
:10BDD000992421E8A22EAAC0EC2CE091830EEA9DC2
:10BDE000F0011124E80DF91DEC0DFD1DED5AF84987
:10BDF00014910C2D000F0D5F1882812F0E94F14EBF
:10BE0000882331F0802F6F2D412F0E94285C7DC048
:10BE1000812F815B823008F0FAC0802F6F2D40E0C7
:10BE20000E94D85D802F6F2D412F0E9473556DC0E9
:10BE30000093C20FF092140F802F6F2D40E00E94EC
:10BE4000D85D63C0802F6F2D412F0E94EA595DC0DD
:10BE5000802F6F2D412F0E94465A57C080914F0F5F
:10BE60008F3F19F4B0924F0F06C08091100F8B15C1
:10BE700010F4B092100F8091FB0E8F3F11F0E81676
:10BE800010F4E092FB0E809166108E1510F4E09293
:10BE90006610802F6F2D45E40E94D85D8091080FB9
:10BEA00080FD03C081608093080F85E488832DC0E6
:10BEB00080914A0F8F5F80934A0F123471F411E41E
:10BEC0000CC0E12FF0E0EC57F040DF01A55BBF4E66
:10BED0000C93EF5EF04FF08210E0802F6F2D412F1A
:10BEE0000E94D85D812F8C51823038F48091080FE8
:10BEF00081FD03C082608093080F812F0E94654FEF
:10BF0000882311F0188201C018830894C11CD11C29
:10BF100021969BE0C916D10409F05ECFB394EBE003
:10BF2000F0E08E0E9F1EFBE0BF1651F0FB2CFF0CC5
:10BF300083E0F80EE401C853D04FCC24DD244CCF6D
:10BF4000809166108F5F809366108091100F8F5FD5
:10BF50008093100F10925410109253101092440FAF
:10BF60009091830E81E8989FB0011124AB01425358
:10BF7000584920E030E0FA018491F901E758F04F88
:10BF80008083F901E05BF04F10822F5F3F4F4F5FDE
:10BF90005F4F2330310579F7FB01EF52F849E49107
:10BFA000E093AC0F82E08093310F80E00E94E95C67
:10BFB00010927E0E10928A0F109241108FEF809394
:10BFC000050F809368101092850E8093370F809331
:10BFD00067108093210F1092490F1092840E91E008
:10BFE0009093820E1092810E9093020110927D0E1A
:10BFF00084E18093C70F1092030185E480930B0FB7
:10C0000090939D0FCDB7DEB7ECE00C948A7D133B87
:10C0100009F403CF163709F400CF143B09F4FDCE21
:10C020001F3F09F405CF812F8650843008F40ACFD2
:10C030008450883008F40CCF8B53843008F40ECF32
:10C040008C5F843008F434CF8B53843008F439CFBC
:10C0500044CFFF920F931F93182F062FF62EF394C1
:10C06000823051F482E041E050E00E940F4882E0CB
:10C070006F2D41E050E008C040E050E00E940F48C2
:10C08000812F6F2D40E050E00E940F481F5F812FED
:10C09000602F40E050E00E940F480F5F812F602F1B
:10C0A00040E050E00E940F481F910F91FF900895CB
:10C0B0000F931F93CF93DF93062FE42FF52FEF01FC
:10C0C000182F01C021961F5FFE014491442379F08F
:10C0D0004F7740524032B1F3552747FD50954C58A9
:10C0E0005F4F812F8150602F0E940F48EBCFDF916F
:10C0F000CF911F910F9108950F931F93CF93DF93CB
:10C100008091840E80FD48C000E00CC0812F602F1C
:10C1100044E950E00E940F481F5F1F31B9F70F5FDD
:10C120000C3111F01BE1F2CF8BE162E040E457E605
:10C130000E9458608BE16AE04BE750E00E940F4894
:10C140008CE16AE04CE750E00E940F488BE162E12D
:10C1500043E457E60E9458604091830E4F5F8BE1A5
:10C1600063E00E94D6588BE16BE0409103010E948E
:10C17000D6588091840E81608093840E10E003E194
:10C180008BE1602F46E80E94C45B812F0E94925C85
:10C190001F5F0E5F1330A1F780917D0E6FE00E944C
:10C1A000357D9830A0F0C0E0D0E06C2FFE01E05B60
:10C1B000F04F8081882331F0660F6D5E8BE146E899
:10C1C0000E94C45B2196C330D10579F709C080E095
:10C1D0000E94925C81E00E94925C82E00E94925CEC
:10C1E000DF91CF911F910F9108958091840E82FD70
:10C1F00009C089E694E00E941D488091840E846005
:10C200008093840E8091840E83FD09C089E290E3BF
:10C210000E9400488091840E88608093840E8091F3
:10C22000840E81FD02C00E94425D8091840E80FDDB
:10C2300002C00E947C600895EF92FF920F931F93BB
:10C24000CF93DF938091800E882309F0E6C20E948D
:10C25000F5602091050F2F3F41F18091780F80FF0D
:10C2600004C090917C0F919504C081FF04C090910F
:10C270007C0F80E00DC082FF04C080917C0F81950F
:10C2800006C083FD02C090E0F4CF80917C0F90E067
:10C29000220F220F220F6091320F660F660F660F7A
:10C2A000690F820F42E30E9441560E94A35680917B
:10C2B0000201882309F447C00BE41FE0B8E5EB2E28
:10C2C000BFE0FB2EC0E0D0E0FE01ED5BFF4E208121
:10C2D0002F3F71F1FE01E85DF04FE081E6FD28C0DF
:10C2E00080916710C81721F18091370FC81701F1AD
:10C2F000E7FF05C0822FF801608142E317C0273CA9
:10C30000B8F4F8016081F70180819181843B910547
:10C3100014F042E301C043E370E0A3E0660F771F2F
:10C32000AA95E1F7822F880F880F880F0E94415647
:10C3300021960F5F1F4F82E090E0E80EF91EC43097
:10C34000D10511F6F8C01091810E012F0F5970918F
:10C35000220FC5E4DFE040E050E0FF24F394FA014F
:10C36000ED53F04F80818F3F09F445C0FA01ED5C39
:10C37000F04F808180FF03C02881219503C081FF99
:10C3800003C0288164E008C0988182FF03C0692F40
:10C39000619501C0692F24E0FA01E259FF4E308116
:10C3A000FA01E95BFF4EE081783128F5872F90E0B4
:10C3B000DC01AA0FBB1FAA0FBB1FA80FB91FA45DEA
:10C3C000BB4F330F330F330F360F3C93EE0FEE0F8F
:10C3D000EE0F2E0F11962C93119712960C93129725
:10C3E00013961C921397112319F01496FC9202C015
:10C3F00014961C927F5F4F5F5F4F2196443051052A
:10C4000009F0ADCF7093220F10E0A12FB0E0FD0135
:10C41000E754F04F3081332309F483C0FD01ED5A16
:10C42000F04FE081EF3F09F47CC08E2F90E0E4FDF7
:10C4300078C0FD01E450F14FE081EE2381F082FFEE
:10C4400003C02E2F219503C083FF03C02E2F90E041
:10C4500007C080FF03C09E2F919501C09E2F20E052
:10C46000323DA1F4FD01E45DF04F8081880F880F1B
:10C47000880FFD01EF59FF4E6081660F660F660F52
:10C48000690FA057B04F4C91415D48C0303D89F5D0
:10C4900086FF06C0FD01E057F04F4081405F19C0A4
:10C4A00080FF05C0FD01E057F04F408112C081FFC1
:10C4B00006C0FD01E057F04F40814C5F0AC0FD010E
:10C4C000E057F04F82FF03C04081485F02C04081C7
:10C4D000445FFD01E45DF04F8081880F880F880F75
:10C4E000AF59BF4E6C91660F660F660F690F4F5BB9
:10C4F00015C0333DB1F4FD01E45DF04F8081880F3C
:10C50000880F880FFD01EF59FF4E6081660F660F9F
:10C51000660F690FA057B04F4C914B5C820F0E9481
:10C5200041568091020190E0880F991F181B1F5FF0
:10C53000153008F46ACF80910201882309F4F9C00C
:10C540001091810E012F0F597091220FC5E4DFE089
:10C5500040E050E0FF24F394FA01ED53F04F808166
:10C560008F3F09F445C0FA01ED5CF04F808180FFF8
:10C5700003C02881219503C081FF03C0288164E0A6
:10C5800008C0988182FF03C0692F619501C0692F9F
:10C5900024E0FA01E259FF4E3081FA01E95BFF4ED7
:10C5A000E081783128F5872F90E0DC01AA0FBB1FCE
:10C5B000AA0FBB1FA80FB91FA45DBB4F330F330FCA
:10C5C000330F360F3C93EE0FEE0FEE0F2E0F11963A
:10C5D0002C93119712960C93129713961C92139703
:10C5E000112319F01496FC9202C014961C927F5FDE
:10C5F0004F5F5F4F21964430510509F0ADCF7093E6
:10C60000220F14E0A12FB0E0FD01E754F04F30817C
:10C61000332309F483C0FD01ED5AF04FE081EF3F71
:10C6200009F47CC08E2F90E0E4FD78C0FD01E45059
:10C63000F14FE081EE2381F082FF03C02E2F219580
:10C6400003C083FF03C02E2F90E007C080FF03C00C
:10C650009E2F919501C09E2F20E0323DA1F4FD0157
:10C66000E45DF04F8081880F880F880FFD01EF593E
:10C67000FF4E6081660F660F660F690FA057B04FBF
:10C680004C91415D48C0303D89F586FF06C0FD01F3
:10C69000E057F04F4081405F19C080FF05C0FD01A9
:10C6A000E057F04F408112C081FF06C0FD01E05706
:10C6B000F04F40814C5F0AC0FD01E057F04F82FF10
:10C6C00003C04081485F02C04081445FFD01E45DDA
:10C6D000F04F8081880F880F880FAF59BF4E6C9143
:10C6E000660F660F660F690F4F5B15C0333DB1F4DF
:10C6F000FD01E45DF04F8081880F880F880FFD01F8
:10C70000EF59FF4E6081660F660F660F690FA057E5
:10C71000B04F4C914B5C820F0E94415680910201B8
:10C7200090E0880F991F181B1F5F153008F46ACF1F
:10C7300046C00BE41FE068E5E62E6FE0F62EC0E091
:10C74000D0E0FE01ED5BFF4E20812F3F71F1FE0135
:10C75000E85DF04FE081E6FD28C080916710C817C2
:10C7600021F18091370FC81701F1E7FF05C0822F33
:10C77000F801608142E317C0273CB8F4F8016081FA
:10C78000F70180819181843B910514F042E301C05F
:10C7900043E370E053E0660F771F5A95E1F7822F6D
:10C7A000880F880F880F0E94415621960F5F1F4FF8
:10C7B00082E090E0E80EF91EC430D10511F60E9427
:10C7C0007C602091220F30EF0DC0822F90E0FC01A1
:10C7D000EE0FFF1FEE0FFF1FE80FF91FE45DFB4F89
:10C7E00030832F5F283188F380917D0E8F5F809397
:10C7F0007D0E9091810E21E092279093810E65E04D
:10C800000E94357D933018F02093020102C01092EF
:10C81000020181E090E00E94AE4DCDB7DEB7E6E0C8
:10C820000C94907DA1E0B0E0E8E1F4E60C94707D1A
:10C830008091820E80688093820E99EBE92E9FE0B2
:10C84000F92E0CE21FE0AA24BB248EE1C82E9CE145
:10C85000DD24DA94F501ED5AF04FE081E7FF0EC0D8
:10C86000F501E557F04FD501AD5DB04F80816C917A
:10C8700040E099830E94D85D998117C0D7018C91BF
:10C88000843D99F4E6FF11C0F501EF59FF4EE081B8
:10C89000EC9DF0011124D8018C91E80FF11DE05EB0
:10C8A000FE4F90839183968F978FF70111927F01AE
:10C8B000D801DD928D010894A11CB11CB5E0AB1626
:10C8C000B10441F608E31FE0EE24FF24F801808163
:10C8D0008823D1F0F701E355F04F808187FF07C02F
:10C8E000F701EB5AFF4ED701A256B04F06C0F70131
:10C8F000E258F04FD701AB5EB04F80816C9140E0C1
:10C900000E94D85DD8011C920894E11CF11C0F5FB5
:10C910001F4FBCE0EB16F104C9F68FEF80936E1049
:10C9200080936F1080937010809371100E941C612F
:10C930002196EAE00C948C7DAF92CF92EF920F9308
:10C940001F9384E90E94D25980E090E068E170E092
:10C950000E94784E1DE1E0EBCE2E812F6EE046E482
:10C9600057E62AE000ECEE24EA940E94E44E812F80
:10C970008A5F06C0E82FF0E0EC53FD4FC0828F5F66
:10C980008E31C0F3115082E090E00E94AE4D1C3019
:10C9900021F788E78093C20F1092140F8AE08093EA
:10C9A0004E1084E068E541E00E94844C11C0109272
:10C9B000220F8091C20F40914E100E9441568091EB
:10C9C000140F8D5F8093140F81E090E00E94AE4DB4
:10C9D0006091140F613658F361506093140F1092F8
:10C9E000220F40914E1042508091C20F0E9441563A
:10C9F00018E08DE06EE046E457E62AE00FEFE12E06
:10CA00007EEFC72EAA240E94844E8AE090E00E9406
:10CA1000AE4D115071F784E190E00E94AE4D8DE073
:10CA20006EE046E457E62AE00FEFE12E3EEFC32E1C
:10CA3000AA240E94844E8AE090E00E94AE4D1F5FBF
:10CA4000183069F785E063E041E00E94844C8AE099
:10CA500061E00E94654D8091870E803418F010923D
:10CA6000870E03C08F5F8093870E1F910F91EF9009
:10CA7000CF90AF9008950E943A499091820E94FF12
:10CA800004C080E198279093820EECE2F4E080EFFE
:10CA90008083359694E0E43AF907D1F71092220F9B
:10CAA00084E90E94D2598AE090E00E94AE4D8091C4
:10CAB000830E0E945F5E81E090E00E94AE4D81E0B7
:10CAC0008093820E83E060E00E944D4D86E19BE5FD
:10CAD0000E94134908950E943A498EE190E00E9415
:10CAE000AE4D0E943A4980E18093820E0895CF9224
:10CAF000DF92EF92FF920F931F930E943A490E9498
:10CB00001264ECE2F4E080EF8083359694E0E43A3E
:10CB1000F907D1F71092220F1092310F1092040FE3
:10CB20008FEF8093210F809367108093050F809380
:10CB3000681080E280934E100E94A3568EE190E030
:10CB40000E94AE4D11E01093F60E8BE08093FA0E2A
:10CB50008EE892E60E9413491093F60E1EE000EF55
:10CB600031E2C32E29E0D22E92E2E92E8BE0F82E9C
:10CB70002FC0ECE2F4E00083359684E0E43AF80755
:10CB8000D1F71092220F0E94A3562091220F0DC0C0
:10CB9000822F90E0FC01EE0FFF1FEE0FFF1FE80F4A
:10CBA000F91FE45DFB4F00832F5F283188F38091EC
:10CBB0004E10813229F4E0924E10F092FA0E04C029
:10CBC000C0924E10D092FA0E84E090E00E94AE4DDA
:10CBD000115078F61092F60E1092FA0E83E28093BE
:10CBE0004E101092220F0E94A3562091220F30EF78
:10CBF0000DC0822F90E0FC01EE0FFF1FEE0FFF1F14
:10CC0000E80FF91FE45DFB4F30832F5F283188F375
:10CC100089E090E00E94AE4D0E943A4987E390E09F
:10CC20000E94AE4D81E061E00E94654D80E18093FD
:10CC3000820E1F910F91FF90EF90DF90CF9008959B
:10CC4000EF92FF920F931F93CF93DF93082F10E083
:10CC5000F801ED53F04F80818F3F09F478C0F8015F
:10CC6000E259FF4EE080F801E95BFF4EF080F801E9
:10CC7000EB5BF04F8081882309F06BC08EE1F89E5A
:10CC8000900111246E2D70E0F901E05EFE4FE60F79
:10CC9000F71FE0818E2F8C51843220F0E156E43072
:10CCA00008F043C0E3944E2D50E0EA94FA01E05EB0
:10CCB000FE4FE20FF31FE0818E2F8C51843218F06B
:10CCC000E156E43090F5F3948EE1F89E9001112442
:10CCD000FA94F901E05EFE4FE60FF71FE0818E2F18
:10CCE0008C51843218F0E156E430F8F4F901E05E3A
:10CCF000FE4FE40FF51FE0818E2F8C51843218F027
:10CD0000E156E43090F48E2D6F2D0E946D528823F1
:10CD100061F48E2D6F2D0E94A752882331F48E2D41
:10CD20006F2D0E9483548823A1F08091490F815078
:10CD30008093490FD801AD53B04FEC91F0E0E3552B
:10CD4000F04F808190E4892780838FEF8C9380E07F
:10CD50003EC0E801CB5BD04F88818F5F88838830ED
:10CD6000A8F18E2D6F2D0E945954882319F00E942E
:10CD700077652CC01882F801E259FF4E4081F80116
:10CD8000ED5CF04F8081282F30E082FF02C08FEFF2
:10CD900007C0C90153E0969587955A95E1F78170D0
:10CDA000F801E259FF4E840F8083F801E95BFF4EE2
:10CDB000E08120FF02C08FEF04C036952795822FB7
:10CDC0008170095B1F4E8E0FF801808381E0CDB723
:10CDD000DEB7E6E00C94907DA0E0B0E0E2EFF6E68E
:10CDE0000C946B7D2091050F2F3FC1F08091411075
:10CDF000882309F44AC080918A0F9091C20F88233A
:10CE000021F5921759F49091140F8091320F9817D1
:10CE100029F41092411081E080938A0F03E410E11D
:10CE2000A8E28A2EAFE09A2EF8E5AF2EFFE0BF2EE3
:10CE3000EBE4EE2EEFE0FE2ECC24DD2455245394BB
:10CE400077247A9470E1672ECEC0892F90E0821B00
:10CE5000910997FF03C0909581959F4F029784F4A5
:10CE60008091140F282F30E08091320F281B310958
:10CE700037FF03C0309521953F4F2230310574F2C2
:10CE80001092411010928A0FC9CF8091020188231D
:10CE900029F28091810E882309F0C0CF4091780F4C
:10CEA00047FF39C080916A10815080936A108823AF
:10CEB00009F0B4CFE091370FF0E0DF01AD5BBF4E7A
:10CEC00088EC8C93DF01A85DB04F8C9190E48927AA
:10CED0008C93E254F04FA081A03180F0A051B0E0DB
:10CEE000FD01EE0FFF1FE05AF04F8FEF90E09183AE
:10CEF0008083A355B04F8C9180688C938FEF809383
:10CF0000050F8093370F80918A0F882309F486CF0D
:10CF10000E94776583CF80917C0F8F5F80937C0F19
:10CF2000883008F47BCF10927C0F942F40FF04C010
:10CF30008091320F815005C041FF06C08091320FB1
:10CF40008F5F8093320F07C042FF02C0215001C0A3
:10CF50002F5F2093050F8091050FE82FF0E03397A6
:10CF6000E0FD5CCF8091320F282F30E0235030401D
:10CF700020FD54CF96FF04C080E448274093780FEB
:10CF8000C90162E070E00E94557D262F30E0CF019C
:10CF900062E070E00E94557D8BE090E0289FF001F8
:10CFA000299FF00D389FF00D1124E60FF11DE85375
:10CFB000F04FE081E63411F481E00BC0E73411F466
:10CFC00082E007C0E83411F484E003C0E93421F4BE
:10CFD00088E08093780F22CF80E88093780F8AE5ED
:10CFE00080936A101BCFF80120812F3F09F4ACC059
:10CFF0008091370FC81609F4A7C0F401908196FDFF
:10D00000A3C097FF2CC090FF07C0F7018081845018
:10D0100080838830D8F408C091FF08C0F701808170
:10D020008C5F8083873C90F0F8010FC092FF07C0AF
:10D03000822F8450F8018083883040F406C0822F0C
:10D040008C5FF8018083803E08F07082F801808157
:10D050008F3F09F079C09058F401908375C0F501B5
:10D06000808191811816190624F401979183808399
:10D070006BC0809167108C1529F48091950F8823DF
:10D0800009F062C0809104018F5F80930401509287
:10D090009D0FF601E254F04F8081F70160818031ED
:10D0A000F0F18051C82FD0E0FE01E355F04F8081B0
:10D0B00086258083FE01E258F04F2083FE01EB5E5F
:10D0C000F04F6083FE01E85CF04FE081EE3C89F4B4
:10D0D00080FF02C040E009C081FF02C041E005C0FE
:10D0E00082FD02C043E001C042E0822F0E94D65A76
:10D0F00029C0EC3C11F447E608C0E33D11F040E0E4
:10D1000004C089E00E94005947E7FE01EB5EF04F42
:10D11000C258D04F888160810E94C45B13C0A82F81
:10D12000B0E0FD01ED5AF04F808186258083FD013E
:10D13000E45DF04F2083FD01EF59FF4E6083A45062
:10D14000B14F1C92F80170820894C11CD11C0F5F72
:10D150001F4F0894811C911C82E090E0A80EB91E1C
:10D160000894E11CF11C94E0C916D10409F03BCFEE
:10D17000CDB7DEB7EFE00C94877D0F931F93CF936D
:10D18000DF9308E51FE0C0E0D0E0F80111921192B2
:10D190008F01CE010E94EC662196C430D105A9F71B
:10D1A0000E9412648FEF8093C30F8093C40F80930B
:10D1B000C50F8093C60FDF91CF911F910F910895F6
:10D1C0008CE068EC40E00E94844C8DE068EC40E02C
:10D1D0000E94844C81E080937D0F0E94BD6881E0B5
:10D1E0000E94E95C80E00E94085C8091820E886069
:10D1F0008093820E0895482FA82FB0E0FD01E956D4
:10D20000F04F8081882319F0815080830BC08FE01C
:10D210008083FD01E057F04F80818F5F80838430F1
:10D2200008F010828091C20F282F30E0FD01E45DEC
:10D23000F04F8081281B310937FF03C030952195BD
:10D240003F4F922F8091140F282F30E0AF59BF4EDF
:10D250008C91281B310937FF03C0309521953F4F32
:10D26000822F923010F4222321F0823028F4992367
:10D2700019F40E9477650895842F0E9460530895E1
:10D28000A0E0B0E0E6E4F9E60C94687D182F062FE4
:10D29000322E0E943A4987E06FEF40E00E94844CB2
:10D2A000D090C20FDD0CDD0CDD0CE090140FEE0C05
:10D2B000EE0CEE0C8091310F80FF04C08091950F31
:10D2C000E81A0DC081FF04C08091950FE80E07C0D9
:10D2D0009091950F82FF02C0D91A01C0D90E80E249
:10D2E00080934E101092310F81E08093810EECE21A
:10D2F000F4E080EF8083359694E0E43AF907D1F7C3
:10D30000F12EFF0CFF0CFF0C000F000F000F10920E
:10D31000220F0E94A356CC2499249394AA24A39468
:10D320005524882410E06D2C7724CE2DD0E04424A1
:10D33000439480EF282E1092220F0E94A3561123AF
:10D3400021F58F2D90E08619970997FF03C09095DE
:10D3500081959F4F582E802F90E08C1B9D0B97FF3F
:10D3600003C0909581959F4F882EFD1418F486E098
:10D37000F80E04C0DF1410F49AEFF90E0E1510F435
:10D380000A5F03C0E01608F406506C2D615082E07D
:10D39000831530F04A2D465D862F8F0D602F04C017
:10D3A000600F4A2D445D8F2D0E944156992011F047
:10D3B000C39401C0CA9492E09C1508F4942484E0BC
:10D3C000851540F0881530F0B12EB394153118F062
:10D3D00011E002C0B12E10E02091220F0DC0822F6B
:10D3E00090E0FC01EE0FFF1FEE0FFF1FE80FF91F8B
:10D3F000E45DFB4F20822F5F283188F381E090E0CD
:10D400000E94AE4D112319F4A4241B2D94CF0E9429
:10D41000776581E0CDB7DEB7E2E10C94847DA6E0CC
:10D42000B0E0E5E1FAE60C94687D8091820E87FD1C
:10D43000F9C210E0812F0E9420661F5F1430D1F7DF
:10D4400088E39FE09C838B83EEE76E2EEFE07E2ED9
:10D4500070E6C72E7FE0D72E65E1E62E6FE0F62E50
:10D460005DEA852E5FE0952E45E5242E40E1342EC1
:10D47000EEE9FFE0FA83E9834424552430E4A32E47
:10D48000742DEB81FC819081992309F4A9C2F301E9
:10D490000081093C08F0A4C2F401408147FFA8C004
:10D4A000F60180819181823D9105E1F5F1010081D4
:10D4B000E981FA811081802F612F0E94E65588232F
:10D4C00009F1802F612F0E941C56A82FB0E0FD01AA
:10D4D000E55BFF4E90819F3F39F09D0125593F4EFE
:10D4E000F9018081882319F08FEFF1010AC0F10161
:10D4F0009083AF5EB04F8C91E981FA81808381E0A7
:10D50000F9018083F10180818F3F39F0E981FA814F
:10D51000608142E00E94C45B05C084EA91E0F601AC
:10D5200091838083F60180819181009709F05BC02F
:10D53000F1011081E981FA810081812F602F0E9421
:10D54000E655882301F1F201E258F04F8FEF808316
:10D5500085E19FE0480E591EF20190818EE1989F6F
:10D56000F00111242FEF91E005C01C92222309F451
:10D570009C932F5FDF01A20FB11DA05EBE4F8C9167
:10D58000863098F3F6CFF3011083F7010083F4019E
:10D590008081F0E98F27F4018083EB81FC81908109
:10D5A0009E3CD1F480FF02C040E009C081FF02C070
:10D5B00041E005C082FD02C043E001C042E080912D
:10D5C000820E90E084709070880F991F880F991FC9
:10D5D000480F812F602F21C0933D09F001C2812F98
:10D5E000602F47E784C10197F60191838083F8C1DA
:10D5F00044FDF6C19E3C09F0D5C045FD24C0809194
:10D60000820E82FFEDC1842F8062F401808380FF4F
:10D6100007C0802FF701608144E00E94D65AE0C124
:10D6200081FF05C0802FF701608145E0F6CF82FFC2
:10D6300005C0802FF701608146E0EFCF802FF70112
:10D64000608147E0EACF6091C20FF701208110911D
:10D65000140F8091490F843009F4C2C146FDC0C146
:10D66000E3ECFFE050E080818F3F29F05F5F31966F
:10D670005430C9F750E0802F90E0861B910997FF46
:10D6800003C0909581959F4F982FE52FF0E0FE8382
:10D69000ED83E259FF4E0083AD81BE81A95BBF4E91
:10D6A0002C93ED81FE81ED5CF04F4083ED81FE8196
:10D6B000ED53F04F70834064F40140838091490F33
:10D6C0008F5F8093490F342F40FF09C08091140F62
:10D6D000821728F4923018F422502C9344C031FF62
:10D6E0000DC08091140F281748F4923038F4ED8162
:10D6F000FE81E95BFF4E2E5F208335C0822F90E0D4
:10D70000811B910997FF03C0909581959F4F982F9A
:10D7100032FF0CC08091C20F801740F4923030F479
:10D72000ED81FE81E259FF4E02500DC033FF0DC066
:10D730008091C20F081748F4923038F4ED81FE81D1
:10D74000E259FF4E0E5F00830EC08D819E818D5386
:10D75000904F9E838D838FEFED81FE8180834A25DC
:10D76000F401408313C0852F0E9420668823A1F412
:10D770008D819E818D53904F9E838D838FEFED81A0
:10D78000FE818083F40180818A2580838091490F06
:10D7900081508093490F24C18CE06FEF40E00E94DC
:10D7A000844C1EC1933D41F58091820E82FF18C1C9
:10D7B000802FF701608140E00E94D85DEB81FC8101
:10D7C000108294E0A92FB0E0FD01E754F04F808172
:10D7D000833D79F083ED80839D01245D304FF3011B
:10D7E0008081F9018083AF59BF4EF70180818C930E
:10D7F000F7C0915038F7F4C080919D0F882309F449
:10D80000EFC09D3C09F076C0202F30E08091C20F20
:10D81000281B310937FF03C0309521953F4FB22EA9
:10D82000F7016081262F30E08091140F281B310909
:10D8300037FF03C0309521953F4F122FF1E0FB15C4
:10D8400018F4223008F051C0802F43E60E94C45BD8
:10D85000BB2011F5F70160818091140F681770F4F7
:10D86000F30180810E94F94F882309F4B9C0F301C4
:10D870008081F70160814FE522E034C0F3018081AF
:10D880000E94834F882309F4ABC0F3018081F70124
:10D8900060814FE521E026C0112309F0A1C0F3010A
:10D8A00090818091C20F981778F4892FF7016081D9
:10D8B0000E94F150882309F493C0F3018081F7019D
:10D8C00060814FE528E00EC0892FF70160810E943A
:10D8D0006F50882309F484C0F3018081F7016081CF
:10D8E0004FE524E00E9440697BC0802F4FE50E94F5
:10D8F000C45B76C09C3C09F073C080917D0F882387
:10D9000009F06EC08091820E82FF33C080910201C7
:10D91000882309F065C0F6018081918143FF0BC027
:10D92000019691838083449798F083E190E09183FE
:10D93000808384E00BC00197F601918380838F3F41
:10D94000910531F028F01182108288E0F401808383
:10D95000F6018081918165E070E00E94417DAB011C
:10D96000440F551F440F551F4959802FF7016081FF
:10D97000BECF8091C20F902F981BF7016081262F98
:10D9800030E08091140F281B310937FF03C0309518
:10D9900021953F4F93302CF010E02430B8F011E087
:10D9A00015C097FD06C0802F4BE60E94C45B11E0B6
:10D9B00014C09F3F31F4802F4FE60E94C45B12E0F9
:10D9C0000CC0243010F413E001C012E0412F440FCA
:10D9D000440F4959802F0E94C45BF60110831182C5
:10D9E0000894411C511C8B819C8101969C838B83E4
:10D9F0000894611C711CE2E0F0E0CE0EDF1E08947A
:10DA0000E11CF11C0894811C911C0894211C311C00
:10DA100089819A8101969A8389839CE049165104F1
:10DA200009F02ECD2696E2E10C94847DEF92FF92D0
:10DA30000F931F93CF93DF93082F10E0F801E9565F
:10DA4000F04F8081882319F081508083DCC0809161
:10DA50000201882369F08091810E882349F0F80142
:10DA6000E057F04F90E08081882309F491E09083A3
:10DA7000A3E5EA2EAFE0FA2EE00EF11EF701908149
:10DA800096FF50C080E48927808382FF13C0F8018D
:10DA9000E45DF04F40814150F801EF59FF4E208185
:10DAA000842F622F2F5F0E94F252882309F462C0F4
:10DAB00088E035C083FF13C0F801E45DF04F40817A
:10DAC0004E5FF801EF59FF4E2081842F622F2F5FA8
:10DAD0000E94F252882309F44DC084E020C0F8016E
:10DAE000E45DF04FE801CF59DF4E80FF0DC0688143
:10DAF0004081262F2F5F842F61504F5F0E94F2528A
:10DB00008823C1F182E00BC0408128812E5F842FE1
:10DB1000622F4F5F0E94F252882361F181E0F7018A
:10DB2000808328C0F801E450F14F80818F5F8083AB
:10DB3000883000F11082892F8064F701808382FF92
:10DB400006C0F801E45DF04F80818150E9CF83FF8A
:10DB500006C0F801E45DF04F80818F5FE1CFE801FE
:10DB6000CF59DF4E80FF03C08881815002C0888179
:10DB70008F5F88833091C20FFCE2EF2EFFE0FF2E13
:10DB8000E00EF11EF7019081E801CF59DF4E2091A0
:10DB9000140F3917C9F46881621758F4832F0E9453
:10DBA000F94F882381F1F701808168814FE522E0F8
:10DBB00027C0832F0E94834F882329F1F70180819A
:10DBC00068814FE521E01CC088812817E1F4931794
:10DBD00060F4892F622F0E94F1508823A1F0F70191
:10DBE000808168814FE528E00BC0892F622F0E9459
:10DBF0006F50882341F0F701808168814FE524E070
:10DC00000E94406901C080E0CDB7DEB7E6E00C9429
:10DC1000907D80910E0F90910F0F90930D0F809338
:10DC20000C0F80E00E942C4890930F0F80930E0FF2
:10DC30000895FF920F931F93ECE2F4E080EF80834E
:10DC4000359694E0E43AF907D1F71092220F81E07B
:10DC500090E00E94AE4D40E050E029E131E00CC080
:10DC600081918D93E617F707D9F7465F5F4F225EE4
:10DC70003F4F4C33510551F0F901E05EFE4FDA01A0
:10DC8000AC55BB4FB901665D7E4FEACF8BE069E0D2
:10DC900048E025E00EEF1FEF0E9478598CE06AE023
:10DCA00048E257E60E9458608CE06BE04DE257E690
:10DCB0000E9458608CE06CE043E357E60E94586095
:10DCC0008CE06DE04BE357E60E94586000E0FF24D3
:10DCD000F3940E94096E20910E0F23FF73C0809170
:10DCE0000C0F83FD6FC010927F0E1092800E40E0EB
:10DCF00050E029E131E00CC08D918193E617F707E0
:10DD0000D9F7465F5F4F225E3F4F4C33510551F0CC
:10DD1000DA01AC55BB4FF901E05EFE4FB901665D1B
:10DD20007E4FEACF002311F4000015C0013019F432
:10DD30000E94776510C0023031F400937F0E81E0BD
:10DD40008093800E08C081E080937F0E8093800EC8
:10DD500061E00E94654D81E090E00E94AE4D1F9110
:10DD60000F91FF90089580910C0F90910D0FB4E0EA
:10DD700096958795BA95E1F781708F1521F000236C
:10DD800011F0015009C025FF07C080910C0F85FDDF
:10DD900003C0033008F40F5F1AE08BE0612F4FE7F8
:10DDA00050E00E940F481F5F1E30B9F7602F665F7A
:10DDB0008BE041E850E00E940F4881E090E00E9433
:10DDC000AE4D87CF24FDCFCFDECF0E94096E80916C
:10DDD0007F0E882309F058C080910E0F82FF06C085
:10DDE00080910C0F82FD02C00E946B6520910E0F86
:10DDF00030910F0F23FF43C080910C0F83FD3FC074
:10DE000081E08093800E84E080937F0E089580915E
:10DE10004110882389F424FF02C081E10BC025FF53
:10DE200002C082E107C026FF02C084E103C027FFD1
:10DE300003C088E18093310F20FF08C080910C0F50
:10DE400080FD04C08091310F80620BC030FF0BC099
:10DE500080910C0F90910D0F90FD05C08091310FB6
:10DE600080648093310F9091820E91FD0DC080915E
:10DE7000310F84FF09C092609093820E08958091C3
:10DE8000950F882321F2D8CF089588E090E00E9472
:10DE90004248843108F084E10895A0E0B0E0E3E571
:10DEA000FFE60C946E7D80E090E00E94456FB82EF6
:10DEB000D090830E81E090E00E94AE4D89E694E020
:10DEC0000E941D4884E90E94D25981E090E00E949E
:10DED000AE4DCC2411E082E0A82EB0EF9B2E88241A
:10DEE00083940E94E56E80E38D1578F090910E0F7B
:10DEF00094FFB6C180910C0F84FDB2C104C0809123
:10DF00000C0F87FDAFC1D3945CC090910E0F95FFAD
:10DF1000ADC180910C0F85FDA9C104C080910C0F8B
:10DF200086FD02C0DA944DC020910E0F30910F0F84
:10DF300032FF0DC080910C0F90910D0F92FD07C024
:10DF400086EFD80E82E38D15E0F5DD243AC033FF6D
:10DF50000EC080910C0F90910D0F93FD08C08AE0C8
:10DF6000D80E81E38D1568F5A1E3DA2E2AC023FFD0
:10DF700025C080910C0F83FD21C0CC2029F087E0C3
:10DF80006FEF41E00E94844C89E06FEF41E00E9416
:10DF9000844CD092830E10927F0E1092800E1092BD
:10DFA000840E86E061E00E94654D85E060E00E949D
:10DFB0004D4DCDB7DEB7ECE00C948A7D112309F40A
:10DFC0004AC18D2D0E945F5EA092040F1092220F15
:10DFD000ECE2F4E09082359684E0E43AF807D1F779
:10DFE00081E090E00E94AE4D0E94425D0E947C6004
:10DFF0001091810E012F0F597091220FC5E4DFE0BF
:10E0000040E050E0FA01ED53F04F80818F3F09F47A
:10E0100045C0FA01ED5CF04F808180FF03C028818C
:10E02000219503C081FF03C0288164E008C0988166
:10E0300082FF03C0692F619501C0692F24E0FA01B6
:10E04000E259FF4E3081FA01E95BFF4EE081783101
:10E0500028F5872F90E0DC01AA0FBB1FAA0FBB1F7A
:10E06000A80FB91FA45DBB4F330F330F330F360F0B
:10E070003C93EE0FEE0FEE0F2E0F11962C9311978F
:10E0800012960C93129713961C921397112319F062
:10E0900014968C9202C014961C927F5F4F5F5F4F64
:10E0A00021964430510509F0ADCF7093220F1091A5
:10E0B0000201110F110FA12FB0E0FD01E754F04F45
:10E0C0003081332309F483C0FD01ED5AF04FE08124
:10E0D000EF3F09F47CC08E2F90E0E4FD78C0FD0195
:10E0E000E450F14FE081EE2381F082FF03C02E2F38
:10E0F000219503C083FF03C02E2F90E007C080FF4F
:10E1000003C09E2F919501C09E2F20E0323DA1F4C7
:10E11000FD01E45DF04F8081880F880F880FFD01BD
:10E12000EF59FF4E6081660F660F660F690FA057AB
:10E13000B04F4C91415D48C0303D89F586FF06C027
:10E14000FD01E057F04F4081405F19C080FF05C0DE
:10E15000FD01E057F04F408112C081FF06C0FD0174
:10E16000E057F04F40814C5F0AC0FD01E057F04F8F
:10E1700082FF03C04081485F02C04081445FFD01CF
:10E18000E45DF04F8081880F880F880FAF59BF4E34
:10E190006C91660F660F660F690F4F5B15C0333DBC
:10E1A000B1F4FD01E45DF04F8081880F880F880F86
:10E1B000FD01EF59FF4E6081660F660F660F690F14
:10E1C000A057B04F4C914B5C820F0E9441568091FA
:10E1D000020190E0880F991F181B1F5F153008F48B
:10E1E0006ACF0E94A35681E060E00E944D4DBD14AD
:10E1F00010F4CC24C3948C2D90E07C01EE0CFF1C19
:10E20000E80EF91EE194AC0113E0440F551F1A9576
:10E21000E1F7481B590B475F8E2D875F60E022E0D6
:10E220000EEF1FEF0E9478598E2D865F61E04BE163
:10E2300057E60E9458604D2D4F5F8E2D805F61E044
:10E240000E94D658CC2031F080E161E041E257E6EF
:10E250000E94586010E081E090E00E94AE4D41CEF7
:10E2600097FD4DCEDD2009F45FCE4FCE96FF5CCEFC
:10E2700055CE1F93182F0E94456F181710F480E099
:10E2800006C088E090E0612F0E94384881E01F912D
:10E2900008950F931F938091830E0E94397181E03E
:10E2A0008093310F1092950F10924E10E091830ED3
:10E2B00081E8E89FF0011124E453F849E491E73143
:10E2C00018F410E000EF22C00E943A4922C00083F7
:10E2D000359684E0E43AF807D1F71092220F809146
:10E2E000950F8F5F8093950F80914E108F5F809375
:10E2F0004E10883010F010924E100E94A35681E00C
:10E3000090E00E94AE4D1F5F183019F0ECE2F4E08F
:10E31000DECF8091830E8F5F8093830E80E18093A8
:10E32000820E1F910F910895AF92BF92DF92EF92EC
:10E33000FF920F931F93DF93CF930F92CDB7DEB76A
:10E340008091820E882311F40C94987A84FF02C085
:10E350000E943B65ECE2F4E080EF8083359694E028
:10E36000E43AF907D1F71092220F8091870E80349A
:10E3700018F01092870E03C08F5F8093870EE09194
:10E38000870EF0E0E151FF47E491E0939C0F0E947B
:10E390000F6A8091820E81FF28C087FD26C000E0B1
:10E3A00010E0F801E754F04F80818823C9F0F801AC
:10E3B000ED5AF04FE081EF3F99F0E4FD11C0823D4E
:10E3C00021F4802F0E94166D0BC0803D21F4802F18
:10E3D0000E942F5405C0833D19F4802F0E94FB68D2
:10E3E0000F5F1F4F05301105E1F60E94EC6680912A
:10E3F000210F8F3F09F050C080910401882309F458
:10E400004BC08091310F982F85FF46C0809103014A
:10E41000882309F441C0809168108F3FE9F590FF8F
:10E4200008C08091C20F8093210F8091140F8150FA
:10E4300009C091FF0AC08091C20F8093210F809183
:10E44000140F8F5F8093AB0F0DC08091C20F20918E
:10E45000140F92FF02C0815001C08F5F8093210F83
:10E460002093AB0F9091310F80E298279093310F5A
:10E470008091950F809342109093060F4091030175
:10E480004150409303018BE16BE00E94D65884E039
:10E490006FEF41E00E94844CE090210F8E2D83505D
:10E4A000873108F0A8C71091AB0F133008F4A3C749
:10E4B0001A3108F0A0C7D0904210DD2029F08091D9
:10E4C000950FD81609F090C18091310F80FF03C0DD
:10E4D000F12EFA9404C081FF04C0F12EF3940E2DA6
:10E4E00008C082FF03C00E2D015002C00E2D0F5F29
:10E4F000F12E8F2D90E0FC0135E0EE0FFF1F3A95D5
:10E50000E1F7880F991FE81BF90BE00FF11DE05EA2
:10E51000FE4F80818C510E945D55882361F08FEF02
:10E520008093210F9091310F95FF7FC180E2982752
:10E530009093310F7AC1E3E4F0E1A0E080818F3F56
:10E5400029F0AF5F3196A430C9F755C720E030E01D
:10E55000422FF901E85CF04F8081882309F446C01E
:10E56000F901E258F04F8081801709F03FC0F901AE
:10E57000EB5EF04F80818F15C9F58FEF8093210FEF
:10E580009091310F95FF04C080E298279093310F4E
:10E59000F901E355F04F808180618083EA2FF0E03C
:10E5A000DF01A254B04F405F4C93BF016D5B7F4EC3
:10E5B000A9014258504FDA018C91DB018C938F01F5
:10E5C000055B104F2B5E304FD9016C91D8016C93D5
:10E5D00094E6DA019C93D9019C93EE0FFF1FE85A51
:10E5E000F04F24EA31E03183208359C02F5F3F4F41
:10E5F0002C30310509F0ACCF40E050E0242FFA0177
:10E60000E45DF04F8081801709F04CC0FA01EF59AA
:10E61000FF4E80818F1509F045C0FA01ED5AF04F89
:10E62000808184FD3FC08FEF8093210F9091310F47
:10E6300095FF04C080E298279093310FFA01E754C8
:10E64000F04F8081823D09F4F0C0FA01ED5AF04F9D
:10E65000808180618083B0E0FD01E254F04F20832F
:10E660009D012D5B3F4EFA01E45DF04F8081F90181
:10E6700080839D01255B304F4F595F4EFA016081C9
:10E68000F9016083FD01E45DF04F98E19083AA0FEA
:10E69000BB1FA85AB04F24EA31E02D933C930E944F
:10E6A000075BC3C04F5F5F4F4530510509F0A6CFF0
:10E6B00067E470E1A0E0B0E04E2D50E0212F30E0A3
:10E6C000FD01ED53F04F80818F3F01F1FD01E259D3
:10E6D000FF4EB080BE1441F4FB01808190E0821BAC
:10E6E000930B0196039758F0FB018081811771F419
:10E6F0008B2D90E0841B950B0196039738F48FEFD8
:10E700008093210FA259BF4E8C938FC011966F5FDB
:10E710007F4FA430B105A1F6AA24BB24F501ED5B1F
:10E72000FF4EE081EF3F09F457C0E01709F054C0F5
:10E73000F501E55BF04F80818F1509F04DC08FEF3B
:10E740008093210F9091310F95FF04C080E29827AC
:10E750009093310F85E064EB41E00E94844CF50119
:10E76000E85DF04F8091060F80688083F501ED5BD6
:10E77000FF4E808190E013E0880F991F1A95E1F712
:10E780008083F501E55BF04F808190E0B3E0880F76
:10E79000991FBA95E1F780838EEB9FE0A80EB91E12
:10E7A000D5018C91E82FF0E0803180F07097DF0187
:10E7B000A355B04F8C9180688C93EE0FFF1FE05AE9
:10E7C000F04F84EA91E0918380832FC0ED5AF04F9F
:10E7D00080818068808329C00894A11CB11CB4E0AA
:10E7E000AB16B10409F09ACF8D2D8E5F8093421045
:10E7F0008830D8F0109242108091060F80FF04C03C
:10E800008091AB0F815005C081FF06C08091AB0F96
:10E810008F5F8093AB0F09C09091210F82FF02C0E0
:10E82000915001C09F5F9093210F8091310F282F4D
:10E8300086FF7BC080915310A82FB0E0FD01E05B04
:10E84000F04F8081882309F470C0A758B04F4C91D5
:10E85000442309F464C03091C20F832F90E00397E2
:10E8600080FD5DC06091140F862F90E0039780FDBE
:10E8700056C020FF02C0625003C021FF03C06E5F7C
:10E88000232F07C022FF03C0232F225002C0232FB3
:10E890002E5F862F90E0FC0175E0EE0FFF1F7A954A
:10E8A000E1F7880F991FE81BF90BE20FF11DE05EFD
:10E8B000FE4FE081433069F4E156E43080F52317E0
:10E8C00019F0822F48E002C0822F46E00E94EA59E8
:10E8D0000FC0413039F4E652E83008F5822F0E942B
:10E8E000D25A06C0E454E630D0F4822F0E94296048
:10E8F00084E06FEF40E00E94844C80915310E82F39
:10E90000F0E0DF01A05BB04F1C92E758F04F10829F
:10E910000E94925C809153108F5F8093531080917E
:10E92000310F90E489278093310F40917C0F44236D
:10E9300011F180918A0F8823F1F08091050F809367
:10E94000C20F8091320F8093140F4093950F8091E6
:10E95000780F80FF02C081E003C081FF04C082E025
:10E960008093310FAAC482FF02C084E0F9CF83FFF5
:10E97000A4C488E0F5CF80914110882361F1809193
:10E98000950F8F5F8093950F883008F496C410928E
:10E99000950F2091C20F8091310F90E082FF02C04D
:10E9A0008FEF06C043E0969587954A95E1F7817011
:10E9B000820F8093C20F2091140F8091310F90E04D
:10E9C00080FF02C08FEF03C0969587958170820FFC
:10E9D0008093140F72C48091310F982F84FF66C406
:10E9E0008091950F882309F0F6C180918A0F8823C2
:10E9F00019F0442309F003C590FF8CC08091820E6A
:10EA000083FF1AC08091140F8330B1F4E091830E1C
:10EA100081E8E89FF0011124E453F849E4912E2F96
:10EA200030E02D5F3F4F8091C20F90E028173907EB
:10EA300019F40E944971E3C4442389F49091C20FF0
:10EA40008091050F981759F42091140F30E08091B0
:10EA5000320F90E002962817390709F44DC16091F2
:10EA6000140F61508091C20F41E00E94E951882348
:10EA700009F448C0863249F090E08E3D09F491E0F7
:10EA80009093850E992309F4BAC44091C20F209146
:10EA9000140F2350842F622F4F5F0091850E0E9428
:10EAA000AF54882309F0ABC49091C20F90936810C3
:10EAB0009093AA0F8091140F682F62506093030FF8
:10EAC0008350809369101092090F8091850E8823DE
:10EAD00009F46AC120E030E0422FF901ED5BFF4EFE
:10EAE0008081891731F4F901E55BF04F8081861749
:10EAF00031F02F5F3F4F2430310571F740E04093F4
:10EB0000671055C18091C20F6091140F61508F5FE3
:10EB100041E05AC191FF6EC0442389F49091C20F25
:10EB20008091050F981759F42091140F30E08091CF
:10EB3000320F90E002972817390709F4DDC0609181
:10EB4000140F6E5F8091C20F42E00E94E951182FAE
:10EB5000882309F447C0843219F08C3D09F04FC472
:10EB60004091C20F2091140F2C5F842F622F4F5FB2
:10EB70000091850E0E94AF54882309F040C4909103
:10EB8000C20F909368109093AA0F8091140F682F72
:10EB90006E5F6093030F8D5F809369101092090F71
:10EBA0001C3D19F0103E09F0FFC081E08093850EF6
:10EBB000509168104091030F20E030E0922FF9014E
:10EBC000ED5BFF4E8081851739F4F901E55BF04F6D
:10EBD0008081841709F4E5C02F5F3F4F2430310551
:10EBE00069F7DEC08091C20F6091140F6E5F8F5F76
:10EBF00042E0EAC092FF6EC0442389F49091140F62
:10EC00008091320F981759F42091C20F30E0809113
:10EC1000050F90E002962817390709F46DC080911E
:10EC2000C20F81506091140F44E00E94E951182FE7
:10EC3000882309F447C0853219F08D3D09F0DFC300
:10EC40004091C20F43502091140F842F622F2F5FE9
:10EC50000091850E0E94AF54882309F0D0C38091A3
:10EC6000C20F982F92509093681083508093AA0FF0
:10EC70006091140F6093030F609369101092090F55
:10EC80001D3D19F0113E09F08FC081E08093850E83
:10EC9000509168104091030F20E030E0922FF9016D
:10ECA000ED5BFF4E8081851739F4F901E55BF04F8C
:10ECB0008081841709F475C02F5F3F4F24303105E0
:10ECC00069F76EC08091C20F6091140F6F5F815021
:10ECD00044E07AC04423A1F49091140F8091320F44
:10ECE000981771F42091C20F30E08091050F90E0E9
:10ECF00002972817390721F481E08093411069C0F9
:10ED00008091C20F8E5F6091140F48E00E94E9511C
:10ED1000182F882309F451C0843219F08C3D09F072
:10ED20006EC34091C20F4C5F2091140F842F622F4D
:10ED30002F5F0091850E0E94AF54882309F05FC3B6
:10ED40008091C20F982F9E5F909368108D5F809383
:10ED5000AA0F6091140F6093030F609369101092D3
:10ED6000090F1C3D11F0103EF9F481E08093850EEF
:10ED7000509168104091030F20E030E0922FF9018C
:10ED8000ED5BFF4E8081851731F4F901E55BF04FB3
:10ED90008081841731F02F5F3F4F2430310571F7A8
:10EDA00090E09093671003C0892F0E94075B81E079
:10EDB00080937D0F10928A0F0CC08091C20F6091DA
:10EDC000140F6F5F8E5F48E00E94E951882309F0BD
:10EDD00016C31092040F8091810E882321F0809138
:10EDE0007E0E882311F58091960F882319F08150AB
:10EDF0008093960F8091960F882361F480914E1036
:10EE00008F5F80934E1093E09093960F883010F0B0
:10EE100010924E109091950F9F5F9093950F809157
:10EE200068108F3F11F09093090F8091950F8830F3
:10EE300008F443C221E020939D0F1092950F80911A
:10EE4000310F80FF3DC01091140F11501093140F1B
:10EE50001F5F809168108F3F09F43FC1F090C20F8F
:10EE6000912F93508091850E882391F48F2D692FD7
:10EE700044E250E099830E940F480F2D0F5F802FCE
:10EE80009981692F45E250E00E940F481250CCC092
:10EE900020937D0F8091050F8F3F09F00AC14EE14D
:10EEA000949F900111246F2D70E0F901E05EFE4FF8
:10EEB000E60FF71F80818156843008F0ABC2D7C0BF
:10EEC00082FF34C00091C20F01500093C20F0F5F48
:10EED000809168108F3F09F400C1902F93501091DA
:10EEE000140F8091850E882349F4892F612F44E205
:10EEF00050E099830E940F48025035C020937D0F47
:10EF00008091050F8F3F09F062C04EE1149F900180
:10EF10001124692F70E0F901E05EFE4FE60FF71F44
:10EF200080818156843008F095C23DC09091681070
:10EF300083FF58C00091C20F0F5F0093C20F0150B2
:10EF40009F3F09F4CAC0902F9D5F1091140F8091CC
:10EF5000850E882391F4892F612F44E250E0998334
:10EF60000E940F480C5F802F612F45E250E00E9405
:10EF70000F481F5F9981892F58C020937D0F809182
:10EF8000050F8F3F21F5AEE11A9F90011124692FE3
:10EF900070E0F901E05EFE4FE60FF71F80818156B9
:10EFA000843008F077C28091310F80FF02C0115089
:10EFB00009C081FF02C01F5F05C082FF02C09150DF
:10EFC00001C09F5F9093050F1093320F63C0E091D3
:10EFD0006710F0E0DF01AD5BBF4E9C93E55BF04F47
:10EFE000108371C01091140F1F5F1093140F1150F4
:10EFF0009F3F09F472C0F090C20F912F9D5F8091E6
:10F00000850E8823F1F48F2D692F44E250E0998317
:10F010000E940F480F2D0F5F802F9981692F45E2C5
:10F0200050E00E940F481C5F8F2D612F46E250E098
:10F030000E940F48802F612F47E250E00E940F4846
:10F0400045C020937D0F8091050F8F3F91F5AEE174
:10F050009A9F900111246F2D70E0F901E05EFE4F40
:10F06000E60FF71F80818156843008F03AC2809104
:10F07000310F80FF02C0915009C081FF02C09F5F25
:10F0800005C082FF02C0FA9401C0F394F092050F0C
:10F090009093320F10927C0F8AE580936A10E09172
:10F0A0006710E093370FF0E0E85DF04F80E4808375
:10F0B0000DC0E0916710F0E0DF01AD5BBF4EFC9248
:10F0C000E55BF04F90838FEF8093370F8FEF809346
:10F0D0006810809367101092850E809141108823EC
:10F0E00009F0EBC08091310F90E189278093310FB7
:10F0F0007091140F272F30E06091C20F462F50E01F
:10F10000C901880F991FF90115E0EE0FFF1F1A952D
:10F11000E1F7E81BF90BE40FF51FE05EFE4FE0811D
:10F120008E2F8C51813409F07CC0CA01039762E0B4
:10F1300070E00E94557DE091830E81E8E89FF00128
:10F140001124E60FF11DC901039762E070E00E94EF
:10F15000557D8BE0689FB0011124E60FF71FED5A33
:10F16000F849E491E23459F4409103014E5F409331
:10F1700003018BE16BE00E94D65889E001C086E074
:10F180006FEF41E00E94844C8091C20F6091140F98
:10F190000E94075B8091AC0F81508093AC0F882355
:10F1A00021F5E091440FF0E0E05BF04F81E08083D7
:10F1B0008AE064EB41E00E94844C9091440F9F5F91
:10F1C0009093440F933020F08FEF8093AC0F0DC0DD
:10F1D000E091830E81E8E89FF0011124E90FF11D11
:10F1E000EF52F849E491E093AC0F80914A0F8150BF
:10F1F00080934A0F882309F060C08091820E82FDBF
:10F200005CC088E06FEF40E00E94844C8091820EE9
:10F2100084608093820E81E080937D0F0E94085C61
:10F220004CC0863151F40E940F6A80914E10813299
:10F2300008F043C00E94E06840C08091080F81FF41
:10F2400032C010927E0EE853E230B8F5872F8F5F00
:10F2500090E0FC01B5E0EE0FFF1FBA95E1F7880FD3
:10F26000991FE81BF90BE40FF51FE05EFE4F80814C
:10F270008853823010F56F5F872F90E0FC0155E0D6
:10F28000EE0FFF1F5A95E1F7880F991FE81BF90B46
:10F29000E60FF11DE05EFE4F8081883371F481E05E
:10F2A00080937E0E0AC010927E0E07C010924E1000
:10F2B0008091040F8F5F8093040F8091810E8823CB
:10F2C00009F496C080917D0F882309F091C0809148
:10F2D000C70F882369F480910B0F8F5F80930B0F0A
:10F2E00094E19093C70F843038F010920B0F04C054
:10F2F00081508093C70F7CC08091080F80FF78C039
:10F3000080919C0F63E00E94357D192F1F598091D9
:10F31000FB0E882349F540914F0F8CE3489F9001E5
:10F320001124235A3F4F6BE070E054E619C0842F3C
:10F3300090E0869FF001879FF00D969FF00D1124BD
:10F34000E853F04F80818554843048F4F901E05E41
:10F35000FE4F5083568F1183178F245C3F4F4F5FB2
:10F360008091100F481718F3B0914F0F3BE0E32E38
:10F37000F12C2CE3A22EB12C37C09091FB0E80E033
:10F38000992309F481E0A82FA90F8B2F90E08E9D7F
:10F39000B0018F9D700D9E9D700D11248A9DA0015E
:10F3A0008B9D500D9A9D500D1124435A5F4F685309
:10F3B000704F15C02A2F30E0FB01E20FF31F808150
:10F3C0008554853058F4F901EE0FFF1FE40FF51F47
:10F3D000E05EFE4F10831183168F178FAF5F809111
:10F3E0006610A81738F3BF5F8091100FB81728F286
:10F3F00010927D0F9DC08FEF8093210F16CA8091D0
:10F40000310F90E189278093310F10924E101092A6
:10F41000960F53CFF394AF2DB0E0FA94FD01E05E68
:10F42000FE4FE20FF31F80818156843008F41FCE17
:10F430001250149F90011124205E3E4F620F731FE3
:10F44000FB0180818156843008F411CEA20FB31FD6
:10F450008C9169C00250A02FB0E0FD01E05EFE4F2C
:10F46000E20FF31F80818156843008F49CCD1F5F2A
:10F47000149F900111241150205E3E4F620F731FA4
:10F48000FB0180818156843008F48DCDA20FB31F1B
:10F490008C9122C00C5F402F50E0FA01E05EFE4FDD
:10F4A000E20FF31F80818156843008F47CCD1F5F0A
:10F4B0001A9F900111241150F901E05EFE4FE60FF2
:10F4C000F71F80818156843008F46DCDF901E05E2C
:10F4D000FE4FE40FF51F80818156843008F463CD20
:10F4E00076CDF3944F2D50E0FA94FA01E05EFE4F92
:10F4F000E20FF31F80818156843008F4B8CD1C5F81
:10F500001A9F90011124F901E05EFE4FE60FF71FEC
:10F5100080818156843008F4AACDF901E05EFE4F67
:10F52000E40FF51F80818156843008F4A0CDC1CD51
:10F530000F90CF91DF911F910F91FF90EF90DF908F
:10F54000BF90AF900895A0E0B0E0E9EAFAE70C942C
:10F55000707D182F0E94B45820E030E007C02F5F64
:10F560003F4F849131968F3FD1F71150F901EB57FE
:10F57000FF471123A1F7E901219684910E945F5E64
:10F580008091820E82608093820E0E941C6181E0D5
:10F5900060E00E944D4D8CE390E00E94AE4D92E001
:10F5A000E8E1AE2E74E1B72E62E1C62E51E1D52E10
:10F5B00040E1E42EFE01EB57FF4784918F3F19F4A1
:10F5C0000E94CC5853C02196893010F401E007C046
:10F5D000082F0850FE01EB57FF472196849188239E
:10F5E00079F48091310F84FF03C08E258093310F11
:10F5F0008091310F85FF21C08E258093310F1DC072
:10F60000813019F4D092310F18C0823019F4C092B1
:10F61000310F13C0833019F4B092310F0EC0843013
:10F6200019F4A092310F09C0853011F4905E03C027
:10F63000863019F4905C9093310FF090310F11C027
:10F64000F092310F0E94096E80910E0F83FD0EC063
:10F6500018E004C00E9494710E941C611150D0F700
:10F6600001509F2D002309F4A5CFEACFCDB7DEB717
:10F67000EAE00C948C7DBF92CF92DF92EF92FF92E2
:10F680000F931F938091800E882309F480C180E03E
:10F690000E94D25981E090E00E94AE4DECE2F4E08D
:10F6A00080EF8083359694E0E43AF907D1F76EE372
:10F6B00070E01AC08491865F8D939F5F31969D3074
:10F6C000C9F7425E5F4F235F3F4FE4E029363E07B4
:10F6D00031F0DA01A05EBE4FF90190E0EBCF635F3D
:10F6E0007F4F6835710521F027EE33E0AB01F1CF94
:10F6F00081E090E00E94AE4D4AE050E029E634E01F
:10F70000DA0166E0AA0FBB1F6A95E1F7AC55BB4F63
:10F7100005C0F90184918D932F5F3F4FF4E0293AA2
:10F720003F07B9F74F5F5F4F4A31510539F784E022
:10F7300061E00E944D4D88E08093310F1092C20F1E
:10F7400080EA8093140FFF24EE24E394BB24B39447
:10F7500040E4C42E30EFD32E70C080E28F1588F1C4
:10F76000EE2071F18F2D90E0FC01E955FF4FDC0197
:10F77000AC59B84F895D9B4F08C024912F3F09F0C9
:10F780002C93E05CFF4FA05CBF4FE817F907A9F787
:10F790008C2D8F1990E0FC01E955FF4FDC01AC592D
:10F7A000B84F895D9B4F08C024912F3F09F02C93DF
:10F7B000E05CFF4FA05CBF4FE817F907A9F7F3948F
:10F7C000EB243E5F3093C20F80914E108F5F809389
:10F7D0004E10883010F010924E100E949358809175
:10F7E000C20F803930F4805F6091140F4EE20E94A6
:10F7F000415681E090E00E94AE4DE0E4F4E0D0821A
:10F80000359694E0E43AF907D1F78091C20F803938
:10F81000A1F484E164E147E024E00DEF1FEF0E94D2
:10F82000785987E165E142E157E60E94586087E137
:10F8300067E146E157E60E9458603091C20F363AC0
:10F8400008F48BCF82E08093310FA1C00E94E56E57
:10F8500080910E0FE1E0FE16A9F484FF2BC0809189
:10F860000C0F90910D0F24E0969587952A95E1F75E
:10F8700081708F15F9F086E062E341E00E94844CCC
:10F88000FF2415C085FF16C080910C0F90910D0FBD
:10F89000B5E096958795BA95E1F781708E1551F090
:10F8A00086E062E341E00E94844CFF24F39400E090
:10F8B00010E02FC080910E0F83FF2BC080910C0FA2
:10F8C00083FD27C085E06FE641E00E94844C1092E2
:10F8D0004E101092830E0E94935881E08093800E08
:10F8E000FF2061F410927F0E1092800E80E18093D1
:10F8F000820E83E061E00E94654D06C0F1E0FF16D4
:10F9000019F482E080937F0E82E090E00E94AE4D79
:10F9100049C08F2D90E0A4E0880F991FAA95E1F7C8
:10F920008C558093140F8091960F882321F081507D
:10F930008093960F07C080914E108F5F80934E107A
:10F94000D092960F80914E10883010F010924E1089
:10F950000E9493580F5F1F4F8091870E803418F0DC
:10F960001092870E03C08F5F8093870E81E090E036
:10F970000E94AE4D81E00936180774F080E00E94C5
:10F98000A37A81E080937F0E8093800E0BC0FF24CA
:10F9900000E010E0F3E0DF2EE0907F0E91E0E9164A
:10F9A00009F454CF1F910F91FF90EF90DF90CF900B
:10F9B000BF90089580917F0E882371F0823039F0D6
:10F9C000843041F0813041F40E943B7B08950E94D5
:10F9D0004D6F08950E94196E08951F930E94054867
:10F9E000ECE2F4E080EF8083359694E0E43AF907A6
:10F9F000D1F710927F0E11E01093800E10924E10EE
:10FA00001092830E1092840E80E18093820E8FE814
:10FA10009AE50E94F84889E290E30E94004889E64E
:10FA200094E00E941D480E949C6482E195E60E9439
:10FA3000134910937F0E8FEF8093210F80936810EE
:10FA40008093431080934410809345108093461018
:10FA50001092F60E1092FA0E0E94E56E0E94DA7C69
:10FA60000E9494710E941C61F7CF991B79E004C039
:10FA7000991F961708F0961B881F7A95C9F78095ED
:10FA80000895AA1BBB1B51E107C0AA1FBB1FA617E5
:10FA9000B70710F0A61BB70B881F991F5A95A9F737
:10FAA00080959095BC01CD01089597FB092E0726FE
:10FAB0000AD077FD04D0E5DF06D000201AF4709557
:10FAC00061957F4F0895F6F7909581959F4F089522
:10FAD0002F923F924F925F926F927F928F929F925E
:10FAE000AF92BF92CF92DF92EF92FF920F931F934C
:10FAF000CF93DF93CDB7DEB7CA1BDB0B0FB6F894FD
:10FB0000DEBF0FBECDBF09942A88398848885F843C
:10FB10006E847D848C849B84AA84B984C884DF80AD
:10FB2000EE80FD800C811B81AA81B981CE0FD11D91
:10FB30000FB6F894DEBF0FBECDBFED010895F89467
:02FB4000FFCFF5
:06FB4200010101150400A1
:00000001FF
